:020000040000fa
:080000000002040000000000f2
:020000040000fa
:040008004c030000a5
:020000040000fa
:04000c004c030000a1
:020000040000fa
:040010004c0300009d
:020000040000fa
:040014004c03000099
:020000040000fa
:040018004c03000095
:020000040000fa
:04001c004c03000091
:020000040000fa
:040020004c0300008d
:020000040000fa
:040024004c03000089
:020000040000fa
:040028004c03000085
:020000040000fa
:04002c004c03000081
:020000040000fa
:040030004c0300007d
:020000040000fa
:040034004c03000079
:020000040000fa
:040038004c03000075
:020000040000fa
:04003c004c03000071
:020000040000fa
:040040004c0300006d
:020000040000fa
:040044004c03000069
:020000040000fa
:040048004c03000065
:020000040000fa
:04004c004c03000061
:020000040000fa
:040050004c0300005d
:020000040000fa
:04005400b473000081
:020000040000fa
:04005800dc73000055
:020000040000fa
:04005c004c03000051
:020000040000fa
:040060004c0300004d
:020000040000fa
:040064004c03000049
:020000040000fa
:040068004c03000045
:020000040000fa
:04006c004c03000041
:020000040000fa
:040070004c0300003d
:020000040000fa
:040074004c03000039
:020000040000fa
:040078004c03000035
:020000040000fa
:04007c004c03000031
:020000040000fa
:040080004c0300002d
:020000040000fa
:040084004c03000029
:020000040000fa
:040088004c03000025
:020000040000fa
:04008c004c03000021
:020000040000fa
:040090004c0300001d
:020000040000fa
:040094004c03000019
:020000040000fa
:040098004c03000015
:020000040000fa
:04009c004c03000011
:020000040000fa
:0400a0004c0300000d
:020000040000fa
:0400a4004c03000009
:020000040000fa
:0400a8004c03000005
:020000040000fa
:0400ac004c03000001
:020000040000fa
:0400b0004c030000fd
:020000040000fa
:0400b4004c030000f9
:020000040000fa
:0400b8004c030000f5
:020000040000fa
:0400bc004c030000f1
:020000040000fa
:0400c0004c030000ed
:020000040000fa
:0400c4004c030000e9
:020000040000fa
:0400c8004c030000e5
:020000040000fa
:0400cc004c030000e1
:020000040000fa
:0400d0004c030000dd
:020000040000fa
:0400d4004c030000d9
:020000040000fa
:0400d8004c030000d5
:020000040000fa
:0400dc004c030000d1
:020000040000fa
:0400e0004c030000cd
:020000040000fa
:0400e4004c030000c9
:020000040000fa
:0400e8004c030000c5
:020000040000fa
:0400ec004c030000c1
:020000040000fa
:0400f0004c030000bd
:020000040000fa
:0400f4004c030000b9
:020000040000fa
:0400f8004c030000b5
:020000040000fa
:0400fc004c030000b1
:020000040000fa
:040100004c030000ac
:020000040000fa
:040104004c030000a8
:020000040000fa
:040108004c030000a4
:020000040000fa
:04010c004c030000a0
:020000040000fa
:040110004c0300009c
:020000040000fa
:040114004c03000098
:020000040000fa
:040118004c03000094
:020000040000fa
:04011c004c03000090
:020000040000fa
:040120004c0300008c
:020000040000fa
:040124004c03000088
:020000040000fa
:040128004c03000084
:020000040000fa
:04012c004c03000080
:020000040000fa
:040130004c0300007c
:020000040000fa
:040134004c03000078
:020000040000fa
:040138004c03000074
:020000040000fa
:04013c004c03000070
:020000040000fa
:040140004c0300006c
:020000040000fa
:040144004c03000068
:020000040000fa
:040148004c03000064
:020000040000fa
:040208004c030000a3
:020000040000fa
:04020c004c0300009f
:020000040000fa
:040210004c0300009b
:020000040000fa
:040214004c03000097
:020000040000fa
:040218004c03000093
:020000040000fa
:04021c004c0300008f
:020000040000fa
:040220004c0300008b
:020000040000fa
:040224004c03000087
:020000040000fa
:040228004c03000083
:020000040000fa
:04022c004c0300007f
:020000040000fa
:040230004c0300007b
:020000040000fa
:040234004c03000077
:020000040000fa
:040238004c03000073
:020000040000fa
:04023c004c0300006f
:020000040000fa
:040240004c0300006b
:020000040000fa
:040244004c03000067
:020000040000fa
:040248004c03000063
:020000040000fa
:04024c004c0300005f
:020000040000fa
:040250004c0300005b
:020000040000fa
:040254004c03000057
:020000040000fa
:040258004c03000053
:020000040000fa
:04025c004c0300004f
:020000040000fa
:040260004c0300004b
:020000040000fa
:040264004c03000047
:020000040000fa
:040268004c03000043
:020000040000fa
:04026c004c0300003f
:020000040000fa
:040270004c0300003b
:020000040000fa
:040274004c03000037
:020000040000fa
:040278004c03000033
:020000040000fa
:04027c004c0300002f
:020000040000fa
:040280004c0300002b
:020000040000fa
:040284004c03000027
:020000040000fa
:040288004c03000023
:020000040000fa
:04028c004c0300001f
:020000040000fa
:040290004c0300001b
:020000040000fa
:040294004c03000017
:020000040000fa
:040298004c03000013
:020000040000fa
:04029c004c0300000f
:020000040000fa
:0402a0004c0300000b
:020000040000fa
:0402a4004c03000007
:020000040000fa
:0402a8004c03000003
:020000040000fa
:0402ac004c030000ff
:020000040000fa
:0402b0004c030000fb
:020000040000fa
:0402b4004c030000f7
:020000040000fa
:0402b8004c030000f3
:020000040000fa
:0402bc004c030000ef
:020000040000fa
:0402c0004c030000eb
:020000040000fa
:0402c4004c030000e7
:020000040000fa
:0402c8004c030000e3
:020000040000fa
:0402cc004c030000df
:020000040000fa
:0402d0004c030000db
:020000040000fa
:0402d4004c030000d7
:020000040000fa
:0402d8004c030000d3
:020000040000fa
:0402dc004c030000cf
:020000040000fa
:0402e0004c030000cb
:020000040000fa
:0402e4004c030000c7
:020000040000fa
:0402e8004c030000c3
:020000040000fa
:0402ec004c030000bf
:020000040000fa
:0402f0004c030000bb
:020000040000fa
:0402f4004c030000b7
:020000040000fa
:0402f8004c030000b3
:020000040000fa
:0402fc004c030000af
:020000040000fa
:040300004c030000aa
:020000040000fa
:040304004c030000a6
:020000040000fa
:040308004c030000a2
:020000040000fa
:04030c004c0300009e
:020000040000fa
:040310004c0300009a
:020000040000fa
:040314004c03000096
:020000040000fa
:040318004c03000092
:020000040000fa
:04031c004c0300008e
:020000040000fa
:040320004c0300008a
:020000040000fa
:040324004c03000086
:020000040000fa
:040328004c03000082
:020000040000fa
:04032c004c0300007e
:020000040000fa
:040330004c0300007a
:020000040000fa
:040334004c03000076
:020000040000fa
:040338004c03000072
:020000040000fa
:04033c004c0300006e
:020000040000fa
:040340004c0300006a
:020000040000fa
:040344004c03000066
:020000040000fa
:040348004c03000062
:020000040000fa
:10040000efa321000e7f22000e01880000000000f3
:10041000000020000000e000020032000001200087
:10042000200288000c00070060d92800010020008d
:1004300011000700000020000000e0000200320070
:1004400000000200000000009a8f0200000000007f
:100450000040da000000fe004440a900002a20000d
:100460000000e0000300320000002000a00188002e
:100470004440a80000000600910188008000780038
:100480000000eb0015003700e280400032a0b4000d
:100490009101ba00e280400032a0b4009102ba009b
:1004a000e280400032a0b4000002eb00472bde00e7
:1004b000f507b200602ce10004003a000059eb009f
:1004c0008301e900fdff3e00040037006128e100e0
:1004d000010032000082eb000b00070011c3ba00dc
:1004e0001101ba000604e00003003a000200e00037
:1004f000e5ff3a0000000600f607b200960188000a
:1005000082007800f5ff37003159ba008301e90015
:100510000c0032002159ba008301e90008003200c2
:100520000400e00003003a00e280400032a0b40082
:10053000f5ff370011d9ba008301e900faff3a004c
:100540008100e800e180400032a0b4000000060015
:10055000000000000000000000000000000000009b
:10056000000000000000000000000000000000008b
:10057000000000000000000000000000000000007b
:10058000000000000000000000000000000000006b
:10059000000000000000000000000000000000005b
:1005a000000000000000000000000000000000004b
:1005b000000000000000000000000000000000003b
:1005c000000000000000000000000000000000002b
:1005d000000000000000000000000000000000001b
:1005e000000000000000000000000000000000000b
:1005f00000000000000000000000000000000000fb
:1006000000000000000000000000000000000000ea
:1006100000000000000000000000000000000000da
:1006200000000000000000000000000000000000ca
:1006300000000000000000000000000000000000ba
:1006400000000000000000000000000000000000aa
:10065000000000000000000000000000000000009a
:10066000000000000000000000000000000000008a
:10067000000000000000000000000000000000007a
:10068000000000000000000000000000000000006a
:1006900000000000000000000040da000000fe0042
:1006a00003f0a200889fbe008a9fbe008c1f7800c6
:1006b0004a010700510133006450e1004f0032004d
:1006c0006420e1005200320003826c0007003b000e
:1006d0000905d0000306d000820f54000c065d000f
:1006e0000200390002003200890178000306780018
:1006f0008582550004003d000003fd008103fd00dc
:100700008502ea008b854200840f720002003b00e4
:1007100060001000e08018006011b8000005eb00d8
:100720007a28e1000a00390006007800c75ddd0084
:10073000f707b200878075002d00370082817100b5
:100740000a017800610560008180d1000080d3003b
:100750008502e900f9ff3b00060440008784480059
:1007600002003b0060041400e0841c000988a30020
:10077000070032008a81710082817100610164008a
:100780008904d1000884d3008b05e80017003700e6
:100790000978a30013003a000b00e00013003400b6
:1007a0008b05e9000804440089844c000a44740065
:1007b0000978a3000d003a000b00e00007003400a8
:1007c0008b05e9000804440089844c0001003a00cc
:1007d0000b0020000978a300f7ff32000001eb00b6
:1007e00002003700828171000a017800c000070012
:1007f0000cf0a70001f0a000090137006420e1001f
:1008000002003a00838f6c00090133000801be002a
:100810000200be0002013700889fbe008a9fbe0012
:100820008c1f7800ed000700f400330003866c0095
:100830006450e1002e0032006420e10033003200f9
:100840006150e1002f0032006120e10031003200f0
:1008500085855500eb07b000090020000804200042
:10086000050037000804440089844c000a00310068
:100870000603430087834b000001530081815b0026
:10088000f8ff33000203be000800a0000804440083
:1008900089844c00f6ff3900c639dd0083017300fe
:1008a00001003200130020008904d1000884d30025
:1008b0000998a300050032000800a7000300a0006b
:1008c0008904d1000884d3008b05e8008904d10095
:1008d0000884d3000001eb000281d20084000700ed
:1008e00001f0a1000cf0a70001f0a000cc0037003f
:1008f0006420e100ce0032000801be000200be000c
:10090000f7ff37006120e100c90032006000b80045
:10091000f3ff37000000200001f82700f0ff370048
:10092000140020000e023700f4ff2f000c023700e5
:100930000003be00940007006011b8000470a70017
:1009400007f0a10007f8a30017003a006509b100fd
:100950000d0032000d003500860220000628e1005f
:1009600003003500030028006000b8000200050005
:100970000000400081804800020149008381490055
:100980008502e900faff3a0000000600f88f4200f5
:10099000050034008100d1000080d3008502e8000a
:1009a000fcff3a00000006006011b8008000eb0078
:1009b000000005000001be00730007000470a700de
:1009c00003f0a10003f8a30013003a006509b10089
:1009d00010003200090035006928e10002003500ee
:1009e0000100280000000500000040008180480050
:1009f0008502e900fcff3a0000000600f88f420083
:100a0000050035008100d1000080d3008502e80098
:100a1000fcff3a00000006008000eb00000005002b
:100a20004f89de0082017800e8013700889fbe0010
:100a30008a9fbe000082700004027100048271006f
:100a4000260032000004be000200be006011b800a3
:100a50006b092000950220000182cf000a003900b6
:100a60000541b1000082cf00070039000541b10007
:100a70000982cf00040039000541b1000882cf008f
:100a8000010039000541b100054252001200320058
:100a90000a003b0082817100610164008100d10085
:100aa0000080d3008984d3000884d3008b05e8003c
:100ab0000442e800f7ff3a0007003700080444004a
:100ac00089844c0000004800818048008b05e900c3
:100ad0000442e900f9ff3a00050007004f05be0097
:100ae0004f04be00000006006011b800cfff3700c1
:100af00081002000618055000b003d000b002000ac
:100b000061fe2f000100e1001d00340082817100b0
:100b1000610164008904d1000884d3000000e8006a
:100b2000faff3a00710020006100640003007000c9
:100b3000020060000900320061044400e0844c00bf
:100b40000988a500050032008b05e8006808e1006f
:100b500002003a008904d1000884d300f20f20007b
:100b60000258e10005003d00c75ddd00f907b20055
:100b70008980750008007800000006000bf8270047
:100b80008b00780000000500c70ade00f107b20004
:100b9000f50fb20008003200e1cf4200020032003f
:100ba0000170a00024000500810f700001003200d8
:100bb0000408050044000500810f700002003a009f
:100bc000140005008502e9000000400081c04800d3
:100bd000fcff3b000170a000240005000004be00e3
:100be000e9ff07000003be000405be000200be00ce
:100bf000e5ff0700844f7500000006000200be00fc
:100c00006450e100050036006420e1000200360077
:100c10000968a30001003a000800be000160a000be
:100c20004f0678004f05be004f04be0000000600ce
:100c3000f0ff2f00f1ff2700f9ff3700889fbe006b
:100c40008a9fbe008c1f7800e4ff0700ebff330093
:100c500003866c006450e100240032006420e1004f
:100c6000270032006150e100220032006120e100e3
:100c7000210032008b854200eb07b1000134b8003f
:100c8000003ab8000804420089844a00013ab800da
:100c90000030b8008880400009014a000400330099
:100ca0000000400081804800020149008b05e900f6
:100cb000c909dd008301700001003200130020002b
:100cc000c814de004814dd004709de001200b2003f
:100cd000c808de000884700085ff070001f0a1004d
:100ce0000cf0a70001f0a000cdff37006120e1006b
:100cf000cfff32000801be000200be00f7ff370040
:100d00006150e100fcff3a00c9ff37006022b800e3
:100d1000060220000000d0008180d2000482d200b0
:100d20008582d2000000a0000202520083825a0095
:100d3000030031000202420083824a000000a10049
:100d40000603e900f3ff3a0000000600efff07008a
:100d50000400be0000000600889fbe008a9fbe00ff
:100d600030044200b0844a0030054b0090854b00af
:100d70006000b1000898be000a90be000440e10087
:100d800005c8e10006d0e10007d8e100020031000b
:100d9000680040001008e8004f05be004f04be0088
:100da00000000600889fbe008a9fbe003004be007f
:100db0002005be000418540005985c0006185d006c
:100dc00007985d00110020000440e10005c8e10023
:100dd00006d0e10007d8e100010039008000eb00f7
:100de000108810004f05be004f04be000000060032
:100df0001200fa00889fbe008a9fbe008c9fbe0032
:100e0000e0b79f00f1b79f0082bf9f0093bf9f0094
:100e10000605be000404be000000eb00d0b79f0032
:100e2000c0b79f00b0b79f00a0b79f0090b79f00ca
:100e30000006eb005fb19700cfb097008201410040
:100e40003fb097000200e00004003d0037000700bb
:100e50007e805700c0ff0700030037003300070003
:100e60007e805700cfff0700dfb697000d00e0003f
:100e70000c0035006fb29700ffb297000fbb9700d0
:100e80009fbb970010002000010020006011b800f7
:100e90000002720081827200020373008383730078
:100ea0001b0007000c06e80001042000810f56001b
:100eb000e0ff3a000d00e00004003d000802be0023
:100ec0000a03be007e805700a3ff07005fa89700bb
:100ed0000000e00005003a001fb29700afb2970093
:100ee0003fb39700cfb39700090007006fb097009a
:100ef000ffb097000fb997009fb997004f06be004b
:100f00004f05be004f04be000080fa00000006003e
:100f10000100070000000600a4b79f00b5b79f00be
:100f2000c6b79f00d7b79f00000006004f09de003c
:100f300082817100b3b79f004f01de0081804000c5
:100f400082807000a1b79f008fb097004f09de002c
:100f5000000040000200700090b79f007fa897003b
:100f60004f01de00818040008280700081b79f00c9
:100f70000d0007004f3ade00000040000400700042
:100f8000f0af9f00080007000402420085824a007b
:100f900006034b0087834b00dfff07000802be00fb
:100fa0000a03be00000006002fb29700bfb29700f0
:100fb0004fb39700dfb3970000000600881f78004a
:100fc00018002000881f780089ff07008f87e9003c
:100fd0004f04780000000600801feb0084ff07002c
:100fe0008f87e90000000600889fbe008a9fbe0030
:100ff000e00f5000e08f5800e00f5900e08f5900db
:101000000c003d006044b8006055b800000054007a
:1010100081805c0002015d0083815d00180020007a
:101020001500070008003d00180007000004eb0051
:10103000050037000004eb000f00070002003d0030
:101040001200070018002000dcff07000800e00085
:10105000060032006022b8006033b8000000520081
:1010600081805a0002015b0083815b004f05be0056
:101070004f04be0000000600e00f5200e08f5a004f
:10108000e00f5b00e08f5b00000006006044b800ea
:101090006055b8000402540085825c0006035d00c0
:1010a00087835d0000000600889fbe008a9fbe0007
:1010b0008c1f7800e00f5000e08f5800e00f5900bf
:1010c000e08f59000d003d006044b8006055b80045
:1010d0000000540081805c0002015d0083815d009e
:1010e0001c0020000820e10009a8e1000ab0e1008e
:1010f0000bb8e1000d003d00080037000006eb00d2
:10110000e00f5200e08f5a00e00f5b00e08f5b00c1
:1011100006003d006044b8006055b8000402540069
:1011200085825c0006035d0087835d00aaff0700df
:101130000c00e000060032006022b8006033b80006
:101140000000520081805a0002015b0083815b0035
:101150004f0678004f05be004f04be000000060099
:10116000889fbe008a9fbe00841f78009bfe0700f8
:101170004f00780011003300f0ff2f00838f6c00c8
:1011800006003b00040565000a00a70008003700c0
:1011900009f0a6001000200008003700820f54005c
:1011a000838f5c00030039001000200001003e0026
:1011b0000000200009f0a7000000ea004f05be0073
:1011c0004f04be000000e00000000600881f780009
:1011d000030478000300e00007003d0060001000f9
:1011e000e080180060011900e081190002003b0056
:1011f00001f02d00030037000cfe070008f0a700e7
:0c12000001f0a0004f0478000000060080
:020000040000fa
:10120c003e00000008200000080000001b5b0000ee
:10121c00440000001b5b000000440000001b0000a9
:10122c005b430000001b00005b3200004b0d000014
:10123c0000430000000000001b5b00003244000073
:10124c0000570000617200006e6900006e670000bc
:10125c003a2000006e6f0000207600006f6c0000da
:10126c007461000067650000206f00006e200000b4
:10127c0056700000756c00006c750000702000004a
:10128c00706900006e000000203d0000200000008e
:10129c00436c00007574000063680000206500005a
:1012ac006e6700006167000065640000212100008a
:1012bc002100000056520000454700002074000039
:1012cc006f6f0000206c00006f7700002c20000076
:1012dc0069730000207400006865000072650000ee
:1012ec002061000020730000686f00007274000021
:1012fc003f000000436c0000757400006368000040
:10130c002064000069730000656e000067610000d6
:10131c00676500006421000021210000002e000000
:10132c00203c0000002e000020000000546f000044
:10133c0020660000696e00006973000068200000e0
:10134c007365000074750000702c000020730000a1
:10135c0074610000727400002075000070200000a1
:10136c007468000065200000706f00007765000055
:10137c007220000073750000707000006c69000032
:10138c00657300002077000069740000682000007d
:10139c00636f00006d6d0000616e00006420000042
:1013ac0027570000270d00000a0000002000000055
:1013bc000d0a00002800000078000000293e000003
:1013cc00004200007573000020500000697200009c
:1013dc0061740000652000007633000000200000de
:1013ec00636c00006f6e000065200000772f00001a
:1013fc00646900006666000065720000656e00009e
:10140c00742000005049000043000000436f0000ae
:10141c006d6d0000756e000069740000792000008d
:10142c0046690000726d0000776100007265000073
:10143c0020760000372e0000302000002d20000008
:10144c00676f00006f2e0000676c00002f670000b4
:10145c00437a0000516e000057200000002000006d
:10146c0028320000344600004a36000034470000a1
:10147c004130000030000000342000000032000039
:10148c002000000041330000004200003400000046
:10149c00423500000042000038000000554e0000ac
:1014ac004b0000002900000049090000004f00001b
:1014bc000900000048090000004c00000900000071
:1014cc00456e00007465000072200000726100001f
:1014dc0077200000766100006c750000652000002c
:1014ec00666f0000722000004252000047000000ae
:1014fc0014340000040d00008206000040030000bc
:10150c00a0010000cf0000006700000044000000b4
:10151c00220000007f00000000000000000000001e
:10152c00000000002c010000000000005802000028
:10153c0000000000b0040000000000006009000082
:10154c0000000000c0120000000000008025000018
:10155c00000000004038000000000000004b0000bc
:10156c0000000000807000000000000000960000e9
:10157c0000000000c0da00000000000000e10000e4
:10158c000000000000c200000100000000f4000098
:10159c000100000000e8000003000000143400000b
:1015ac00040d00008206000040030000a0010000b2
:1015bc00cf0000007f000000670000004400000026
:1015cc0022000000415200005431000000000000d5
:1015dc00204800007a00000046720000657100008f
:1015ec00756500006e6300006965000073200000e3
:1015fc003c200000314800007a200000617200009d
:10160c00652000006e6f00007420000073750000f0
:10161c00707000006f72000074650000642e000092
:10162c0000000000001800001c1d0000436f0000ab
:10163c00756c0000646e000027740000206b0000c5
:10164c00656500007020000075700000000000004f
:10165c00001800001c1d0000030b0000131b0000f1
:10166c0053500000493100000000000030780000a9
:10167c0030310000323300003435000036370000c2
:10168c003839000041420000434400004546000048
:10169c003062000000300000303000002c000000f0
:1016ac0030300000000000000142000050760000c5
:1016bc003300000021000000001000000023000097
:1016cc00000f0000424000004005000041020000f5
:1016dc0000310000414c00005300000000290000c4
:1016ec0000200000570000002052000000490000bc
:1016fc003243000031000000080800000808000018
:10170c00080000000000000042420000494f0000a9
:10171c003100000052410000573100000000000071
:10172c00353f000062610000000000004f430000e4
:10173c004431000000000000000000000000000028
:020000040000fa
:10174c002000fa000000eb00000f78000000eb0016
:10175c0010c488000000eb0000c4880001c48000a5
:10176c00210f98000000eb00300f98000000eb00f8
:10177c00400f98000000eb00b0cf88000000eb0099
:10178c00000f9800408821008040eb000148780051
:10179c000000eb00100f98000000eb001007980001
:1017ac000000eb00200798000000eb0030079800c9
:1017bc000040eb00205f98000040eb00305f980089
:1017cc000000eb0060079800150037000000eb00ec
:1017dc00700798000c0037006e00900052882100b2
:1017ec007800b900800078007e00900000804000f6
:1017fc00000041008040eb00014878007e00900022
:10180c000000e800700798007e009000ff0f500069
:10181c00f1ff34006e0090000000e80060079800b3
:10182c006e009000e20f5000e8ff34000000eb0067
:10183c0070c68800b1cf8000000320000088b9007a
:10184c00000078008102200080804000008d210083
:10185c0000804000f26d0200000000006090280043
:10186c00f26d0200000000002a04370070c68000f0
:10187c000000e0006500320070c680000000e90046
:10188c0070c688000000eb00700798001d00370040
:10189c0002c4800070c680007800b9008000780017
:1018ac007e0090000080400051882100e1407800cb
:1018bc00008021000170790070c680007800b900aa
:1018cc00800078007e00900000804000518821004c
:1018dc00614078002c7302000000000000c48000fe
:1018ec000000e80000c488007e0090000000e800c2
:1018fc007007980001c48000f00720000080600091
:10190c0000c4880070c680007800b90080007800a0
:10191c007e009000008040005188210061407800da
:10192c000004e000daff3a000000eb0070c688000b
:10193c0037003700809c2100104078006440600024
:10194c000004e00032003200b1cf80000003200020
:10195c000088b90000007800fa004000008d2100da
:10196c000080400010007800000001000004e0003e
:10197c0027003200b1cf8000000320000088b9009e
:10198c00000078008102200080804000008d210042
:10199c0000804000f26d0200000000006090280002
:1019ac00f26d02000000000011c4800000c4800031
:1019bc00808f50001600320010c480007007980011
:1019cc000d003700018021007e0090000080400057
:1019dc00104078002c73020000000000fe00900004
:1019ec00f007200000806000700798007e009000d7
:1019fc000000e80070079800fe00900000c4800012
:101a0c00808f5000efff3a0001003700000000000b
:101a1c0036720200000000000004e000c5ff320036
:101a2c005e730200000000000004e00003003200be
:101a3c006a73020000000000b60337000673020050
:101a4c0000000000405f98004e5890000080fb00a2
:101a5c00cf80de00f207200003002000820f500030
:101a6c00838f580031033e000060010026033700cd
:101a7c00d90237004f0137002c033700d70037004d
:101a8c00f202370065013700280337007700370072
:101a9c0026033700090337002403370023033700dc
:101aac000603370008023700200337006d013700aa
:101abc001e0337001d0337001c0337001b033700c0
:101acc001a033700190337001803370017033700c0
:101adc0016033700150337000101370013033700d5
:101aec001203370011033700100337000f033700c0
:101afc000e0337000d0337000c0337000b033700c0
:101b0c000a033700090337000803370007033700bf
:101b1c0006033700050337000403370003033700bf
:101b2c00020337000103370000033700ff023700c0
:101b3c00fe023700fd023700fc023700fb023700c3
:101b4c00fa023700f9023700f8023700f7023700c3
:101b5c00f6023700f5023700f4023700f3023700c3
:101b6c00f2023700f1023700f0023700ef023700c3
:101b7c00ee023700ed023700ec023700eb023700c3
:101b8c00ea023700e9023700e8023700e7023700c3
:101b9c00e6023700e5023700e4023700e3023700c3
:101bac00e2023700e1023700e0023700df023700c3
:101bbc00de023700dd023700dc023700db023700c3
:101bcc00da023700d9023700d8023700d7023700c3
:101bdc00d6023700d5023700d4023700d3023700c3
:101bec00d2023700d1023700d0023700cf023700c3
:101bfc00ce023700cd023700cc023700cb023700c3
:101c0c00ca023700c9023700c8023700c7023700c2
:101c1c00c6023700c5023700c4023700c3023700c2
:101c2c00c2023700c1023700c0023700bf023700c2
:101c3c00be023700bd023700bc023700bb023700c2
:101c4c00ba023700b9023700b8023700b7023700c2
:101c5c00b6023700b5023700b4023700b3023700c2
:101c6c00b2023700b10237005c00370010c48000ac
:101c7c00ae089000808f50005400320000c48000e9
:101c8c00ae089000808f50000f003a0000c4800016
:101c9c008000e900f00720000080600000c488008c
:101cac0000c48000018021000041eb0082707800ac
:101cbc0001c48000210f980080902800f26d020072
:101ccc0000000000130337000000eb0060079800d1
:101cdc002e0890008000e900f007200000806000d2
:101cec00200f9800c0902800f26d02000000000048
:101cfc00ae08900071079800200037007e0090001d
:101d0c000000e80001802100e14078000280210001
:101d1c007e00900000004100014878000180210005
:101d2c007e00900000804000104078000004e0002d
:101d3c0007003200018021007e00900000804000ee
:101d4c00104078002c7302000000000003003700e4
:101d5c0000c2b3002c730200000000006e00900063
:101d6c000000e800600798007e0090008000e8000a
:101d7c00f00720000080600070079800fe009000c3
:101d8c0000c48000808f5000dcff3a0000c480004b
:101d9c008000e900f00720000080600000c488008b
:101dac0000912800f26d0200000000006e0090000f
:101dbc000040780084700200000000003091280080
:101dcc00f26d020000000000d202370070c0b300b8
:101ddc002c73020000000000ce02370000c480000b
:101dec00ae089000808f5000390032000000eb00ec
:101dfc0060079800ae08900071079800200037002b
:101e0c007e0090000000e80001802100e140780095
:101e1c00028021007e009000000041000148780003
:101e2c00018021007e00900000804000104078006e
:101e3c000004e00007003200018021007e009000c9
:101e4c0000804000104078002c730200000000005d
:101e5c000300370000c2b3002c7302000000000026
:101e6c006e0090000000e800600798007e00900073
:101e7c008000e800f00720000080600070079800e8
:101e8c00fe00900000c48000808f5000dcff3a0000
:101e9c0000c480008000e900f00720000080600092
:101eac0000c4880000912800f26d020000000000c0
:101ebc006e0090000040780084700200000000006a
:101ecc0030912800f26d02000000000091023700f2
:101edc0070c0b3002c730200000000008d023700ac
:101eec000673020000000000405f9800ce5890007e
:101efc00b0c5b30080cf50007f023a0006730200d9
:101f0c0000000000405f98004e5890000080fb00dd
:101f1c0011042000810f50005100320011042000e8
:101f2c00810f500007003c0011032000810f50006e
:101f3c000e00320041032000810f500013003200cc
:101f4c007402370031042000810f5000320032003f
:101f5c0031042000810f5000da00350041042000cc
:101f6c00810f5000120032006a0237000673020023
:101f7c0000000000405f9800ce589000e0c7b3000e
:101f8c0080cf500093013200080037000673020026
:101f9c0000000000405f9800ce589000e0c7b300ee
:101fac0080cf5000a8013200000000005902370019
:101fbc00000000001e089000e40f500005003400e3
:101fcc004e870200000000000000eb00100f98008c
:101fdc005002370010c48000ae089000808f500073
:101fec00090032002e0890008000e900f007200064
:101ffc0000806000200f9800c0902800f26d020055
:10200c00000000004302370070c0b3002c730200c4
:10201c00000000003f0237000000000000c48000f8
:10202c00ae089000808f5000090032002e089000fe
:10203c008000e800f007200000806000200f98006e
:10204c0050912800f26d02000000000031023700b0
:10205c0070c0b3002c730200000000002d0237008a
:10206c00000000000000eb00400f980010c480003e
:10207c000000e90080007800f0072000008060007c
:10208c007007980083003700018021007e009000cb
:10209c0000804000104078000004e00078003a0016
:1020ac007e0090008000e900f007200000806000b6
:1020bc0001802100614078000004e00070003200d3
:1020cc004e0890000000e800400f9800ce089000e9
:1020dc003e089000808f5000690036003e0890004a
:1020ec000000e800300f980011c4800000c480008c
:1020fc00808f5000120032000900370000c48000ad
:10210c00018021000041eb008270780000c4800047
:10211c008000e900f00720000080600000c4880007
:10212c0001c4800010c48000808f5000f3ff3a007f
:10213c0000c48000018021000041eb008270780017
:10214c007e0090008000e900f00720000080600015
:10215c006007980011003700018021006e0090008c
:10216c0000804000104078000004e00006003a00b7
:10217c006e0090008000e800f007200000806000f6
:10218c00000f9800090037006e0090008000e900f5
:10219c00f00720000080600060079800ee009000bf
:1021ac0000c48000808f5000ebff3a009091280013
:1021bc00f26d020000000000b1cf8000000320008f
:1021cc000088b90000007800810220008080400067
:1021dc00008d210000804000f26d02000000000024
:1021ec0060902800f26d0200000000008e08900044
:1021fc006107980017003700018021006e009000e5
:10220c0000804000104078002c7302000000000099
:10221c0000c4800002802100ee009000810041008b
:10222c0011417800018021008270780000c4800088
:10223c008000e800f00720000080600000c48800e7
:10224c006e0090008000e800f00720000080600025
:10225c0060079800ee0090007e009000808f500088
:10226c00e5ff3a0000c48000018021000041eb0032
:10227c008270780001c48000210f9800090037009b
:10228c007e0090008000e900f007200000806000d4
:10229c0070079800fe00900000c48000808f5000f2
:1022ac0079ff3a00fe00900000c48000808f50003f
:1022bc0093013a0070c0b3002c73020000000000c0
:1022cc0094013700000000000000eb00400f980064
:1022dc0010c480000000e90080007800f0072000a6
:1022ec000080600070079800840037000180210096
:1022fc007e00900000804000104078000004e00058
:10230c0079003a007e0090008000e900f007200080
:10231c000080600001802100614078000004e00032
:10232c00710032004e0890000000e800400f980049
:10233c003e0890008000e9004e089000808f50000d
:10234c0069003a003e0890000000e900300f980048
:10235c0011c4800000c48000808f50001200320035
:10236c000900370000c48000018021000041eb000f
:10237c008270780000c480008000e900f007200023
:10238c000080600000c4880001c4800010c480007c
:10239c00808f5000f3ff3a0000c4800001802100c0
:1023ac000041eb00827078007e0090008000e90014
:1023bc00f0072000008060006007980011003700d3
:1023cc00018021006e0090000080400010407800d9
:1023dc000004e00006003a006e0090008000e80067
:1023ec00f007200000806000000f98000900370003
:1023fc006e0090008000e900f00720000080600073
:10240c0060079800ee00900000c48000808f5000a0
:10241c00ebff3a0090912800f26d020000000000e2
:10242c00b1cf8000000320000088b90000007800c4
:10243c008102200080804000008d2100008040003f
:10244c00f26d02000000000060902800f26d0200a6
:10245c00000000008e0890006107980017003700fc
:10246c00018021006e009000008040001040780038
:10247c002c7302000000000000c4800002802100c8
:10248c00ee00900081004100114178000180210094
:10249c008270780000c480008000e800f007200003
:1024ac000080600000c488006e0090008000e8008e
:1024bc00f00720000080600060079800ee0090009c
:1024cc007e009000808f5000e5ff3a0000c4800031
:1024dc00018021000041eb008270780001c4800073
:1024ec00210f9800090037007e0090008000e90061
:1024fc00f00720000080600070079800fe0090003c
:10250c0000c48000808f500078ff3a00fe009000dd
:10251c0000c48000808f5000fb003a003e08900001
:10252c00e10f500027003a0090912800f26d020054
:10253c0000000000b1cf8000000320000088b9002b
:10254c00000078008102200080804000008d210076
:10255c0000804000f26d0200000000006090280036
:10256c00f26d0200000000000900370000c480007a
:10257c00018021000041eb008270780000c48000d3
:10258c008000e900f00720000080600000c4880093
:10259c0001c4800010c48000808f5000f3ff3a000b
:1025ac0000c48000018021000041eb0082707800a3
:1025bc0001c48000210f98000000eb00300f980040
:1025cc00d400370070c0b3002c7302000000000070
:1025dc00d00037000000000010c48000ae0890004e
:1025ec00808f50001400320010c48000ae089000a0
:1025fc000080500080007800f00720000080600010
:10260c006007980000912800f26d020000000000a5
:10261c006e00900000407800847002000000000002
:10262c0030912800f26d02000000000011c48000ff
:10263c00210f9800b700370070c0b3002c73020054
:10264c0000000000b30037000000000000c4800050
:10265c00ae089000808f50001400320001c480003e
:10266c002e0890000080500080007800f0072000b9
:10267c00008060006007980000912800f26d020055
:10268c00000000006e009000004078008470020092
:10269c0000000000f0912800f26d02000000000024
:1026ac0001c48000210f98009a00370070c0b3005d
:1026bc002c73020000000000960037001000200070
:1026cc00000f78000000eb00300f980000c4800071
:1026dc00018021000041eb008270780000c4800072
:1026ec008000e800f00720000080600000c4880033
:1026fc0001c48000210f980010922800166e020071
:10270c0000000000830037001e0890000000e80065
:10271c00100f98001e089000f40f50007c003a0037
:10272c0012740200000000007a00370000c4800020
:10273c008000e800f00720008080600010c480005a
:10274c00808f5000680032004e589000ff4f5000b0
:10275c0065003600ce589000e0c7b30080cf500023
:10276c0061003e0001c480002e089000808f500054
:10277c0013003a004e5890002c7302000000000029
:10278c0000c480004e5990000180210082707800b6
:10279c0000c480008000e800f0072000008060008a
:1027ac0000c4880000c48000018021000041eb00bf
:1027bc008270780001c48000210f9800550037000a
:1027cc0001c480002e08900000805000800078002a
:1027dc00f00720000080600060079800009128003e
:1027ec00f26d0200000000006e00900000407800c6
:1027fc008470020000000000f0912800f26d0200cd
:10280c000000000000c48000700798001c00370016
:10281c007e0090000000e80002802100fe00900085
:10282c008100410011417800018021008270780004
:10283c00018021007e009000008040001040780054
:10284c000004e00009003200018021007e009000ad
:10285c0000804000104078002c7302000000000043
:10286c0020922800f26d0200000000007e00900013
:10287c008000e900f00720000080600070079800dd
:10288c00fe0090002e0890000001e900f0072000e7
:10289c0000006100808f5000ddff3a004e58900020
:1028ac002c73020000000000ce5890000280210022
:1028bc002e08900000004100014878002e0890007e
:1028cc008000e800f007200000806000200f9800d6
:1028dc0000c480008000e800f00720000080600049
:1028ec0000c488000b00370070c0b3002c730200ca
:1028fc000000000007003700000000000500370052
:10290c000000000003003700000000000100370049
:10291c00000000001e0078000000e000d3fb320035
:10292c0000c480002007980010c480003007980075
:10293c000000eb00000f78000000eb00100798007f
:10294c00408821008040eb00014878000040eb00fb
:10295c00205f98000040eb00305f98005405370072
:10296c0010c480000180210061407800405f980015
:10297c004e5890000080fb00cf80de00e207200064
:10298c0003002000820f5000838f580009053e0081
:10299c00006001000b053700060537000505370000
:1029ac000405370003053700020537000105370021
:1029bc0000053700ff043700fe043700010537001f
:1029cc00fc043700fb043700fe043700f904370021
:1029dc00f8043700f7043700f6043700f504370025
:1029ec00f4043700f3043700f2043700f104370025
:1029fc00f0043700ef043700ee043700ed04370025
:102a0c00ec043700eb043700ea043700e904370024
:102a1c00e8043700eb043700c4043700ea0237003f
:102a2c00330137003d013700ff013700ed0137005e
:102a3c00e0043700c2023700de043700dd04370043
:102a4c00dc043700df0437006c04370087043700e0
:102a5c004e04370066033700650337006403370004
:102a6c0063033700620337006103370060033700ec
:102a7c005f0337005e0337005d033700cd0437007a
:102a8c00cc04370004023700cc003700c9043700ef
:102a9c00470037005001370042013700c5043700aa
:102aac006c003700cc013700c2043700c10437007a
:102abc00c0043700bf043700be043700bd04370024
:102acc00bc0437006d003700ba043700b904370076
:102adc00b804370093003700b6043700b50437004c
:102aec00e2013700b3043700b2043700b1043700f9
:102afc004f013700af043700ae043700ad04370088
:102b0c00140337002f043700250337006704370000
:102b1c0048043700a7043700150137002f00370091
:102b2c00420037009e013700a20437003100370005
:102b3c003300370016003700200037009d043700a3
:102b4c009c043700590037002200370099043700e5
:102b5c002400370061003700960437009f033700cc
:102b6c009404370093043700920437001f00370099
:102b7c006c0137008f0437008e0437008d0437004a
:102b8c00fd023700aa0037000f033700cb003700d7
:102b9c00780707000000e0008c043a0010c48000a5
:102bac003007980000c4800020079800900437007c
:102bbc00d48c0200000000008d043700c008070010
:102bcc00b0cf80000000e0008204320056090700fc
:102bdc0087043700d006070085043700920a0700e7
:102bec00830437006a0a070081043700dd090700f7
:102bfc007f0437005c5e0200000000007c0437009c
:102c0c00b0cf80000000e00005003a00d1012000a8
:102c1c00505a2000be8c02000000000074043700e3
:102c2c00fc5c02000000000071043700819c210054
:102c3c00114078000000a1000010a100804878002d
:102c4c0061012000a0572000be8c02000000000093
:102c5c0067043700819c2100114078000000a0001f
:102c6c000010a1008048780051012000005920007c
:102c7c00be8c0200000000005d043700819c210026
:102c8c00114078000030a00080487800c10120007d
:102c9c00e07e2000328c0200000000001092280020
:102cac00166e02000000000051043700819c2100c8
:102cbc00114078000030a10080487800b10120005c
:102ccc00307d2000328c02000000000010922800a1
:102cdc00166e02000000000045043700b0cf8000e3
:102cec000000e00005003a00d1012000505a2000fd
:102cfc00be8c0200000000003d043700cb62a9002e
:102d0c00c962a90051012000205c2000328c020015
:102d1c000000000010922800166e02000000000057
:102d2c0033043700b0cf80000000e00005003a000b
:102d3c00d1012000505a2000be8c0200000000007f
:102d4c002b043700809c21001040780070406000fc
:102d5c000004e00004003a0021022000f0e9200009
:102d6c00be8c020000000000c962a800cb62a90062
:102d7c0041012000705d2000328c02000000000038
:102d8c0010922800166e02000000000021e3a8003b
:102d9c00b0002000568a020000000000f104200060
:102dac00810f500003003e0070922800166e020046
:102dbc000000000021e3a9000d04370010c48000be
:102dcc008000e800f00720000080600010c488003c
:102ddc004206070040040700700798007e00900030
:102dec00ec70020000000000a0942800f26d0200bc
:102dfc00000000007e00900000407800847002000b
:102e0c0000000000a0942800f26d020000000000f9
:102e1c007e00900000407800426e0200000000002e
:102e2c0010922800166e020000000000f00337001c
:102e3c0010c480008000e800f007200000806000d3
:102e4c0010c48800250607002304070070079800ab
:102e5c007e009000004078000080fb00ea8b0200ae
:102e6c0000000000700798007e009000ec700200db
:102e7c0000000000a0942800f26d02000000000089
:102e8c007e0090000040780084700200000000007a
:102e9c00a0942800f26d0200000000007e0090005b
:102eac0000407800426e02000000000010922800e2
:102ebc00166e020000000000cd033700b0cf80007a
:102ecc000000e00005003a0011c0b30010c0b300d0
:102edc004884020000000000c5033700a101200057
:102eec00b05e2000be8c020000000000c003370062
:102efc005100200050602000be8c02000000000039
:102f0c00000000002a720200000000000004e00033
:102f1c00fcff32000000fe00b5033700648d020098
:102f2c00000000000004e000ac033200a10020000f
:102f3c00a0602000be8c02000000000040062000b3
:102f4c008a8b020000000000128a020000000000c0
:102f5c00000000002a720200000000000004e000e3
:102f6c00fcff320081bf2a0001400100a0033700a2
:102f7c005c0507000000e8006007980002003700bd
:102f8c0020640200000000006e0090000000e900c8
:102f9c00600798006e0090000000e000f8ff3a0017
:102fac00930337004f0507000000e8006007980006
:102fbc0002003700fe630200000000006e0090006b
:102fcc000000e900600798006e0090000000e0002f
:102fdc00f8ff3a0086033700420507000000e800be
:102fec00600798000b003700610120004061200051
:102ffc00328c02000000000042640200000000005d
:10300c00b86d02000000000010922800166e02003d
:10301c00000000006e0090000000e90060079800be
:10302c006e0090000000e000efff3a0070033700e4
:10303c00b0cf80000000e00005003a00d101200074
:10304c00505a2000be8c02000000000068033700bc
:10305c00c002a900c202a80021e3a80020002000a1
:10306c008a8b020000000000a0002000568a02009b
:10307c0000000000011b2000810f50001b003600d7
:10308c0090002000568a020000000000712b2000e6
:10309c00810f50001500360011012000a0622000a5
:1030ac00328c02000000000010922800166e020004
:1030bc0000000000b1cf8000000320000088b900a0
:1030cc00000078000102200080804000008d21006b
:1030dc00008040001000780000000100e0942800ff
:1030ec00166e0200000000000c003700c002a900a0
:1030fc00c202a90000962800166e02000000000013
:10310c0021012000b0632000328c0200000000007e
:10311c0010922800166e02000000000021e3a900a6
:10312c0033033700b0cf80000000e00005003a0008
:10313c00d1012000505a2000be8c0200000000007b
:10314c002b033700b1cf8000000320000088b900aa
:10315c00000078002102200080804000008d2100ba
:10316c00008040001000780000000100009828004a
:10317c00166e020000000000c002a900c202a900e5
:10318c0021012000b0632000328c020000000000fe
:10319c0010922800166e0200000000001403370085
:1031ac00f1002000c0362000328c0200000000002c
:1031bc00728a02000000000011002000b0372000cd
:1031cc00328c02000000000010922800166e0200e3
:1031dc000000000006033700848a02000000000093
:1031ec0003033700bf04070060079800610020004c
:1031fc0090652000328c0200000000006e009000f0
:10320c001c7002000000000021002000f06520006e
:10321c00be8c0200000000006e009000b28b020019
:10322c0000000000f2023700ae04070060079800af
:10323c006100200090652000328c0200000000002c
:10324c006e0090001c7002000000000021002000a5
:10325c0030ee2000be8c0200000000006e009000da
:10326c008a8b020000000000e1023700b0cf800022
:10327c000000e00005003a00d1012000505a200067
:10328c00be8c020000000000d902370072640200fc
:10329c0000000000d60237004088210011c0b300a6
:1032ac0001487800100020007007980010003700cb
:1032bc0011c480007e00900080804000f007200048
:1032cc000080600001802100e1407800e0c3b30081
:1032dc0080cf500003003a00408821008040eb0072
:1032ec00014878007e0090000000e800700798000c
:1032fc0011c480007e00900080804000f007200008
:10330c000080600001802100614078000004e00032
:10331c00e7ff3a007e009000fa0f500003003400e3
:10332c004088210011c0b30001487800408821007a
:10333c00104078000004a2000004e000a902320052
:10334c0010c480008000e800f007200000806000be
:10335c0010c48800e00207007007980011c48000b8
:10336c00f00720000080600001802100e14078001f
:10337c00d0c3b30080cf500042003a007e009000d2
:10338c000000e0003b0034007e009000e30f500092
:10339c0038003c0010c480008000e800f0072000da
:1033ac000080600010c488007e0090000000e900de
:1033bc00700798000000eb00600798000c003700c5
:1033cc007e009000528821007800b90080007800bf
:1033dc006e00900000804000000041008040eb0037
:1033ec00014878006e0090000000e800600798002b
:1033fc006e009000f70f5000f1ff34000000eb005e
:10340c00600798001300370010c480000180210071
:10341c00614178007e009000538821007800b9004b
:10342c00800078006e009000008040000080410019
:10343c00024878006e0090000000e80060079800d9
:10344c0010c480008000e800f007200000806000bd
:10345c0010c4880010c4800001802100e140780075
:10346c00e0c3b30080cf5000e7ff3a00000000003b
:10347c005f0237004088210011c0b300014878007a
:10348c005b0237007e0090000000e0001c003a0058
:10349c000000eb0060079800150037006e009000ec
:1034ac00004078000040e80084700200000000003a
:1034bc0050992800f26d0200000000005288210093
:1034cc006e0090007800b900000078000000410008
:1034dc00f26d02000000000060902800166e0200e1
:1034ec00000000006e0090000000e80060079800eb
:1034fc006e009000e20f5000e8ff34003c023700f1
:10350c007e0090000000e000090034007e00900076
:10351c00e30f500006003c0010922800166e0200cb
:10352c0000000000fe00900071c6880030023700d9
:10353c004088210011c0b300014878002c023700ec
:10354c0010c480008000e800f007200000806000bc
:10355c0010c4880060020700400798005f04070051
:10356c0011c48000f0072000008060000180210061
:10357c00e140780090c2b30080cf50000e003a00ba
:10358c00b1cf8000000320000088b9000000780053
:10359c00fc004000008d210000804000900078006d
:1035ac004e0090000100010010922800166e0200df
:1035bc00000000000e0237004088210011c0b3004b
:1035cc00014878000a0237004088210011c0b3007e
:1035dc000148780010002000700798001000370098
:1035ec0011c480007e00900080804000f007200015
:1035fc000080600001802100e140780020c2b3000f
:10360c0080cf500003003a00408821008040eb003e
:10361c00014878007e0090000000e80070079800d8
:10362c0011c480007e00900080804000f0072000d4
:10363c000080600001802100614078000004e000ff
:10364c00e7ff3a0040882100104078000004a200f7
:10365c000004e000e501320071002000106620003b
:10366c00328c02000000000020c2b3002c73020058
:10367c00000000002100370011c48000f00720007a
:10368c000080600010c4880010c4800001802100fc
:10369c00614078002c7302000000000010c4800010
:1036ac0001802100614078000000fb004007980079
:1036bc00809c210010407800684060000004e0000d
:1036cc00040032004e009000ea8b02000000000063
:1036dc0040079800b1cf8000000320000088b9009b
:1036ec0000007800e8004000008d210000804000c0
:1036fc00900078004e0090000100010010c4800082
:10370c000000e80010c4880011c48000f0072000fd
:10371c000080600001802100e140780020c2b300ed
:10372c0080cf5000d4ff3a0011c48000f007200075
:10373c000080600010c4880020c2b3002c7302000b
:10374c000000000010922800166e0200000000001d
:10375c00a7013700b1cf8000000320000088b9001a
:10376c0080007800008d210000804000100078005f
:10377c00000001009e013700b1cf80000003200043
:10378c000088b900000078008080e800008d2100de
:10379c000080400010007800000001009401370008
:1037ac00b1cf8000000320000088b9000000780031
:1037bc00e4004000008d21000080400010007800e3
:1037cc00000001008a013700b1cf80000003200007
:1037dc000088b90000007800e6004000008d210050
:1037ec0000804000100078000000010080013700cc
:1037fc007100200010662000328c020000000000d6
:10380c00b50107004007980010c480000000e900d3
:10381c0010c4880011c48000f007200000806000f4
:10382c0010c488002f0307000000e8006007980010
:10383c004b030700700f98007e0890000000e0001a
:10384c005c0032007e08900080407800709b210064
:10385c00014878007e089000e80f50000500340005
:10386c00819c2100114078000050a0008048780015
:10387c0050003700819c2100114078000050a100bd
:10388c00804878004b0037004e009000e28a02001e
:10389c0000000000809c2100104078000042b20023
:1038ac000004e00004003a00709b210010407800f6
:1038bc00e84f500009003a00809c2100104078002d
:1038cc000042b2000004e0000b003200709b2100ab
:1038dc0010407800f04f500007003200b0c3b30026
:1038ec002c73020000000000709b21001040780037
:1038fc008470020000000000809c210010407800c1
:10390c00684060000004e000040032004e009000ab
:10391c00ea8b02000000000040079800b1cf800045
:10392c00000320000088b90000007800e800400087
:10393c00008d210000804000900078004e00900027
:10394c00010001005007980000c2b3002c73020064
:10395c0000000000809c2100104078000044b20060
:10396c000004e0001300320061002000806620009b
:10397c00328c020000000000809c21001040780076
:10398c00684060000004e000040032005e0090001b
:10399c00ea8b020000000000500798005e009000c7
:1039ac00e28a02000000000000c2b3002c73020087
:1039bc00000000006e0090000000e9006007980015
:1039cc006e0090000000e000afff3a00109228005b
:1039dc00166e020000000000050137006100200097
:1039ec0080662000328c020000000000f702070005
:1039fc00305f9800bb0207000000e80060079800e9
:103a0c00d7020700700f98007e0890000000e000bd
:103a1c00100032007e08900080407800709b2100de
:103a2c00014878007e089000e80f50000500340033
:103a3c00819c2100114078000050a0008048780043
:103a4c0004003700819c2100114078000050a10037
:103a5c00804878003e5890000004e00039003200a5
:103a6c00a0cf8000205f98003e5890000080fb00a3
:103a7c000000e900a0cf880032003700b1cf8000f1
:103a8c00000320000088b90000007800ea00400024
:103a9c00008d210000804000100078000000010023
:103aac0050079800809c210010407800684060000e
:103abc000004e000040032005e009000ea8b02007b
:103acc0000000000500798005e009000e28a02009f
:103adc0000000000809c2100104078000042b200e1
:103aec000004e00004003a00709b210010407800b4
:103afc00e84f500009003a00809c210010407800eb
:103b0c000042b2000004e0000b003200709b210068
:103b1c0010407800f04f500007003200b0c3b300e3
:103b2c002c73020000000000709b210010407800f4
:103b3c00847002000000000000c2b3002c7302006d
:103b4c00000000006e0090000000e9006007980083
:103b5c006e0090000000e000c8ff3a003e58900054
:103b6c000004e000050032002e5890000080fb009d
:103b7c00a0cf88000040eb00305f98001092280026
:103b8c00166e020000000000990037008100200032
:103b9c00e0662000be8c020000000000b1cf800067
:103bac00000320000088b90000007800ec00400001
:103bbc00008d210000804000100078000000010002
:103bcc008b0037008100200060672000be8c020053
:103bdc0000000000b1cf8000000320000088b90075
:103bec0000007800ee004000008d210000804000b5
:103bfc0010007800000001007d003700e10020007b
:103c0c00e0672000be8c020000000000b1cf8000f5
:103c1c00000320000088b90000007800f00040008c
:103c2c00008d210000804000100078000000010091
:103c3c006f003700e1002000c0682000be8c02003d
:103c4c0000000000b1cf8000000320000088b90004
:103c5c0000007800f2004000008d21000080400040
:103c6c00100078000000010061003700c100200046
:103c7c00d0642000328c020000000000b1cf800024
:103c8c00000320000088b90000007800f400400018
:103c9c00008d210000804000100078000000010021
:103cac00b86d020000000000510037000d02070043
:103cbc0060079800d1002000a06a2000328c02001e
:103ccc00000000006e009000e28a0200000000007c
:103cdc006e0090000000e8006007980009003700b3
:103cec00b1cf8000000320000088b90000007800ec
:103cfc00f6004000008d210000804000100078008c
:103d0c00000001006e0090000000e90060079800c0
:103d1c006e0090000000e000f1ff3a0010922800c5
:103d2c00166e02000000000031003700ed010700a4
:103d3c000000e80060079800a1002000706b2000d4
:103d4c00328c0200000000000f003700b1cf800061
:103d5c00000320000088b90000007800f800400043
:103d6c00008d210000804000100078000000010050
:103d7c000080fb00b86d02000000000000c2b30020
:103d8c002c730200000000006e0090000000e9009f
:103d9c00600798006e0090000000e000ebff3a0016
:103dac0001012000a0692000be8c02000000000070
:103dbc000f0037004088210011c0b3000148780083
:103dcc000b00370000000000090037000000000065
:103ddc00070037000000000005003700000000005d
:103dec000300370000000000010037000000000055
:103dfc0010c480008000e800f00720000080600004
:103e0c0010c4880040882100104078000004e000b5
:103e1c002100320051012000106c2000328c020075
:103e2c0000000000be00900010c48000808f500085
:103e3c000800310010c48000804078003e009000e3
:103e4c000040780000c050008470020000000000a8
:103e5c000900370010c48000804078003e009000bc
:103e6c000040780080c0500000c8b30000c0400083
:103e7c008470020000000000408821008040eb00ac
:103e8c0001487800100020001007980010922800bc
:103e9c00166e02000000000011c4800000c48000f7
:103eac00808f500002003a0010002000100798008c
:103ebc001e0090000000e000a9fa32002e009000d5
:103ecc0010c488002e00900000c488000000eb0095
:103edc00000f780057f637000400fa000000eb00e2
:103eec00000f78000000eb001007980011c4800050
:103efc001e00780080804000f007200000806000e9
:103f0c0001802100e140780000c3b30080cf500055
:103f1c003c00340011c480001e00780080804000fa
:103f2c00f00720000080600001802100e140780053
:103f3c0090c3b30080cf500032003c0011c480000d
:103f4c001e00780080804000f00720000080600098
:103f5c0001802100614078000000fb000003b100eb
:103f6c00100798001e0fe800110037001e0090008b
:103f7c006a00b900000078001007980011c4800096
:103f8c001e00780080804000f00720000080600058
:103f9c0001802100614078000000fb000003b100ab
:103fac009e00900000804000100798001e0fe80053
:103fbc0011c480001e00780080804000f0072000b3
:103fcc000080600001802100e1407800f0c2b30065
:103fdc0080cf50002f01340011c480001e007800e7
:103fec0080804000f00720000080600001802100ec
:103ffc00e140780090c3b30080cf5000dbff340069
:10400c002d01370011c480001e0078008080400014
:10401c00f00720000080600001802100e140780062
:10402c0000c3b30080cf500015013a001e0fe8000a
:10403c0011c480001e00780080804000f007200032
:10404c000080600001802100e140780020c6b300b0
:10405c0080cf50000a00320011c480001e0078008e
:10406c0080804000f007200000806000018021006b
:10407c00e140780020c4b30080cf500027003a0004
:10408c001e0fe800100037001e00900000004000da
:10409c001007980011c480001e007800808040003a
:1040ac00f007200000806000018021006140780052
:1040bc000000fb000003b1009e0090000080400057
:1040cc00100798001e0fe80011c480001e00780035
:1040dc0080804000f00720000080600001802100fb
:1040ec00e140780010c3b30080cf5000e6ff3200ef
:1040fc0011c480001e00780080804000f007200072
:10410c000080600001802100e140780000c3b30012
:10411c0080cf5000dcff3200e700370011c4800074
:10412c001e00780080804000f007200000806000b6
:10413c0001802100e140780080c7b30080cf50009f
:10414c000a00320011c480001e00780080804000fc
:10415c00f00720000080600001802100e140780021
:10416c0080c5b30080cf500080003a001e0fe800dd
:10417c00410037001e0090004400dd00100798003d
:10418c0011c480001e00780080804000f0072000e1
:10419c000080600001802100e1407800f0c2b30093
:1041ac0080cf50001700340011c480001e0078002e
:1041bc0080804000f007200000806000018021001a
:1041cc00e140780090c3b30080cf50000d003c005c
:1041dc0011c480001e00780080804000f007200091
:1041ec000080600001802100614078000000fb002d
:1041fc000003b1009e009000008040001007980062
:10420c001c00370011c480001e0078008080400024
:10421c00f00720000080600012c480009e0078002f
:10422c0001014100f10720008100610002802100a2
:10423c0062c1780001c2b30001417100018021000c
:10424c008270780011c480001e00780080804000cd
:10425c00f0072000008060000180210061407800a0
:10426c000000fb007005b1009e0090000080400033
:10427c00100798001e0fe80011c480001e00780083
:10428c0080804000f0072000008060000180210049
:10429c00e1407800f0c2b30080cf50000a00340037
:1042ac0011c480001e00780080804000f0072000c0
:1042bc000080600001802100e140780090c3b300d1
:1042cc0080cf5000abff340011c480001e0078007a
:1042dc0080804000f00720000080600001802100f9
:1042ec00e140780000c4b30080cf50000a003400d5
:1042fc0011c480001e00780080804000f007200070
:10430c000080600001802100e140780060c4b300af
:10431c0080cf500097ff340011c480001e0078003d
:10432c0080804000f00720000080600001802100a8
:10433c00e140780000c6b30080cf50005700340035
:10434c0011c480001e00780080804000f00720001f
:10435c000080600001802100e140780060c6b3005d
:10436c0080cf500083ff34005300370011c480000d
:10437c001e00780080804000f00720000080600064
:10438c0001802100e1407800f0c2b30080cf5000e2
:10439c004400340011c480001e007800808040006e
:1043ac00f00720000080600001802100e1407800cf
:1043bc0090c3b30080cf50003c003c0011c480007f
:1043cc001e00780080804000f00720000080600014
:1043dc0001802100614078000000fb000003b10067
:1043ec0010079800110037001e0090006a00b900f9
:1043fc00000078001007980011c480001e0078009f
:10440c0080804000f00720000080600001802100c7
:10441c00614078000000fb000003b1009e0090009a
:10442c0000804000100798001e0fe80011c48000a7
:10443c001e00780080804000f007200000806000a3
:10444c0001802100e1407800f0c2b30080cf500021
:10445c001800340011c480001e00780080804000d9
:10446c00f00720000080600001802100e14078000e
:10447c0090c3b30080cf5000dbff34000e00370038
:10448c004088210011c0b300014878000000eb0007
:10449c001200370000000000070037000000000089
:1044ac00050037000000000003003700000000008a
:1044bc00010037000000000011c480001e007800cd
:1044cc000080400010c4880011c48000f007200058
:1044dc000080600010c488001e0090000080fa006c
:1044ec00000006000200fa0010c480008000e80002
:1044fc00f00720000080600001802100e14078007e
:10450c00a0c3b30080cf500012003a0010c480004a
:10451c000080e80010c4880011c48000f00720005f
:10452c000080600010c488006bfe0700000f78004c
:10453c0010c480000000e90010c4880011c4800081
:10454c00f00720000080600010c488001e00780076
:10455c0001003700100020000080fa000000060067
:10456c000200fa0010c480008000e800f007200070
:10457c000080600001802100e1407800b0c3b300ee
:10458c0080cf50000e003a0010c480008080e800fc
:10459c00f00720000080600010c488004efe070069
:1045ac00000f780010c480008000e900f0072000a4
:1045bc000080600010c488001e00780001003700e5
:1045cc000000eb000080fa00000006000000fa007a
:1045dc0010c480008000e800f0072000008060001c
:1045ec0001802100e140780080c7b30080cf5000eb
:1045fc0007003a0010c480008000e800f00720009b
:10460c000080600010c4880010c0b3003100370077
:10461c0010c480008000e800f007200000806000db
:10462c0001802100e140780040c6b30080cf5000eb
:10463c0007003a0010c480008000e800f00720005a
:10464c000080600010c4880020c0b3002100370037
:10465c0010c480008000e800f0072000008060009b
:10466c0001802100e140780020c6b30080cf5000cb
:10467c0007003a0010c480008000e800f00720001a
:10468c000080600010c4880030c0b30011003700f7
:10469c0010c480008000e800f0072000008060005b
:1046ac0001802100e140780070c7b30080cf50003a
:1046bc0007003a0010c480008000e800f0072000da
:1046cc000080600010c4880040c0b30001003700b7
:1046dc000040eb000080fa00000006000000fa0029
:1046ec000500370010c480008000e800f0072000af
:1046fc000080600010c4880010c48000018021007c
:10470c00e140780000c2b30080cf5000f5ff3200ca
:10471c000080fa00000006000400fa000000eb0024
:10472c001007980010c480008000e800f0072000fb
:10473c000080600010c48800e8ff0700e6fd070059
:10474c00100798001e0090000000e00058003a008e
:10475c000000eb00000f7800130037001e007800fb
:10476c00004078000040e800847002000000000067
:10477c0090992800f26d0200000000009e00780065
:10478c00000320000088b90000007800810220009e
:10479c0080804000008d210000804000166e0200d9
:1047ac00000000001e0fe8001e007800e30f500010
:1047bc00eaff340071012000606d2000be8c020005
:1047cc0000000000408821008040eb000148780088
:1047dc0013002000420020001100200010002000d7
:1047ec00030107000000e900100798001e0090006c
:1047fc00e20f4000030032001e009000e10f400069
:10480c0005003a00e1002000d06e2000be8c0200b2
:10481c000000000050003700b1cf800000032000e2
:10482c000088b90000007800210220008080400040
:10483c00008d210000804000100078000000010075
:10484c00128a0200000000001e009000b0cf880009
:10485c00b1cf8000000320000088b9000000780070
:10486c00fe004000008d2100008040001000780008
:10487c000000010000982800166e020000000000e5
:10488c001e0090000000e00004003200c222a800cc
:10489c00c0992800166e0200000000005100200094
:1048ac0050572000be8c0200000000002a00370088
:1048bc001e0090000000e900100798001e009000f8
:1048cc00e30f500020003c00b1cf8000000320001b
:1048dc000088b90000007800210220008080400090
:1048ec00008d2100008040001000780000000100c5
:1048fc00128a0200000000001e009000b0cf880059
:10490c00b1cf8000000320000088b90000007800bf
:10491c00fe004000008d2100008040001000780057
:10492c00000001001e0090000000e00001003200b9
:10493c00c222a8005100200050572000be8c02005b
:10494c00000000000400370051012000c07220005c
:10495c00be8c02000000000000c480008000e90052
:10496c00f00720000080600010c488000080fa006e
:10497c00000006001400fa0010002000000f780060
:10498c0010c480000000e90080007800f0072000cf
:10499c000080600010079800420037000180210061
:1049ac001e00900000804000104078000004e000e1
:1049bc0037003a001e0090008000e800f00720004d
:1049cc000080600001802100614078000004e0005c
:1049dc002f0032001e007800004078008470020026
:1049ec000000000090992800f26d02000000000009
:1049fc0010002000200798000c0037009e0090004b
:104a0c002e00900080804000f007200000806000a5
:104a1c0001802100614078002c730200000000002e
:104a2c002e0090000000e800200798009e009000e7
:104a3c002e00900080804000f00720000080600075
:104a4c0001802100614078000004e000ebff3a0097
:104a5c001e0090008000e800f007200080806000bd
:104a6c001e00780000004000000047006600400077
:104a7c00010878001e0fe8001e007800e70f5000b8
:104a8c000d00320010922800166e0200000000008b
:104a9c001e0090008000e900f007200000806000fc
:104aac00100798009e00900010c48000808f50006a
:104abc00baff3a000100370000000000c09d28003a
:104acc00166e02000000000071002000107420001f
:104adc00be8c020000000000130020001e017800b4
:104aec00110020000000eb004100070010079800a7
:104afc001e009000e10f4000030032001e009000e9
:104b0c000000e00005003a0010922800166e02002a
:104b1c000000000010002000330037000000eb0004
:104b2c00000f78001100370001c480001e007800cf
:104b3c0080804000f0072000808060001e00900004
:104b4c000000400000004700300090001e014000b3
:104b5c00f007200000006100028021006241780013
:104b6c000080210002f078001e0fe8001e0090006b
:104b7c000000400000004700300090009e00400004
:104b8c00f007200000806000018021006140780067
:104b9c000004e000e4ff3a0000c480008000e9005b
:104bac00f00720000080600010c4880011c4800051
:104bbc001e007800008040008080e800f007200094
:104bcc000080600000c4880000c480008000e90000
:104bdc00f007200000806000018021000041eb0004
:104bec00827078000000eb000080fa0000000600e4
:104bfc001a00fa00100f9800210f9800320f98003d
:104c0c00430f98000000eb00000f78000000eb0051
:104c1c00100798000000eb00200798000000eb0044
:104c2c0030079800e09d2800f26d020000000000a3
:104c3c001e0890000000e00004003d00209e2800ab
:104c4c00f26d020000000000040037001e08900006
:104c5c00004078008470020000000000409e280094
:104c6c00f26d0200000000005c00370006730200c9
:104c7c0000000000004f98000e4890000000fb0060
:104c8c00ed0f500023003200ed0f500005003c00ea
:104c9c00e80f50000a003200ea0f50001d003200ed
:104cac0031003700d1022000810f50001c0032006f
:104cbc0081072000810f5000260032002a003700a7
:104ccc001e0078000000e000050032001e0fe90015
:104cdc0080902800f26d0200000000003f003700b9
:104cec003e0090000000e000060032000000eb00e7
:104cfc003007980080902800f26d02000000000040
:104d0c003600370070c0b3002c73020000000000a6
:104d1c003200370010002000100798002f003700d9
:104d2c001e0078000000e00006003a00d0c2b3007c
:104d3c002c730200000000001000200030079800c7
:104d4c002600370070c0b3002c7302000000000076
:104d5c00220037004e0890000000e00002003200f4
:104d6c000080eb00540037008e489000f0c2b30076
:104d7c0080cf5000160034008e48900090c3b300d2
:104d8c0080cf500012003c001e007800e30f500052
:104d9c000600340070c0b3002c7302000000000049
:104dac0040002000000f78000c0037000e489000e7
:104dbc002c730200000000006c0047001e00400035
:104dcc008e489000014878001e0fe8000300370061
:104ddc0070c0b3002c730200000000001e00900095
:104dec000000e000a1ff320010922800166e0200b5
:104dfc00000000001e0078000000e00002003a00f5
:104e0c001e0890002c0037000000eb0020079800d3
:104e1c001e0fe9009e007800510798000e00370025
:104e2c002e0090006a00b90000007800200798005e
:104e3c005e0090001e0050000000470040489000ab
:104e4c000000fb000003b100ae00900000804000a9
:104e5c00200798001e0fe9001e0078000000e000fb
:104e6c00efff3d00ae0090002e089000808f5000a8
:104e7c000c003500ae0090003e089000808f500072
:104e8c0008003c003e0090000000e00003003200ef
:104e9c002e0090000000ea00070037002e00900062
:104eac0005003700b101200080ec2000be8c020010
:104ebc000000000053ff37000080fa0000000600dd
:104ecc000200fa00709e2800f26d02000000000043
:104edc00e0c2b3002c73020000000000c09f210050
:104eec00104078002c73020000000000c1cf80003d
:104efc00f0442000808f500003003a00509f28009f
:104f0c00f26d02000000000010922800166e0200e4
:104f1c0000000000c0a02800f26d0200000000009c
:104f2c00b0c5b3002c730200000000000000eb00c1
:104f3c00000f7800110037001e0078000000e00020
:104f4c000300320000c2b3002c730200000000000a
:104f5c009e007800000320000088b9000000780053
:104f6c008102200080804000008d210000804000e4
:104f7c00f26d0200000000001e0fe8001e00780019
:104f8c00e30f5000ecff3600d0c5b3002c730200c9
:104f9c0000000000d1002000a0802000328c020014
:104fac0000000000a1bf2a000000eb00d471020039
:104fbc0000000000000f78001e0078004800de00a2
:104fcc00004078008470020000000000e0c2b300d2
:104fdc002c730200000000001e00780000407800d6
:104fec00847002000000000010922800166e02006f
:104ffc00000000006100200030762000328c02009e
:10500c0000000000c0cf80003e71020000000000d4
:10501c007100200010ec2000328c02000000000017
:10502c00d0cf80003e7102000000000050a3280089
:10503c00f26d020000000000c1cf8000f04420009f
:10504c00808f500004003a0020a42800f26d02006a
:10505c00000000000300370050a42800f26d02008d
:10506c0000000000d0cf800021042300810f5000ed
:10507c001200320021042300810f500004003e0076
:10508c0031002300810f5000080032001700370058
:10509c0031042300810f50000c0032006104230006
:1050ac00810f50000d0032001000370080a4280042
:1050bc00f26d02000000000010003700b0a42800c0
:1050cc00f26d0200000000000c003700e0a4280084
:1050dc00f26d0200000000000800370010a5280047
:1050ec00f26d0200000000000400370040a528000b
:1050fc00f26d0200000000000000000080a52800f6
:10510c00166e020000000000e101200090762000e5
:10511c00be8c0200000000000000eb00000f7800c5
:10512c000080fa00000006000000fa005100200088
:10513c0050922000328c020000000000c1bf2a00f7
:10514c000000eb00d4710200000000003e71020070
:10515c000000000061002000a0922000328c0200b0
:10516c0000000000e1bf2a000000eb00d471020037
:10517c00000000003e7102000000000010922800a8
:10518c00166e020000000000c100200070782000a4
:10519c00be8c020000000000720007001016800098
:1051ac00610060000000e0000500320011012000e9
:1051bc00a0622000328c02000000000004003700c6
:1051cc0021012000b0632000328c0200000000009e
:1051dc00c0c2b3002c7302000000000000c2b30078
:1051ec002c7302000000000051168000008020008b
:1051fc00008060000000e00005003200410120004a
:10520c00705d2000328c02000000000004003700aa
:10521c0051012000205c2000328c020000000000b4
:10522c00c0c2b3002c7302000000000000c2b30027
:10523c002c73020000000000809c210010407800bc
:10524c00704060000004e0000500320021022000e4
:10525c0030792000be8c02000000000004003700f2
:10526c00e1012000507b2000be8c020000000000f9
:10527c00809c210010407800684060000004e00031
:10528c0005003a00b1012000307d2000328c020074
:10529c000000000004003700c1012000e07e200067
:1052ac00328c020000000000c0c2b3002c7302005c
:1052bc000000000000c2b3002c73020000000000cc
:1052cc00b1012000b01a2100328c02000000000055
:1052dc00709b2100104078008470020000000000d8
:1052ec0010922800166e020000000000809c210025
:1052fc001040780063406000e14f500005003a0018
:10530c005101200000592000be8c0200000000005a
:10531c000400370061012000a0572000be8c020061
:10532c0000000000b1cf8000000320000088b9000d
:10533c00000078006102200080804000008d210078
:10534c00008040001000780000000100c100200027
:10535c0070782000be8c0200000000000080fa0073
:10536c00000006000000fa00a10020004007210008
:10537c00be8c02000000000061042000c00c210063
:10538c00be8c020000000000a1012000e0072100fb
:10539c00328c020000000000b1cf8000000320001e
:1053ac000088b90000007800410220008080400095
:1053bc00008d2100008040001000780000000100ea
:1053cc00a100200080092100328c020000000000a6
:1053dc000040200050000700001020004e00070085
:1053ec00002020004c000700000420004a000700a9
:1053fc00000820004800070010922800166e0200da
:10540c00000000004100200020112100328c02001d
:10541c000000000021e3a800a0002000568a020032
:10542c00000000008271020000000000110020004a
:10543c00b0372000328c02000000000090c0b30096
:10544c002c7302000000000090002000568a02001d
:10545c00000000008271020000000000110020001a
:10546c00b0372000328c02000000000090c0b30066
:10547c002c73020000000000c0002000568a0200bd
:10548c0000000000827102000000000011002000ea
:10549c00b0372000328c02000000000090c0b30036
:1054ac002c73020000000000b0002000568a02009d
:1054bc0000000000827102000000000011002000ba
:1054cc00b0372000328c02000000000090c0b30006
:1054dc002c7302000000000021e3a9000040200012
:1054ec001c000700001020001a00070000202000fc
:1054fc001800070000042000160007000008200018
:10550c001400070010922800166e02000000000024
:10551c000080fa00000006000200fa00000f78007c
:10552c00401680001e0060000000e0000400320005
:10553c00a0a52800f26d0200000000000300370057
:10554c00d0a52800f26d0200000000000080fa00d7
:10555c00000006000200fa00000f780050168000d0
:10556c001e0060000000e0000400320000a62800cd
:10557c00f26d0200000000000300370030a6280086
:10558c00f26d0200000000000080fa00000006002e
:10559c000200fa0010c480008000e800f007200030
:1055ac000080600010c488004cfc07004afa070019
:1055bc00000f78001e0078000000e00006003400a8
:1055cc001e007800e40f500003003c001e00e900b0
:1055dc00a0cf88000e003700408821008040eb00ef
:1055ec00014878002102200070812000be8c02004e
:1055fc00000000008001eb004200200011002000a0
:10560c00100020007afd07000000e900a0cf880000
:10561c002101200090832000be8c020000000000bd
:10562c000080fa00000006000200fa000040eb00c7
:10563c00004f780010c480008000e800f0072000c4
:10564c000080600010c4880024fc070022fa0700c8
:10565c00104798001e4090000004e0000800320043
:10566c001e409000ea4f500005003e001e40900086
:10567c008040e900209f210001487800100037008d
:10568c00408821008040eb0001487800d1082000c0
:10569c0060872000be8c0200000000008001eb003f
:1056ac00a2002000110020009000200050fd0700f7
:1056bc00004078008040e900209f210001487800dc
:1056cc00209f210010407800e94f500012003a0052
:1056dc0002fc070000fa0700004f78001e4078001b
:1056ec000004e0000c003a00408821008040eb00f0
:1056fc000148780060a62800166e02000000000029
:10570c008001eb00f2ff27008000eb00200220005c
:10571c0037fd0700004f7800410120003090200039
:10572c00be8c02000000000011012000a019210015
:10573c00be8c020000000000000000002a72020073
:10574c00000000000004e000fcff3200209f21005c
:10575c0010407800e94f500003003a001e407800da
:10576c0052730200000000000072020000000000f2
:10577c00010037000000000006730200000000006a
:10578c0001c2b300814f5000faff3a000000000044
:10579c000080fa00000006005752490054452000d2
:1057ac00424954003a2020002a6e6500787420008b
:1057bc00636c6f00636b2000285e29002077690002
:1057cc006c6c200075736500207468006973200090
:1057dc0076616c0075654e006f206400657669001b
:1057ec0063652c002074720079202800414c410024
:1057fc00524d2900205345004152430048206d0072
:10580c00616372006f20660069727300744144001a
:10581c0044524500535320004d414300524f200049
:10582c0020302e004d616300726f20006d656e009c
:10583c00754d610063726f00202020002020310024
:10584c00574952004520610064647200657373000f
:10585c000d0a200020202a00315749005245200013
:10586c00524f4d0020434f004d4d41004e442000ff
:10587c004d414300524f73003a0d0a002035310060
:10588c002e52450041442000524f4d00202830003c
:10589c007833330029202a00666f72002073690068
:1058ac006e676c0065206400657669006365200096
:1058bc00627573000d0a200038352e004d415400de
:1058cc0043482000524f4d002028300078353500d9
:1058dc0029202a00666f6c006c6f770065642000cd
:1058ec0062792000363462006974200061646400bf
:1058fc0072657300730d0a0020323000342e530091
:10590c004b49500020524f004d2028003078430066
:10591c00432920002a666f006c6c6f007765640069
:10592c002062790020636f006d6d61006e640d0064
:10593c000a20320033362e00414c4100524d2000db
:10594c00534541005243480020283000784543001d
:10595c00290d0a0020323400302e530045415200ec
:10596c0043482000524f4d0020283000784630002c
:10597c0029414c0041524d002053450041524300f7
:10598c0048202800307845004329530045415200f7
:10599c0043482000283078004630290044657600c2
:1059ac006963650020494400732061007265200022
:1059bc0061766100696c6100626c6500206279003f
:1059cc00204d410043524f002c2073006565200090
:1059dc00283029002e52450041442000524f4d00e2
:1059ec002028300078333300293a20004d415400f0
:1059fc0043482000524f4d002028300078353500a8
:105a0c0029534b0049502000524f4d0020283000a4
:105a1c007843430029556e006b6e6f00776e200043
:105a2c006d616300726f2c002074720079203f004e
:105a3c00206f720020283000292066006f72200031
:105a4c0068656c0070425500532052004553450068
:105a5c005420570061726e00696e67003a202a006c
:105a6c0053686f00727420006f7220006e6f2000fc
:105a7c0070756c006c2d750070202a004e6f200024
:105a8c006465760069636500206465007465630075
:105a9c0074656400204453003138530032302000c8
:105aac0048696700682050007265730020446900e3
:105abc0067205400686572006d4453003138420011
:105acc003230200050726f00672052006573200046
:105adc00446967002054680065726d0044533100be
:105aec0038323200204563006f6e20004469670035
:105afc002054680065726d00445332003430340019
:105b0c00204563006f6e7200616d200074696d003a
:105b1c00652043006869700044533200343331000f
:105b2c0020314b002045450050524f004d556e0022
:105b3c006b6e6f00776e200064657600696365009c
:105b4c0050574d0020646900736162006c656400fd
:105b5c00314b48007a2d34002c303000304b48004b
:105b6c007a205000574d46007265710075656e00c5
:105b7c0063792000696e20004b487a002050720037
:105b8c0065736300616c65003a505200323a440010
:105b9c007574790020637900636c650020696e0070
:105bac002025200050574d00206163007469760059
:105bbc0065455200524f52003a205000574d20007c
:105bcc0061637400697665002c20670020746f0097
:105bdc0020646900736162006c65410055582000b7
:105bec0046726500717565006e6379003a2041005c
:105bfc0055582000494e500055542f0048492d004f
:105c0c005a41550058204800494748004155580012
:105c1c00204c4f0057564f004c544d0045544500f6
:105c2c0052204d004f444500564f4c005441470004
:105c3c0045205000524f4200453a20005645720014
:105c4c00726f720028292000406c69006e653a0062
:105c5c0020407000676d730070616300653a20002e
:105c6c006279740065732e00546f6f00206c6f00a6
:105c7c006e67210053796e007461780020657200a4
:105c8c00726f72004e6f200045455000524f4d0010
:105c9c004572610073696e0067646f006e65530036
:105cac00617669006e672000746f2000736c6f0062
:105cbc00742049006e7661006c69640020736c007e
:105ccc006f744c006f616400696e6700206672002f
:105cdc006f6d2000736c6f007420450052524f00a2
:105cec00523a2000636f6d006d616e006420680095
:105cfc00617320006e6f200065666600656374003a
:105d0c002068650072654100434b4e0041434b00d7
:105d1c004932430020535400415254002042490060
:105d2c005449320043205300544f50002042490044
:105d3c005449320043206d006f6465003a0d0a002f
:105d4c0020312e0020536f0066747700617265005d
:105d5c000d0a2000322e2000486172006477610029
:105d6c0072655300657420007370650065643a00b9
:105d7c000d0a2000312e20007e354b00487a0d0094
:105d8c000a2032002e207e0035304b00487a0d0060
:105d9c000a2033002e207e00313030004b487a0030
:105dac000d0a2000342e20007e343000304b480089
:105dbc007a574100524e49004e473a002048410064
:105dcc00524457004152450020493200432069009b
:105ddc0073206200726f6b00656e20006f6e200086
:105dec007468690073205000494321002028520038
:105dfc004556200041332900536574002073700010
:105e0c00656564003a0d0a0020312e002031300007
:105e1c00304b48007a0d0a0020322e00203430001e
:105e2c00304b48007a0d0a0020332e0020314d00f3
:105e3c00487a490032432000286d6f0064207300bb
:105e4c00706429003d28200020302e004d61630035
:105e5c00726f20006d656e00750d0a0020312e00ea
:105e6c0037626900742061006464720065737300aa
:105e7c002073650061726300680d0a0020322e00e9
:105e8c004932430020736e006966660065725300e8
:105e9c0065617200636869006e67200049324300d7
:105eac00206164006472650073732000737061007c
:105ebc0063652e0020466f00756e640020646500db
:105ecc00766963006573200061743a00536e690053
:105edc00666665007228420041534900432952000e
:105eec006561640079612f00412f400020636f00d1
:105efc006e7472006f6c7300204155005820700056
:105f0c00696e61002f412f00402063006f6e74009a
:105f1c00726f6c007320430053207000696e430055
:105f2c006f6d6d00616e6400206e6f0074207500e3
:105f3c007365640020696e0020746800697320002a
:105f4c006d6f6400655075006c6c2d0075702000d1
:105f5c0072657300697374006f727300204f460092
:105f6c00465075006c6c2d007570200072657300c6
:105f7c00697374006f727300204f4e0053656c0090
:105f8c00662d74006573740020696e0020486900ea
:105f9c005a206d006f646500206f6e006c795200a2
:105fac004553450054424f004f544c004f41440060
:105fbc004552410055582000494e500055542f0071
:105fcc0048492d005a2c200052454100443a2000eb
:105fdc00504f57004552200053555000504c49002b
:105fec00455320004f4e50004f5745005220530050
:105ffc00555050004c49450053204f004646440034
:10600c004154410020535400415445003a2044006f
:10601c00454c4100592075007357520049544500b6
:10602c003a205200454144003a2043004c4f430073
:10603c004b2c200031434c004f434b002c203000a4
:10604c004441540041204f005554500055542c00ed
:10605c002031440041544100204f5500545055000c
:10606c00542c200030202a0070696e0020697300c7
:10607c00206e6f0077204800695a43004c4f430054
:10608c004b20540049434b00533a200052454100e9
:10609c004420420049543a00205379006e74610048
:1060ac007820650072726f007220610074206300aa
:1060bc006861720020782e002065780069742800d1
:1060cc0077697400686f75007420630068616e00f6
:1060dc00676529006e6f20006d6f6400652063009a
:1060ec0068616e00676523003a204e006f207300d4
:1060fc006f667400776172006520720065736500cd
:10610c0074206f006e207600342c200075736500af
:10611c00207468006520720065736500742062004d
:10612c00757474006f6e2e004e6f6e00657869008a
:10613c00737465006e74200070726f00746f63006e
:10614c006f6c2100782e200065786900740d0a00b0
:10615c00496e7600616c690064206300686f6900a9
:10616c0063652c00207472007920610067616900fe
:10617c006e444500564944003a68740074703a0005
:10618c002f2f6400616e670065726f00757370006d
:10619c00726f74006f747900706573002e636f00fa
:1061ac006d2a2d002d2d2d002d2d2d002d2d2d008a
:1061bc002a4f7000656e200064726100696e2000c9
:1061cc006f7574007075740073202800483d48008a
:1061dc00692d5a002c204c003d474e0044294e009e
:1061ec006f726d00616c20006f75740070757400b7
:1061fc0073202800483d33002e3376002c204c00b1
:10620c003d474e0044294d005342200073657400f5
:10621c003a204d004f5354002073690067206200f0
:10622c00697420006669720073744c00534220003c
:10623c00736574003a204c004541530054207300a0
:10624c0069672000626974002066690072737400cb
:10625c0020426f006f746c006f61640065722000e7
:10626c00762031002e20480045580d000a203200bf
:10627c002e20440045430d000a2033002e204200fe
:10628c00494e0d000a2034002e2052004157440084
:10629c00697370006c61790020666f00726d61002b
:1062ac0074207300657456006f6c74006167650030
:1062bc00206d6f006e6974006f7273003a203500a8
:1062cc00563a2000207c2000332e3300563a200012
:1062dc00207c2000565055004c4c5500503a200064
:1062ec005365740020736500726961006c20700046
:1062fc006f72740020737000656564003a2028008a
:10630c0062707300290d0a0020312e0020333000fa
:10631c00300d0a0020322e002031320030300d00ba
:10632c000a2033002e203200343030000d0a2000b9
:10633c00342e200034383000300d0a0020352e0069
:10634c002039360030300d000a2036002e20310066
:10635c0039323000300d0a0020372e00203338003f
:10636c00343030000d0a2000382e2000353736002e
:10637c0030300d000a2039002e203100313532002a
:10638c0030300d000a3130002e20420052472000e0
:10639c0072617700207661006c75650041646a005b
:1063ac007573740020796f0075722000746572002b
:1063bc006d696e00616c410072652000796f75002b
:1063cc002073750072653f002043460047313a0048
:1063dc002043460047323a00285c2d002f5f5c00ba
:1063ec002d2928005c5f2f002d295300656c65005a
:1063fc00637420006f7574007075740020747900dc
:10640c0070653a000d0a2000312e20004f70650097
:10641c006e206400726169006e202800483d4800bf
:10642c00692d5a002c204c003d474e0044290d008c
:10643c000a2032002e204e006f726d00616c20001d
:10644c0028483d00332e3300562c20004c3d47008d
:10645c004e442900523257002028730070642000eb
:10646c0068697a00293d2800202030002e4d6100fb
:10647c0063726f00206d65006e750d000a2031008f
:10648c002e4953004f37380031362d003320410050
:10649c0054520d000a2032002e4953004f37380059
:1064ac0031362d00332070006172730065206f004f
:1064bc006e6c790049534f002037380031362d006f
:1064cc0033204100545220002852450053455400bb
:1064dc00206f6e0020435300290d0a0052455300d3
:1064ec004554200048494700482c2000434c4f009d
:1064fc00434b2000544943004b2c20005245530081
:10650c00455420004c4f570049534f00203738005a
:10651c0031362d003320720065706c007920280014
:10652c00757365007320630075727200656e74007c
:10653c00204c53004220730065747400696e670030
:10654c00293a200050726f00746f63006f6c3a0030
:10655c0020736500726961006c33200077697200ea
:10656c0065322000776972006552460055756e00e1
:10657c006b6e6f00776e5200656164002074790059
:10658c0070653a0020746f0020656e0064766100bf
:10659c0072696100626c6500206c65006e67740046
:1065ac006844610074612000756e690074733a0070
:1065bc00206e6f0020696e0064696300617469006d
:1065cc006f6e44006174610020756e006974200068
:1065dc006c656e0067746800202862006974730033
:1065ec00293a200043532000454e4100424c4500bf
:1065fc004443530020444900534142004c4544005d
:10660c0052335700202873007064200063736c00b1
:10661c00206869007a293d00282029000d0a4400d1
:10662c00697363006f6e6e006563740020616e00a9
:10663c007920640065766900636573000d0a430078
:10664c006f6e6e0065637400202856007075200014
:10665c00746f20002b355600292061006e642000d9
:10666c0028414400432074006f202b00332e33004c
:10667c005629430074726c00415558004d4f44002c
:10668c0045204c0045445000554c4c0055502000c2
:10669c00485055004c4c550050204c00565245006b
:1066ac0047414400432061006e6420007375700004
:1066bc00706c790035565600505533002e33560009
:1066cc0041444300427573002068690067684200ca
:1066dc007573200048692d005a20300042757300f4
:1066ec00204869002d5a2000314d4f0044452000b0
:1066fc00616e640020565200454720004c45440012
:10670c0073207300686f75006c6420006265200054
:10671c006f6e2100466f75006e642000206572005c
:10672c00726f7200732e4d004f534900434c4b0057
:10673c004d4953004f435300204f4b00204641001e
:10674c00494c5300657420007370650065643a0011
:10675c000d0a2000312e200033304b00487a0d00fa
:10676c000a2032002e20310032354b00487a0d00c1
:10677c000a2033002e20320035304b00487a0d00b1
:10678c000a2034002e2031004d487a00436c6f00f3
:10679c00636b2000706f6c006172690074793a0051
:1067ac000d0a2000312e200049646c0065206c001d
:1067bc006f7720002a646500666175006c740d00ab
:1067cc000a2032002e204900646c650020686900a4
:1067dc0067684f007574700075742000636c6f00ef
:1067ec00636b200065646700653a0d000a20310078
:1067fc002e204900646c650020746f0020616300da
:10680c0074697600650d0a0020322e002041630069
:10681c0074697600652074006f206900646c6500f3
:10682c00202a640065666100756c7400496e700006
:10683c007574200073616d00706c650020706800c9
:10684c00617365003a0d0a0020312e00204d69005d
:10685c0064646c0065202a006465660061756c00d8
:10686c00740d0a0020322e0020456e006453500037
:10687c00492028007370640020636b007020730043
:10688c006b652000736d7000206373006c206800d2
:10689c00697a29003d28200020302e004d616300cc
:1068ac00726f20006d656e00750d0a0020312e0090
:1068bc00536e690066662000435320006c6f7700ae
:1068cc000d0a2000322e53006e69660066206100ae
:1068dc006c6c20007472610066666900632d700038
:1068ec00202d6600202a4200797465007320640014
:1068fc00726f7000706564002a464100494c450077
:10690c00442c20004e4f200044415400414461006f
:10691c007461200062697400732061006e64200051
:10692c0070617200697479003a0d0a0020312e00f2
:10693c0020382c00204e4f004e4520002a64650064
:10694c00666175006c7420000d0a2000322e200048
:10695c00382c2000455645004e200d000a203300ef
:10696c002e2038002c204f00444420000d0a20001b
:10697c00342e2000392c20004e4f4e00455374000d
:10698c006f70200062697400733a0d000a203100a8
:10699c002e203100202a640065666100756c74003d
:1069ac000d0a2000322e200032526500636569000a
:1069bc0076652000706f6c006172690074793a0022
:1069cc000d0a2000312e200049646c006520310036
:1069dc00202a640065666100756c74000d0a200045
:1069ec00322e200049646c00652030005541520065
:1069fc0054202800737064002062720067206400c9
:106a0c006270200073622000727870002068690048
:106a1c007a293d0028202000302e4d006163720041
:106a2c006f206d00656e75000d0a2000312e54002c
:106a3c0072616e007370610072656e00742062008a
:106a4c007269640067650d000a2032002e4c6900e3
:106a5c00766520006d6f6e0069746f00720d0a0010
:106a6c0020332e004272690064676500207769004c
:106a7c0074682000666c6f00772063006f6e740082
:106a8c00726f6c000a0d2000342e410075746f007b
:106a9c0020426100756420004465740065637400d5
:106aac00696f6e0055415200542062007269640097
:106abc006765520065736500742074006f20650073
:106acc0078697400526177002055410052542000bf
:106adc00696e70007574550041525400204c490089
:106aec005645200044495300504c4100592c20007d
:106afc007d2054004f205300544f50004c495600f9
:106b0c0045204400495350004c4159002053540037
:106b1c004f5050004544570041524e00494e4700db
:106b2c003a207000696e7300206e6f0074206f0045
:106b3c0070656e002064720061696e002028480048
:106b4c00695a290020524500564944003a0d0a0062
:106b5c00496e7600616c690064206300686f69009f
:106b6c0063652c00207472007920610067616900f4
:106b7c006e6d7300525320004c4f57002c20430075
:106b8c004f4d4d00414e4400204d4f0044455200a6
:106b9c0053204800494748002c20440041544100f0
:106bac00204d4f00444541006464720065737300ce
:106bbc00206f6600205043004638350037343f00c4
:106bcc005468690073206d006f6465002072650065
:106bdc00717569007265730020616e00206164003c
:106bec006170740065724c0043442000747970002d
:106bfc00653a0d000a2031002e2048004434340040
:106c0c00373830002028750073696e0067205000fb
:106c1c00434638003537340020494f002065780052
:106c2c0070616e0064657200294c4300442028009a
:106c3c00747970002061640064722900203d20008a
:106c4c0028202000302e4d00616372006f206d00f3
:106c5c00656e75000d0a2000312e4c004344200057
:106c6c005265730065740d000a2032002e496e00c7
:106c7c00697420004c4344000d0a2000332e43005d
:106c8c006c65610072204c0043440d000a203400f6
:106c9c002e43750072736f00722070006f73690061
:106cac0074696f006e206500783a28003429200042
:106cbc00300d0a0020362e005772690074652000d2
:106ccc007465730074206e00756d620065727300dc
:106cdc00206578003a28360029203800300d0a004b
:106cec0020372e005772690074652000746573009c
:106cfc0074206300686172006163740065727300d4
:106d0c00206578003a283700292038003044690083
:106d1c0073706c00617920006c696e0065733a00c9
:106d2c000d0a2000312e200031200d000a203200e7
:106d3c002e204d00756c740069706c0065494e0016
:106d4c00495443004c4541005243550052534f00a7
:106d5c005220530045544e006f204100434b2c00f1
:106d6c002063680065636b002061640061707400cf
:106d7c00657243004c4b09004d4f530049094300c9
:106d8c0053094d0049534f0050696e0073746100f4
:106d9c00746573003a474e00440933002e33560095
:106dac0009352e0030560900414443000956500065
:106dbc005509410055580900500950000950090067
:106dcc0049094900092d09004f574400092d0900b4
:106ddc002d2d090054784400092d090052784400e7
:106dec0053434c000953440041092d00092d500018
:106dfc004743090050474400092d09002d312e004e
:106e0c0028425200290932002e2852004429090038
:106e1c00332e28004f52290009342e0028595700d0
:106e2c00290935002e2847004e290900362e280046
:106e3c00424c290009372e002850550029093800ea
:106e4c002e28470052290900392e280057542900b2
:106e5c0009302e0028426c006b2947004e44090073
:106e6c00474e440009414400430935002e3056007a
:106e7c0009332e0033560900565055000941550070
:106e8c00580965007865630075746500203a200028
:106e9c0020617500746f7200616e670065202b00b5
:106eac004d487a00292b6b00487a290052617700f3
:106ebc00207661006c75650020666f0072204200c0
:106ecc0052472000284d490044493d0031323700db
:106edc0029574100524e49004e473a0020506f004e
:106eec0073736900626c65002062750066666500ec
:106efc00726f7600657266006c6f7700416e790078
:106f0c00206b6500792074006f206500786974002f
:106f1c005370610063652000746f2000636f6e0016
:106f2c0074696e0075654e00756d620065722000a7
:106f3c006f662000626974007320720065616400e2
:106f4c002f777200697465003a204300533a0d00a4
:106f5c000a2031002e204300530d0a0020322e004f
:106f6c00202f430053202a006465660061756c0075
:106f7c0074506f0073697400696f6e0020696e0045
:106f8c002064650067726500657353006572760056
:106f9c006f20610063746900766557006169740045
:106fac00696e67002061630074697600697479000a
:106fbc002e2e2e002a2a2000456172006c792000aa
:106fcc004578690074212a002a42610075643e00ec
:106fdc0031366d003a20420050204300616e6e0045
:106fec006f7420006d6561007375720065203e0042
:106ffc002031360030303000303030002c2044004e
:10700c006f6e65002e0a0d0043616c0063756c0099
:10701c0061746500643a2000090a0d004573740020
:10702c00696d6100746564003a20200009206200db
:10703c007073200047656e00657261006c09090071
:10704c000909090050726f00746f63006f6c2000a7
:10705c00696e740065726100637469006f6e200064
:10706c002d2d2d002d2d2d002d2d2d002d2d2d00f8
:10707c002d2d2d002d2d2d002d2d2d002d2d2d00e8
:10708c002d2d2d002d2d2d002d2d2d002d2d2d00d8
:10709c002d2d2d002d2d2d002d2d2d002d2d2d00c8
:1070ac002d2d2d002d2d2d002d2d2d002d2d2d00b8
:1070bc002d2d2d002d2d2d002d2d2d002d2d2d00a8
:1070cc002d2d2d00203f09005468690073206800a5
:1070dc00656c70000909090028302900094c690009
:1070ec00737420006375720072656e0074206d00fd
:1070fc00616372006f7320003d582f007c580900ab
:10710c00436f6e007665720074732000582f720006
:10711c0065766500727365002058090009287800af
:10712c0029094d00616372006f207800207e0900f0
:10713c0053656c00667465007374090009095b0083
:10714c0009537400617274002023090052657300a6
:10715c0065742000746865002042500020202000d7
:10716c00090909005d095300746f7000202409009f
:10717c004a756d00702074006f2062006f6f740090
:10718c006c6f61006465720009097b00095374001f
:10719c006172740020776900746820007265610068
:1071ac00642026002f25090044656c0061792000bd
:1071bc0031207500732f6d0073090900097d0900da
:1071cc0053746f00702061002f412f004009410063
:1071dc0055585000494e2000286c6f00772f4800fe
:1071ec00492f5200454144002909090022616200df
:1071fc006322090053656e00642073007472690089
:10720c006e6720006209530065742000626175008e
:10721c006472610074650900090931003233200081
:10722c00632f4300094155005820610073736900b6
:10723c00676e6d00656e74002028610075782f00f4
:10724c00435329000909300078313200332064009f
:10725c002f4409004d656100737572006520410073
:10726c0044432000286f6e0063652f00434f4e008f
:10727c00542e290009306200313130000953650069
:10728c006e64200076616c007565200066094d0007
:10729c00656173007572650020667200657175001a
:1072ac00656e63007909090072095200656164001a
:1072bc0020672f0053094700656e650072617400ea
:1072cc0065205000574d2f0053657200766f0900f2
:1072dc00092f0900434c4b00206869002068090005
:1072ec00436f6d006d616e006468690073746f00ac
:1072fc007279090009095c0009434c004b206c00b1
:10730c006f20690009566500727369006f6e690021
:10731c006e666f002f7374006174750073696e0074
:10732c00666f0900095e0900434c4b00207469002c
:10733c00636b20006c2f4c0009426900746f720063
:10734c006465720020286d0073622f004c5342005c
:10735c00290909002d0944004154200068692000c6
:10736c006d09430068616e00676520006d6f6400f5
:10737c0065090900095f090044415400206c6f0045
:10738c00206f090053657400206f750074707500d0
:10739c007420740079706500090909002e094400f5
:1073ac004154200072656100642070002f50090068
:1073bc0050756c006c7570002072650073697300f9
:1073cc00746f7200732028006f6666002f4f4e009a
:1073dc00290921000942690074207200656164006a
:1073ec0020730900536372006970740020656e008d
:1073fc0067696e0065090900093a09005265700059
:10740c006561740020652e00672e2000723a3100f1
:10741c0030207600095368006f772000766f6c007f
:10742c0074732f00737461007465730009092e0066
:10743c000942690074732000746f2000726561004a
:10744c00642f770072697400652065002e672e002a
:10745c002030780035352e00322077002f57090068
:10746c005053550020286f0066662f004f4e2900a0
:10747c0009093c00783e2f003c783d00203e2f004f
:10748c003c303e000955730065726d0061637200fb
:10749c006f2078002f617300736967006e2078008d
:1074ac002f6c690073742000616c6c000000fa0092
:1074bc00819c2100114078000060a0008048780079
:1074cc0040a3210010407800684060000004e000f8
:1074dc0002003200cac2a90001003700cac2a800cb
:1074ec0040a3210010407800684060000004e000d8
:1074fc0003003200f0c2b3002c7302000000000045
:10750c00a100200090ab2000be8c02000000000007
:10751c000080fa00000006000000fa00819c2100a7
:10752c00114078000060a1008048780040a3210041
:10753c0010407800684060000004e0000200320057
:10754c00cac2a90001003700cac2a80040a321008a
:10755c0010407800684060000004e0000300320036
:10756c00f0c2b3002c73020000000000a100200048
:10757c0090ab2000be8c0200000000000080fa00de
:10758c00000006000000fa0040a321001040780023
:10759c00684060000004e00002003200cac2a8008b
:1075ac0001003700cac2a90040a321001040780096
:1075bc00684060000004e00003003200f0c2b30039
:1075cc002c73020000000000b100200030ac200041
:1075dc00be8c0200000000000080fa0000000600d3
:1075ec000000fa0000c0eb00730207000080fb00f3
:1075fc000080fa00000006000400fa001007980052
:10760c001e009000004078006b020700004f7800cd
:10761c00809c2100104078000044b2000004e0007f
:10762c00020032001e80fb00010037000000eb005e
:10763c000080fa00000006000000fa0001022000a1
:10764c0000ca2000328c020000000000609b210068
:10765c00104078000040e800847002000000000038
:10766c0000c2b3002c7302000000000040a32100f4
:10767c00100078006140600084700200000000007f
:10768c0000c2b3002c7302000000000040a32100d4
:10769c00100078000000d10061406000847002008e
:1076ac000000000000c2b3002c73020000000000b8
:1076bc0040a32100100078004200de006140600011
:1076cc00847002000000000000c2b3002c730200a2
:1076dc000000000040a32100100078004300de00f1
:1076ec0061406000847002000000000000c2b30022
:1076fc002c73020000000000809c21001080fb0015
:10770c004400de0061406000847002000000000054
:10771c0000c2b3002c7302000000000031002000f6
:10772c0020ae2000328c0200000000000080fa0025
:10773c00000006000c00fa00742302000000000098
:10774c00721f020000000000000f7800742302007a
:10775c0000000000721f02000000000010079800db
:10776c007423020000000000721f020000000000e1
:10777c00200798007423020000000000721f020012
:10778c000000000030079800742302000000000085
:10779c00721f0200000000004007980074230200d2
:1077ac0000000000721f020000000000500798004b
:1077bc001e0078000000e000090034001e00780074
:1077cc00e40f500006003c001e00780000407800da
:1077dc008040e900609b21000148780002003700de
:1077ec000000eb00000f78001e0090000000e0008d
:1077fc000f0034001e009000e20f50000c003c0003
:10780c001e009000004078000040e900e14060005c
:10781c0040a32100e1c0600090417800e2cfb300aa
:10782c0002c16100814071000148780002003700fc
:10783c000000eb00000f78002e0090000000e0002c
:10784c00100034002e009000e20f50000d003c00a0
:10785c002e009000004078000040e900e1406000fc
:10786c0040a32100e1c0600081c04000904178003d
:10787c00d2cfb30002c16100814071000148780091
:10788c00020037000000eb00000f78003e00900073
:10789c000000e000110034003e009000e20f5000a8
:1078ac000e003c003e009000004078000040e900d3
:1078bc00e140600040a3210061c160002100200074
:1078cc008110dd0090417800b2cfb30002c161009d
:1078dc008140710001487800020037000000eb0085
:1078ec00000f78004e0090000000e0001100340002
:1078fc004e009000e20f50000e003c004e00900035
:10790c00004078000040e900e140600040a3210005
:10791c0061c16000310020008110dd0090417800d1
:10792c0072cfb30002c16100814071000148780040
:10793c00020037000000eb00000f78005e009000a2
:10794c000000e000110034005e009000e20f5000d7
:10795c000e003c005e009000004078000040ea0001
:10796c00e1406000809c210061c16000410020006a
:10797c008110dd0090417800f2ceb30002c16100ad
:10798c008140710001487800020037000000eb00d4
:10799c00000f78001e0078000000e0007d003a0027
:1079ac00408821008040eb000148780071032000e2
:1079bc0000bc2000be8c0200000000008001eb0027
:1079cc00420020001100200010002000fe250200c3
:1079dc0000000000004078008040e900609b21001e
:1079ec00014878005103200070bf2000be8c0200bb
:1079fc00000000008001eb0022002000110020009c
:107a0c0010002000fe25020000000000004078005d
:107a1c000040e900e140600040a32100e1c06000ab
:107a2c0090417800e2cfb30002c161008140710047
:107a3c000148780031042000c0c22000be8c020036
:107a4c00000000008001eb0022002000110020004b
:107a5c0020002000fe2502000000000000407800fd
:107a6c000040e900e140600040a32100e1c060005b
:107a7c0081c0400090417800d2cfb30002c16100b8
:107a8c00814071000148780011032000f0c62000ed
:107a9c00be8c0200000000008001eb0022002000e0
:107aac001100200010002000fe2502000000000044
:107abc00004078000040e900e140600040a3210054
:107acc0061c16000210020008110dd009041780030
:107adc00b2cfb30002c1610081407100014878004f
:107aec00d1012000601c2100be8c020000000000af
:107afc008001eb002200200011002000200020005b
:107b0c00fe25020000000000004078000040e90063
:107b1c00e140600040a3210061c160003100200001
:107b2c008110dd009041780072cfb30002c161007a
:107b3c008140710001487800f1042000e09320009e
:107b4c00be8c0200000000008001eb00220020002f
:107b5c001100200010002000fe2502000000000093
:107b6c00004078000040ea00e1406000809c210069
:107b7c0061c16000410020008110dd00904178005f
:107b8c00f2ceb30002c1610081407100014878005f
:107b9c0001003700a8fe0700819c210011407800ed
:107bac000060a100804878000080fa000000060008
:107bbc000000fa00609b2100104078000080fb0060
:107bcc0081b12800614078009a00070040a3210091
:107bdc00100078004300de00614060000080fb0074
:107bec00610060004600dd0052168000f1fb2f00a2
:107bfc008100610001007000501688000080fa00be
:107c0c00000006000000fa00d90007000080fa000e
:107c1c00000006000200fa00000f78001e00780039
:107c2c008000eb00f200200003002000820f5000c7
:107c3c00838f580070003e00006001000f00370079
:107c4c00130037001e003700700037006a00370041
:107c5c00690037006800370067003700660037009e
:107c6c006500370022003700260037002a00370055
:107c7c002e00370032003700360037004103200059
:107c8c0000cc2000be8c0200000000006000370019
:107c9c007100200070562000be8c02000000000015
:107cac00f1002000b0182100be8c02000000000082
:107cbc0011c0b3000040eb00cf00070054003700a8
:107ccc007100200070562000be8c020000000000e5
:107cdc00f1002000b0182100be8c02000000000052
:107cec0011c0b30010c0b300c30007004800370038
:107cfc0041a32100114078000000a10080487800c9
:107d0c001800370041a32100114078000000a000aa
:107d1c00804878001300370041a3210011407800ff
:107d2c000010a100804878000e00370041a321000c
:107d3c00114078000010a00080487800090037003e
:107d4c0041a32100114078000020a1008048780058
:107d5c000400370041a32100114078000020a0004e
:107d6c008048780040a3210010007800614060003a
:107d7c000080fb00610060004600dd0012128000f4
:107d8c00f1fb2f00810061000100700010128800cf
:107d9c0040a32100100078000000d1006140600079
:107dac000080fb00610060004800dd0012128000c2
:107dbc00f1ef2f00810061000100700010128800ab
:107dcc0040a32100100078004200de0061406000fa
:107ddc000080fb00610060004900dd001212800091
:107dec00f1df2f008100610001007000101288008b
:107dfc0011fe07000600370041022000e01d2000a4
:107e0c00be8c0200000000000100370000000000e2
:107e1c000080fa00000006000000fa0001012000ba
:107e2c0040062100be8c0200000000000080fa0019
:107e3c00000006000200fa00004f780041e2a900a1
:107e4c00809c210010407800704060000004e0002d
:107e5c0004003200cf22a800cf02a800cec2a80096
:107e6c0003003700cf22a900cf02a900cec2a9007f
:107e7c004135800000fe2f00008060007000b300d0
:107e8c004035880041368000f00f2e008080600065
:107e9c0000702000010070004036880041368000e0
:107eac0000fe2f00008060000030a00040368800eb
:107ebc00cac2a800c8c2a900c902a900c8e2a80089
:107ecc00c922a9001e80fb001012880042a2a80043
:107edc0040a3210010007800614060000080fb008e
:107eec00610060004600dd0012128000f1fb2f00e3
:107efc0081006100010070001012880040a3210075
:107f0c00100078000000d100614060000080fb0090
:107f1c00610060004800dd0012128000f1ef2f00bc
:107f2c0081006100010070001012880040a3210044
:107f3c00100078004200de00614060000080fb0011
:107f4c00610060004900dd0012128000f1df2f009b
:107f5c008100610001007000101288004422ef00c3
:107f6c004022ef0041e2a8000080fa000000060069
:107f7c000000fa0041e2a90040358000f001b30096
:107f8c004035880041368000f00f2e0000806000e4
:107f9c00403688004136800000fe2f0000806000d3
:107fac0040368800cf22a900cf02a900cec2a9007a
:107fbc000080fa00000006000200fa00004f780072
:107fcc001e80fb004012880000000000210480008d
:107fdc0000402000008060000000e000fbff320049
:107fec0040128000004f78008540a9001e407800a8
:107ffc000080fa00000006000400fa0020479800f8
:10800c003147980010c0b300004f78004272020054
:10801c0000000000d6ff0700890007002e409000ea
:10802c000004e00002003a0042e2a80062e2a8006c
:10803c002e409000e14f500004003e0041e2a800a9
:10804c0061e2a80001003700000000001e4078002b
:10805c000004e0000a003a005116800000042000e1
:10806c00008060000000e00005003200d0c5b300c5
:10807c00d07202000000000010c0b300004f780066
:10808c000112800000022000008060000000e0006f
:10809c0030003a00011380000002200000806000d4
:1080ac000000e0002b003a004012800010479800be
:1080bc001e407800e14f500005003a00b0c5b300f7
:1080cc00d0720200000000000040eb00004f78006e
:1080dc003e4090000004e000050032001e4090007d
:1080ec000080fb0014710200000000000600370045
:1080fc00c0c5b300d0720200000000001e4090000a
:10810c00d07202000000000040138000104798005d
:10811c003e4090000004e0000b00320080c2b3002f
:10812c00d0720200000000001e4090000080fb0096
:10813c00147102000000000090c2b300d072020063
:10814c0000000000030037001e409000d0720200b7
:10815c00000000000112800000042000008060007c
:10816c000000e0000a003a00011380000004200027
:10817c00008060000000e00005003a00e1cf8000c4
:10818c0000202000008060000000e000120032009f
:10819c00e1cf800000202000008060000000e000a3
:1081ac0002003a0092720200000000004022ef0030
:1081bc006022ef003e4090000004e000040032001a
:1081cc00c0b12800166e0200000000008dff3700c1
:1081dc00c222a900110037005672020000000000f4
:1081ec003672020000000000e14f500096ff3a008a
:1081fc000673020000000000104798003e409000fb
:10820c000004e00004003200d0b22800166e020018
:10821c000000000001003700000000007b00070098
:10822c00609b2100104078000080fb0081b1280089
:10823c0061407800fffe07000080fa000000060095
:10824c000000fa00c8c2a800c902a800c8e2a80031
:10825c00c922a8005135800000fe2f00008060006c
:10826c006000b300503588007135800000fe2f008f
:10827c00008060006000b3007035880041358000dc
:10828c0000fe2f00008060009000b3004035880095
:10829c0041358000f00f2e008080600000802000af
:1082ac0001007000403588006135800000fe2f0011
:1082bc00008060007000b30060358800613580007c
:1082cc00f00f2e0080806000008020000100700004
:1082dc0060358800609b2100104078000080fb0016
:1082ec0081b12800614078000080fb0010128800ea
:1082fc0040a3210010007800614060000080fb006a
:10830c00610060004600dd0012128000f1fb2f00be
:10831c0081006100010070001012880040a3210050
:10832c00100078000000d100614060000080fb006c
:10833c00610060004800dd0012128000f1ef2f0098
:10834c008100610001007000101288004422ef00cf
:10835c004022ef00609b2100104078000080fb0061
:10836c0081b12800614078000080fb001013880068
:10837c0040a3210010007800614060000080fb00e9
:10838c00610060004600dd0012138000f1fb2f003d
:10839c0081006100010070001013880040a32100cf
:1083ac00100078000000d100614060000080fb00ec
:1083bc00610060004800dd0012138000f1ef2f0017
:1083cc008100610001007000101388006422ef002e
:1083dc006022ef004822ef006822ef004322a90040
:1083ec006322a9004362a80042a2a9006362a8000c
:1083fc0062a2a90040c2a90060c2a9004402a80060
:10840c006402a8000080fa00000006000000fa00d8
:10841c0041e2a9004362a90061e2a9006362a900dc
:10842c0050358000f001b300503588007035800065
:10843c00f001b3007035880040358000f001b300c6
:10844c00403588004135800000f0210001007000ab
:10845c004035880060358000f001b300603588003d
:10846c006135800000f0210001007000603588004b
:10847c000080fa00000006000000fa0060b328003b
:10848c00f26d0200000000000080fa0000000600ff
:10849c000e00fa00881f7800609b210011c0b30009
:1084ac000148780041a32100114078000000a10090
:1084bc008048780041a32100114078000010a000f2
:1084cc008048780041a32100114078000020a100d1
:1084dc0080487800819c2100114078000040a00069
:1084ec0080487800609b2100104078000080fb00e1
:1084fc00e1b22800614078004efe0700deff070065
:10850c00067302000000000051a32100804878008f
:10851c0050a32100104078000080fb004400de00d6
:10852c008040780060a321000148780060a32100fe
:10853c00104078000080fb00e40f50008c013200ea
:10854c00e40f500005003c000000e0000800320081
:10855c00e10f500064013200e3013700e60f5000d8
:10856c008b013200e80f50009c013200de01370015
:10857c0050a32100104078000080fb00e50f500054
:10858c000e003c00e40f500037003d00e10f50009e
:10859c0015003200e10f500003003c000000e00029
:1085ac000d0032004b013700e20f5000100032007a
:1085bc00e30f50001600320046013700ed0f50005b
:1085cc001b003200ee0f500020003200e60f50006e
:1085dc008f0032003f01370065fe07004f04780022
:1085ec000080fa0000000600a3ff07003d013700e1
:1085fc0061168000f0fb2f00008060006016880080
:10860c0010c0b3002c7302000000000035013700cd
:10861c0061168000000420000100700060168800c4
:10862c0010c0b3002c730200000000002d013700b5
:10863c0010c0b3002c730200000000008040eb005f
:10864c0010c0b3006cfe07002601370010c0b30049
:10865c002c730200000000008040eb000040eb0097
:10866c0065fe07001f0137000673020000000000c2
:10867c000080fb00500798005e0090004800dd0071
:10868c005007980006730200000000000080fb00f9
:10869c00de00900001007000500798000673020085
:1086ac00000000000080fb00600798006e00900046
:1086bc004800dd006007980006730200000000000f
:1086cc000080fb00ee009000010070006007980035
:1086dc00de00900000002100808f500004003e005e
:1086ec00ee00900000002100808f50000400360046
:1086fc000040eb002c73020000000000f900370072
:10870c000000eb00000f78000600370080cf8000df
:10871c001e0440000673020000000000004c7800ac
:10872c001e0fe8005e0090009e007800808f5000c5
:10873c00f6ff390050a3210010407800e44f5000a0
:10874c0001003a00cac2a9000000eb00000f78003b
:10875c000500370080cf80001e00400010407800dc
:10876c0015fe07001e0fe8005e0090009e007800ca
:10877c00808f5000f7ff390010002000b28b0200f0
:10878c00000000000000eb00000f7800060037002e
:10879c0080cf80001e04400000c0eb0006fe0700e6
:1087ac00004c78001e0fe8006e0090009e007800d0
:1087bc00808f5000f6ff390050a321001040780044
:1087cc00e44f500001003a00cac2a80010c0b30028
:1087dc002c730200000000000000eb00000f78007a
:1087ec000600370080cf80001e004000104078004b
:1087fc002c730200000000001e0fe8006e009000b9
:10880c009e007800808f5000f6ff3900b5003700cd
:10881c0010c0b3002c7302000000000006730200ad
:10882c000000000051a321008048780050a32100d3
:10883c00104078000080fb00e10f5000080032006f
:10884c00e20f5000100032000000e0009c003a00e3
:10885c0010c0b3002c730200000000009c00370015
:10886c0010c0b3002c730200000000000040eb00ad
:10887c002c7302000000000010c0b3002c73020027
:10888c0000000000920037006000b800100798004c
:10889c00210798000000eb00000f78001300370050
:1088ac00067302000000000051a3210080487800ec
:1088bc001e009000ae0090004809dd00c801de00eb
:1088cc00830171004801dd0050a3210010407800a5
:1088dc000080fb008000eb000000710081807100c3
:1088ec0010079800210798001e0fe8001e00780062
:1088fc00e30f5000eaff36006000b8003007980024
:10890c00410798000000eb00000f780013003700bf
:10891c00067302000000000051a32100804878007b
:10892c003e009000ce0090004809dd00c801de003a
:10893c00830171004801dd0050a321001040780034
:10894c000080fb008000eb00000071008180710052
:10895c0030079800410798001e0fe8001e007800b1
:10896c00e30f5000eaff36001e019000ae019000ac
:10897c00f0ff2f0001002000800f5100818f590063
:10898c0012003e003e019000ce019000f0ff2f003f
:10899c0001002000800f5100818f59000b003e0018
:1089ac001e019000ae0190003e009000ce009000a1
:1089bc000201400083814800f0ff2f0001002000dd
:1089cc00800f5100818f5900040036000040eb00ed
:1089dc002c730200000000003800370010c0b300f8
:1089ec002c730200000000009e009000010f780024
:1089fc002d00370000c2b3006ffd07001e00780089
:108a0c004800de00004078006bfd07001e00780077
:108a1c000040780068fd07000040eb0066fd070091
:108a2c002c730200000000003e009000ce0090006d
:108a3c0061005000e0805800300798004107980012
:108a4c003e009000ce009000e00f5000e08f5800e8
:108a5c0001003a001900370080c2b30056fd070030
:108a6c001e0078004800de000040780052fd070030
:108a7c001e007800004078004ffd07000040eb001e
:108a8c004dfd07002c730200000000003e0090001a
:108a9c00ce00900061005000e08058003007980034
:108aac00410798001e0fe8003e009000ce00900099
:108abc00e00f5000e08f5800ceff3a000400370062
:108acc000040eb002c7302000000000000000000ce
:108adc00040037000040eb002c7302000000000083
:108aec00000000008400370050a3210010407800e3
:108afc00ef40600050a321000148780050a32100f2
:108b0c00104078008040e80050a321000148780014
:108b1c0010c0b3002c7302000000000070a32100f1
:108b2c008040eb00014878000a0037000673020011
:108b3c000000000020fd07002c7302000000000064
:108b4c0070a32100104078008040e80070a3210041
:108b5c000148780070a321009040780050a32100b8
:108b6c001040780080cf5000f0ff390062003700d1
:108b7c0050a32100104078005a9102000000000020
:108b8c0010c0b3002c730200000000005a00370024
:108b9c0050a3210010407800e740600050a3210052
:108bac000148780050a3210090407800609b210080
:108bbc0001487800609b2100104078000080fb0089
:108bcc00e1b22800614078009afc070010c0b300a5
:108bdc002c730200000000004700370041a3210065
:108bec00114078000000a1008048780041a32100ca
:108bfc00114078000010a1008048780041a32100aa
:108c0c00114078000020a10080487800819c210050
:108c1c00114078000040a1008048780050a321004a
:108c2c00104078000080fb00640060000000e00051
:108c3c000400320041a32100114078000000a00084
:108c4c008048780050a32100104078000080fb0081
:108c5c00620060000000e0000400320041a321002b
:108c6c00114078000010a0008048780050a321002b
:108c7c00104078000080fb0061006000004078002c
:108c8c000004e0000400320041a3210011407800f0
:108c9c000020a0008048780050a3210010407800ec
:108cac000080fb00680060000000e00004003a0057
:108cbc00819c2100114078000040a0008048780081
:108ccc00609b2100104078000080fb00e1b228007e
:108cdc006140780057fc070010c0b3002c730200f1
:108cec0000000000040037000040eb002c73020071
:108cfc00000000000000000001fe37000200fa0036
:108d0c008e8f0200000000000004e0002100320001
:108d1c0090118000680060000000e0000400320048
:108d2c003100200040cf2000328c020000000000f7
:108d3c0090118000640060000000e000040032002c
:108d4c003100200070cf2000328c020000000000a7
:108d5c007c8f020000000000000f78009011800052
:108d6c00620060000000e00008003200f10020000a
:108d7c00a0cf2000328c0200000000009111800076
:108d8c00d0ff2f0000806000901188001e0078003a
:108d9c0005003700f100200090d02000328c02003a
:108dac00000000000000eb000080fa00000006004c
:108dbc000200fa00000f78001e007800648f020099
:108dcc00000000000000eb000080fa00000006002c
:108ddc000000fa0001022000f0db2000328c0200bf
:108dec0000000000609b210010407800847002009d
:108dfc000000000000c2b3002c7302000000000051
:108e0c00609b210010407800e94f500007003a00a9
:108e1c00c01180001c7002000000000000c2b300f2
:108e2c002c730200000000000c003700609b210036
:108e3c00104078000080fb0080004000e0a7280074
:108e4c0000804000100078001c7002000000000040
:108e5c0000c2b3002c7302000000000040a12100ee
:108e6c001000780063406000847002000000000075
:108e7c0000c2b3002c7302000000000040a12100ce
:108e8c00100078004200de00614060008470020037
:108e9c000000000000c2b3002c73020000000000b0
:108eac0040a12100100078004300de00614060000a
:108ebc00847002000000000000c2b3002c7302009a
:108ecc0000000000809c21001080fb004400de00ac
:108edc0061406000847002000000000000c2b3001a
:108eec002c730200000000003100200020ae200096
:108efc00328c0200000000000080fa000000060026
:108f0c001000fa000000eb00100798006000b80099
:108f1c00200798003107980074230200000000001d
:108f2c00721f020000000000000f78001e00780085
:108f3c00ea0f500005003a00742302000000000004
:108f4c00721f02000000000010079800742302003a
:108f5c0000000000721f0200000000004007980093
:108f6c007423020000000000721f020000000000c9
:108f7c00500798007423020000000000721f0200ca
:108f8c00000000006007980074230200000000003d
:108f9c00721f020000000000700798001e0078008d
:108fac000000e000090034001e007800ea0f5000b9
:108fbc0006003c001e007800004078008040e9006c
:108fcc00609b210001487800020037000000eb0094
:108fdc00000f78004e0090000000e0000f003400fd
:108fec004e009000e40f50000c003c004e0090002e
:108ffc00004078000040e900e340600040a12100ff
:10900c00e3c0600090417800c2cfb30002c16100a0
:10901c008140710001487800020037000000eb002d
:10902c00000f78005e0090000000e000110034009a
:10903c005e009000e20f50000e003c005e009000bd
:10904c00004078000040e900e140600040a12100b0
:10905c0061c16000210020008110dd00904178008a
:10906c00b2cfb30002c161008140710001487800a9
:10907c00020037000000eb00000f78006e0090003b
:10908c000000e000110034006e009000e20f500070
:10909c000e003c006e009000004078000040e9009b
:1090ac00e140600040a1210061c16000310020005e
:1090bc008110dd009041780072cfb30002c16100d5
:1090cc008140710001487800020037000000eb007d
:1090dc00000f78007e0090000000e00011003400ca
:1090ec007e009000e20f50000e003c007e009000cd
:1090fc00004078000040ea00e1406000809c2100c4
:10910c0061c16000410020008110dd0090417800b9
:10911c00f2ceb30002c161008140710001487800b9
:10912c00020037000000eb00000f78001e007800f2
:10913c000000e00079003a00408821008040eb00fc
:10914c0001487800d108200060872000be8c020006
:10915c00000000008001eb00a200200011002000a4
:10916c0010002000fe2502000000000000407800e6
:10917c008040e900609b210001487800609b210041
:10918c0010407800e94f50000d003a00c10120005a
:10919c00f0142100be8c0200000000008001eb00e6
:1091ac00f2ff27001100200020022000fe25020003
:1091bc0000000000100798001e009000c0118800ed
:1091cc004105200080d12000328c020000000000fc
:1091dc008001eb0042002000110020001000200054
:1091ec00fe25020000000000004078000040e9006d
:1091fc00e340600040a12100e3c060009041780092
:10920c00c2cfb30002c161008140710001487800f7
:10921c0011022000c0d62000328c02000000000099
:10922c008001eb0022002000110020001000200023
:10923c00fe25020000000000004078000040e9001c
:10924c00e140600040a1210061c1600021002000cc
:10925c008110dd0090417800b2cfb30002c16100f3
:10926c00814071000148780021032000d0d82000f3
:10927c00328c0200000000008001eb002200200074
:10928c001100200010002000fe250200000000004c
:10929c00004078000040e900e140600040a121005e
:1092ac0061c16000310020008110dd009041780028
:1092bc0072cfb30002c16100814071000148780097
:1092cc00f1042000e0932000be8c0200000000009e
:1092dc008001eb0022002000110020001000200073
:1092ec00fe25020000000000004078000040ea006b
:1092fc00e1406000809c210061c1600041002000c1
:10930c008110dd0090417800f2ceb30002c1610003
:10931c0081407100014878001a003700609b2100e1
:10932c0010407800e94f500015003a001e009000e4
:10933c00cf80de0020079800310798002e019000a6
:10934c00be01900000902000d10320008606020090
:10935c000000000061005000e080580020079800d9
:10936c0031079800ae009000110798006000b8001b
:10937c0020079800310798001e009000c01188004b
:10938c0093fe07000080fa00000006000000fa00bf
:10939c00609b210010407800e94f500017003a0004
:1093ac0040a12100100078004200de006140600006
:1093bc000042780040a1210010007800634060005a
:1093cc008041780040a12100100078004300de00ad
:1093dc006140600000417800809c21001080fb00ff
:1093ec004400de006140600080407800c0118000c5
:1093fc00a88e0200000000001c00370040a12100d4
:10940c00100078004200de006140600000427800ed
:10941c0040a121001000780063406000804178007a
:10942c0040a12100100078004300de006140600084
:10943c0000417800809c21001080fb004400de007d
:10944c006140600080407800609b210010407800f3
:10945c000080fb0080024000e0a728000080420052
:10946c0010007800a88e02000000000040a121002e
:10947c001040780063406000e34f500003003a0056
:10948c00709b210091c0b300014878003a8f020014
:10949c0000000000c111800040118000808f50003e
:1094ac000400310001022000b0162100be8c020025
:1094bc00000000000080fa00000006000000fa0026
:1094cc00488f0200000000000080fa000000060037
:1094dc000200fa00000f78001e007800e20f500026
:1094ec006b003200e20f500005003e000000e0006f
:1094fc0008003200e10f50000f00320095003700d9
:10950c00e30f500008003200e40f500082003200dc
:10951c0090003700a1062000f0dd2000328c020004
:10952c000000000093003700c062a900c082a800b0
:10953c00c8c2a800c902a900b100200090e4200014
:10954c00be8c020000000000d100200040e520008d
:10955c00be8c020000000000648d020000000000c0
:10956c000004a2000004e0007f003a00911180008a
:10957c00d0ff2f00008060009011880001003700a0
:10958c000000000090118000610060000000e0000d
:10959c0007003200111180000020200000806000c4
:1095ac000000e00002003a00b01180002011880099
:1095bc003672020000000000e14f500009003a0032
:1095cc009111800000202000008060000000e0006d
:1095dc0004003a0006730200000000000080fb004b
:1095ec00a011880090118000620060000000e00073
:1095fc0004003a0010118000620060000000e000de
:10960c000900320091118000d0ff2f000080600013
:10961c009011880011118000d0ff2f000080600095
:10962c0010118800c222a9001e007800e30f500020
:10963c00d3ff3a00101680004400de006140600049
:10964c000080fb00610060004800dd0052168000c5
:10965c00f1ef2f00810061000100700050168800ae
:10966c00501680004600de00614060000080fb0068
:10967c00610060004300dd001216800071ff2f00b6
:10968c00810061000100700010168800bdff3700da
:10969c00e100200010e62000be8c0200000000005b
:1096ac00f1002000b0182100be8c02000000000068
:1096bc0091118000d0ff2f00008060009011880075
:1096cc000100370000000000901180006100600074
:1096dc000000e00007003200111180000020200083
:1096ec00008060000000e00002003a00b011800031
:1096fc00201188003672020000000000e14f50007b
:10970c00f0ff3a0006730200000000000080fb002e
:10971c00000f780017003700488f0200000000008f
:10972c000000eb00e30007003a8f0200000000008d
:10973c00c111800040118000808f50000c0031005e
:10974c0001022000b0162100be8c020000000000b7
:10975c000800370041022000e01d2000be8c0200f2
:10976c00000000000300370000000000010037007b
:10977c00000000000080fa00000006000000fa0063
:10978c0091118000d0ff2f000080600090118800a4
:10979c0041a12100114078000040a00080487800d1
:1097ac00819c2100114078000020a00080487800a6
:1097bc00c1012000f0e62000be8c02000000000079
:1097cc000080fa00000006000000fa0041a1210010
:1097dc00114078000040a10080487800819c210055
:1097ec00114078000020a100804878004101200041
:1097fc00b0e82000be8c0200000000000080fa00df
:10980c00000006000200fa000000eb00000f7800d8
:10981c003400370040a121001040780070406000f7
:10982c000004e0002b00320020a92800166e020074
:10983c00000000006100200080662000328c0200d5
:10984c000000000090118000680060000000e00043
:10985c00040032003100200040cf2000328c020086
:10986c000000000090118000640060000000e00027
:10987c00040032003100200070cf2000328c020036
:10988c00000000007c8f020000000000e28a020051
:10989c000000000090118000620060000000e000f9
:1098ac0008003200f1002000a0cf2000328c020012
:1098bc000000000091118000d0ff2f00008060009c
:1098cc009011880020a92800166e020000000000ec
:1098dc00020037007c8f0200000000001000200006
:1098ec00000f78008e8f0200000000000004e000e2
:1098fc00c8ff3a001e00780000f0a7000000ea0044
:10990c000000ea004f00de00004078000080fa0002
:10991c00000006000000fa00b1002000b00a21008f
:10992c00be8c0200000000000080fa00000006005f
:10993c000000fa001e21ef001021ef008000200033
:10994c00800888000821ef000621ef001621ef00a7
:10995c001421ef0080002000f00888000080fa003d
:10996c00000006000000fa0011e1a9001fe1a900a7
:10997c0030348000f001b300303488001e21ef0039
:10998c001021ef000621ef000821ef000080fa0003
:10999c00000006001200fa0070079800010f9800f2
:1099ac006000b80030079800410798006000b800cc
:1099bc0050079800610798006000b800008fbe0047
:1099cc001000200020079800340037002e00900073
:1099dc00c200dd0040a92800008040001001be003c
:1099ec007e0090008e089000800f5100818f5900ee
:1099fc00270036002e0090000000e900c200dd00b8
:109a0c0040a92800008040001001be0052079800b9
:109a1c00630798002e009000c200dd0040a92800ca
:109a2c00008040001001be003207980043079800e8
:109a3c003e019000ce0190005e009000ee00900080
:109a4c0000005100818059008101d1000081d300b8
:109a5c005e009000ee0090000201400083814800ff
:109a6c007e0090008e089000800f5100818f59006d
:109a7c00030031003e009000ce0090000200370041
:109a8c005e009000ee009000008fbe0006003700d4
:109a9c002e0090000000e800200798002e00900097
:109aac00ee0f5000c9ff34001e00be000080fa000b
:109abc00000006000c00fa00500798000000eb00b4
:109acc00000f78006000b80030079800410798003c
:109adc006000b8001007980021079800cae2a9009e
:109aec00c8e2a8005e0090000000e00007003a0009
:109afc003101200020202100be8c0200000000005b
:109b0c0003003700000000000100370000000000d7
:109b1c005116800000082000008060000000e0006a
:109b2c000400320010118000610060000000e000b1
:109b3c00f4ff320010118000610060000000e000b2
:109b4c000900320031118000010f780085ff0700f9
:109b5c00e100200050212100be8c0200000000001a
:109b6c006000b8007d0037000000eb00000f7800ab
:109b7c00440037006eff0700000000005116800003
:109b8c0000082000008060000000e000fbff3200b5
:109b9c001fe1a80011e1a800000000005116800090
:109bac0000082000008060000000e000fbff3a008d
:109bbc0011e1a9001fe1a90030348000f001b300cd
:109bcc00303488001e21ef001021ef004008800087
:109bdc008000eb0030079800410798003e00900091
:109bec00ce009000c000dd0000002000300798007f
:109bfc0041079800300880008000eb003e01900087
:109c0c00ce0190000200400083804800300798008d
:109c1c00410798001e0078000000e000150032009b
:109c2c001e009000ae009000e00f5000e08f580036
:109c3c0005003a003e019000ce01900012079800fa
:109c4c00230798000b0037001e019000ae01900016
:109c5c003e009000ce009000800f5100818f590083
:109c6c00040036003e019000ce01900012079800cf
:109c7c00230798006000b80030079800410798004f
:109c8c001e0fe8001e007800f80f5000b9ff3600d8
:109c9c0034ff07001e019000ae019000004022002e
:109cac00410f2000860602000000000010079800fb
:109cbc00210798005e0090000000e00025003a00ab
:109ccc001e019000ae019000009f24002100200096
:109cdc00800f5100818f590005003600f1022000e1
:109cec0030222100be8c0200000000001900370059
:109cfc00f100200020252100328c02000000000021
:109d0c001e009000ae0090007c6e0200000000006f
:109d1c004100200000272100be8c02000000000042
:109d2c00f100200010262100328c020000000000ff
:109d3c001e009000ae00900016ff07007c6e020023
:109d4c00000000004100200000272100be8c020012
:109d5c00000000001e009000ae0090000080fa0091
:109d6c00000006000000fa0080ae2800f26d020030
:109d7c00000000000080fa00000006000000fa005d
:109d8c0041a12100114078000000a1000010a100a9
:109d9c008048780041a12100114078000020a100ea
:109dac008048780041a12100114078000030a100ca
:109dbc0080487800819c2100114078000040a00070
:109dcc0080487800a0568400b0d0880041a12100c2
:109ddc00114078000040a1008048780040a121008b
:109dec00100078004200de00614060000042780004
:109dfc0040a1210010007800634060008041780091
:109e0c0040a12100100078004300de00614060009a
:109e1c0000417800809c21001080fb004400de0093
:109e2c006140600080407800b0d08000a88e0200b5
:109e3c00000000003a8f020000000000c9ff07007c
:109e4c0001003700000000008e8f020000000000af
:109e5c000004e0000d00320040a121001040780009
:109e6c00704060000004e000060032007c8f0200ad
:109e7c0000000000004078002c730200000000007d
:109e8c00020037007c8f020000000000901180005f
:109e9c00620060000000e0000400320091118000bc
:109eac00d0ff2f00008060009011880036720200f5
:109ebc0000000000e14f5000e2ff3a000673020080
:109ecc000000000081a121008048780080a12100c1
:109edc00104078000080fb004400de0080407800d9
:109eec0090a121000148780090a121001040780039
:109efc000080fb00e40f5000bd003200e40f500066
:109f0c0005003c000000e0000b003200e10f5000a7
:109f1c009200320062013700e60f5000bc003200a4
:109f2c00e60f50005e01350068005000e10f500054
:109f3c005b013e00e800370080a121001040780052
:109f4c000080fb00e20f500014003200e20f5000c2
:109f5c0005003c000000e0000a003200e10f500058
:109f6c000c00320078003700e70f5000230032005d
:109f7c00ef0f500050003200e30f5000170032007a
:109f8c0071003700488f0200000000000080fa00ca
:109f9c000000060073ff07006f00370010c0b3000d
:109fac002c73020000000000901180006200600021
:109fbc000000e0000400320091118000d0ff2f005f
:109fcc00008060009011880041a1210011407800b0
:109fdc000040a000804878005f00370041a12100bc
:109fec00114078000040a1008048780010c0b300f8
:109ffc002c730200000000005700370010c0b300a3
:10a00c002c73020000000000488f020000000000ca
:10a01c0006730200000000000080fb004800dd0019
:10a02c00b0d0880010c0b3002c73020000000000f8
:10a03c0006730200000000008080fb00b0d080009e
:10a04c0001007000b0d0880040a121001000780001
:10a05c004200de00614060000042780040a1210017
:10a06c0010007800634060008041780040a121001e
:10a07c00100078004300de00614060000041780071
:10a08c00809c21001080fb004400de0061406000d9
:10a09c0080407800b0d08000a88e02000000000044
:10a0ac003a8f02000000000010c0b3002c730200b5
:10a0bc00000000002800370010c0b3002c73020011
:10a0cc000000000091118000d0ff2f000080600084
:10a0dc0090118800030037000000000001003700d9
:10a0ec000000000090118000610060000000e000a2
:10a0fc000700320011118000002020000080600059
:10a10c000000e00002003a00b0118000201188002d
:10a11c003672020000000000e14f5000eeff3a00e2
:10a12c009111800000202000008060000000e00001
:10a13c00ebff3a0006730200000000000080fb00f9
:10a14c00a0118800e7ff37000040eb002c730200e1
:10a15c000000000000000000d500370080a12100a5
:10a16c0010407800ef40600080a121000148780089
:10a17c0080a12100104078008040e80080a12100df
:10a18c000148780010c0b3002c73020000000000de
:10a19c00a0a121008040eb00014878000d003700a1
:10a1ac0006730200000000000080fb00648f0200b8
:10a1bc000000000010c0b3002c730200000000006f
:10a1cc00a0a12100104078008040e800a0a121004f
:10a1dc0001487800a0a121009040780080a12100c6
:10a1ec001040780080cf5000edff3900b0003700f0
:10a1fc0080a12100104078005a910200000000005c
:10a20c0010c0b3002c73020000000000a80037003f
:10a21c0080a1210010407800ef40600080a1210057
:10a22c000148780080a1210010407800ea4f5000ce
:10a23c000300360080a12100a1c0b30001487800c2
:10a24c0080a12100104078000080fb0080004000bd
:10a25c0040ad28000080400010007800b0d088008d
:10a26c00488f02000000000040a12100100078007f
:10a27c004200de00614060000042780040a12100f5
:10a28c0010007800634060008041780040a12100fc
:10a29c00100078004300de0061406000004178004f
:10a2ac00809c21001080fb004400de0061406000b7
:10a2bc0080407800b0d08000a88e02000000000022
:10a2cc003a8f02000000000010c0b3002c73020093
:10a2dc00000000007600370041a1210011407800f9
:10a2ec000000a1000010a1008048780041a12100cd
:10a2fc00114078000020a1008048780041a1210085
:10a30c00114078000030a10080487800819c210029
:10a31c00114078000040a1008048780080a1210005
:10a32c00104078000080fb00680060000000e00036
:10a33c000c00320040a12100100078006340600046
:10a34c000014a000e340600040a12100e3c06000c5
:10a35c0090417800c2cfb30002c16100814071000e
:10a36c000148780080a12100104078000080fb009b
:10a37c00640060000000e0000c00320040a12100ed
:10a38c0010007800634060000004a000e34060000f
:10a39c0040a12100e3c0600090417800c2cfb3001f
:10a3ac0002c16100814071000148780080a1210048
:10a3bc00104078000080fb00620060000000e000ac
:10a3cc000400320041a12100114078000020a000bf
:10a3dc008048780080a12100104078000080fb00ac
:10a3ec0061006000004078000004e00004003200ce
:10a3fc0041a12100114078000030a0008048780075
:10a40c0080a12100104078000080fb0070006000eb
:10a41c000000e00004003a00819c2100114078000b
:10a42c000040a00080487800488f02000000000027
:10a43c0040a12100100078004200de006140600065
:10a44c000042780040a121001000780063406000b9
:10a45c008041780040a12100100078004300de000c
:10a46c006140600000417800809c21001080fb005e
:10a47c004400de006140600080407800b0d0800075
:10a48c00a88e0200000000003a8f020000000000bd
:10a49c0010c0b3002c730200000000000400370051
:10a4ac000040eb002c7302000000000000000000d4
:10a4bc0065fe37000000fa0000b92800f26d0200ba
:10a4cc00000000000080fa00000006000000fa0006
:10a4dc00881f7800819c2100114078000040a0006a
:10a4ec0080487800819c2100114078000030a10048
:10a4fc0080487800609b210011c0b30001487800af
:10a50c00709b210081c0b30001487800209e21007f
:10a51c0021c0b3000148780080c0eb0020c0b3001c
:10a52c008e7d020000000000c922a900c902a9000a
:10a53c00c8e2a80010c0b300408002000000000078
:10a54c00dcff07000673020000000000319e2100b2
:10a55c0080487800309e2100104078000080fb007d
:10a56c004400de0080407800409e210001487800c5
:10a57c00409e2100104078000080fb00e30f50004b
:10a58c0003013200e30f500007003c00e10f5000c4
:10a59c0099003200e10f5000eb003c000000e0009d
:10a5ac000d0032007b033700e60f50002e03320003
:10a5bc00e60f500003003c00e40f50002203320071
:10a5cc0074033700e80f50003d033200ea0f5000cf
:10a5dc00240132006f033700309e210010407800b8
:10a5ec000080fb00cf80de00d200200003002000a2
:10a5fc00820f5000838f58007a003e0000600100eb
:10a60c00690337000c0037000d00370012003700cb
:10a61c00170037001d0037002300370044003700b7
:10a62c00480037004c003700520037005800370004
:10a63c005e003700640037009eff07006d00370096
:10a64c00147e02000000000010c0b3002c73020046
:10a65c000000000067003700607e02000000000070
:10a66c0010c0b3002c730200000000006100370022
:10a67c000040eb00408002000000000010c0b3005e
:10a68c002c730200000000005a00370010c0b30009
:10a69c00408002000000000010c0b3002c730200c8
:10a6ac000000000053003700209e2100104078006d
:10a6bc00e24f500006003a00527f020000000000fa
:10a6cc0080407800509e2100014878000600370039
:10a6dc00f00f2000867e0200000000008040780011
:10a6ec00509e210001487800809c21001040780089
:10a6fc00684060000004e00008003200509e210019
:10a70c00104078000080fb00ea8b02000000000083
:10a71c0080407800509e210001487800509e210016
:10a72c00104078002c73020000000000310037004c
:10a73c00a27f0200000000002c7302000000000049
:10a74c002c00370054800200000000002c73020023
:10a75c00000000002700370010c0b300ee7f02009d
:10a76c000000000010c0b3002c73020000000000b9
:10a77c00200037000040eb002c800200000000009d
:10a78c0010c0b3002c730200000000001900370049
:10a79c0010c0b3002c8002000000000010c0b300f9
:10a7ac002c73020000000000120037000040eb0088
:10a7bc001a8002000000000010c0b3002c730200cd
:10a7cc00000000000b00370010c0b3001a8002001c
:10a7dc000000000010c0b3002c7302000000000049
:10a7ec00040037000040eb002c7302000000000056
:10a7fc0000000000eb023700309e21001040780072
:10a80c00ef406000309e210001487800309e21000e
:10a81c00104078008040e800309e2100014878000c
:10a82c0010c0b3002c73020000000000509e2100e9
:10a83c008040eb00014878003c00370006730200b2
:10a84c0000000000619e210080487800809c21005f
:10a85c0010407800684060000004e00008003200fe
:10a86c00609e2100104078000080fb00ea8b020003
:10a87c000000000080407800609e210001487800b4
:10a88c00209e210010407800e24f500009003a0051
:10a89c00609e2100104078000080fb00fc7e0200ce
:10a8ac000000000010c0b3002c7302000000000078
:10a8bc0019003700609e2100104078000080fb00da
:10a8cc00867e02000000000080407800609e21001f
:10a8dc0001487800809c210010407800684060009e
:10a8ec000004e00008003200609e21001040780057
:10a8fc000080fb00ea8b0200000000008040780022
:10a90c00609e210001487800609e21001040780074
:10a91c002c73020000000000509e210010407800b3
:10a92c008040e800509e210001487800509e210094
:10a93c0090407800309e21001040780080cf50006d
:10a94c00beff390097023700309e2100104078007e
:10a95c00ef406000309e210001487800309e2100bd
:10a96c00104078008040e800309e210001487800bb
:10a97c00309e210010407800ee7f020000000000a5
:10a98c0010c0b3002c7302000000000085023700d9
:10a99c00309e210010407800ef406000309e210076
:10a9ac0001487800309e2100104078008040e8007b
:10a9bc00309e21000148780010c0b3002c730200b7
:10a9cc00000000000673020000000000419e210000
:10a9dc0080487800509e21008040eb0001487800b0
:10a9ec0016003700409e2100104078000004e00063
:10a9fc0004003d0010c0b300c87f0200000000003e
:10aa0c00030037000040eb00c87f0200000000008c
:10aa1c00409e2100104078000040400080407800ab
:10aa2c00409e210001487800509e21001040780083
:10aa3c008040e800509e210001487800509e210083
:10aa4c0090407800309e21001040780080cf50005c
:10aa5c00e4ff390010c0b3002c73020000000000aa
:10aa6c0050023700309e2100104078000080fb001f
:10aa7c00410a2000810f500016003200410a2000cc
:10aa8c00810f500004003c00010a2000810f50008f
:10aa9c0008003200e7013700510a2000810f5000f6
:10aaac00b4003200710a2000810f50001c013200ea
:10aabc00e0013700067302000000000081a32100b2
:10aacc008048780010c0b3002c7302000000000016
:10aadc00dc01370080a32100104078000080fb00cf
:10aaec00e10f500003003200e20f5000360032003c
:10aafc009b00370006730200000000000080fb0082
:10ab0c0040cf880040cf80006300b900000078007f
:10ab1c0040cf88000000eb0050cf880009003700c0
:10ab2c0081cf800050cf800000844000067302006b
:10ab3c0000000000004c780050cf80000000e800be
:10ab4c0050cf880051cf800040cf8000808f5000c4
:10ab5c00f3ff39000000eb0050cf880012003700e3
:10ab6c0081cf800050cf80000080e8000080400042
:10ab7c001041780081cf800050cf80000000e800a9
:10ab8c00008040009040780083cf800050cf800040
:10ab9c0000804100104078006c02070050cf80000c
:10abac006300400050cf880051cf800040cf800020
:10abbc00808f5000eaff390010c0b3002c730200e4
:10abcc00000000006a00370006730200000000005d
:10abdc000080fb0040cf880040cf80004200dd00a9
:10abec0040cf88000000eb0050cf880009003700f0
:10abfc0081cf800050cf800000844000067302009b
:10ac0c0000000000004c780050cf80000000e800ed
:10ac1c0050cf880051cf800040cf8000808f5000f3
:10ac2c00f3ff39000000eb0050cf880044003700e0
:10ac3c000040eb00c87f0200000000000040eb0069
:10ac4c00c87f0200000000000040eb00c87f02003b
:10ac5c00000000000040eb00c87f02000000000074
:10ac6c0081cf800050cf80000080400010407800e1
:10ac7c000080fb00fc7e02000000000081cf800001
:10ac8c0050cf80000000e8000080400010407800a9
:10ac9c000080fb00fc7e02000000000081cf8000e1
:10acac0050cf80000080e800008040001040780009
:10acbc000080fb00fc7e02000000000081cf8000c1
:10accc0050cf8000630040000080400082cf8000a5
:10acdc0051cf8000e380400081004100914078001a
:10acec00efc0600001487800509e21008040eb00ce
:10acfc0001487800060037004f020700509e2100e3
:10ad0c00104078008040e800509e210001487800f7
:10ad1c0081cf800050cf8000630040000080400055
:10ad2c0090407800509e21001040780080cf500059
:10ad3c00f1ff3e0050cf80006400400050cf8800ef
:10ad4c0051cf800040cf8000808f5000b8ff390079
:10ad5c0010c0b3002c730200000000000400370088
:10ad6c000040eb002c73020000000000000000000b
:10ad7c003401370080a32100104078000080fb00d4
:10ad8c00e10f500003003200e20f5000410032008e
:10ad9c006200370006730200000000000080fb0018
:10adac0040cf88000673020000000000419e210085
:10adbc00804878000000eb0050cf8800300037004e
:10adcc00409e210090407800609e21000148780050
:10addc00509e21008040eb00014878001a0037009b
:10adec00609e2100104078000080fb006100600034
:10adfc00004078000004e0000400320010c0b300f2
:10ae0c00c87f020000000000030037000040eb0088
:10ae1c00c87f020000000000609e210010407800f6
:10ae2c000080fb000000d10080407800609e210073
:10ae3c0001487800509e2100104078008040e800c6
:10ae4c00509e210001487800509e2100104078004f
:10ae5c00e34f5000e2ff3600527f0200000000007a
:10ae6c00527f020000000000004078002c730200aa
:10ae7c000000000050cf80000000e80050cf880098
:10ae8c0051cf800040cf8000808f5000ccff390024
:10ae9c002200370006730200000000000080fb0057
:10aeac0040cf88000000eb0050cf88001600370020
:10aebc0022c0b30060b92000a10b200025020700be
:10aecc005a02070022c0b30060bb2d00a10b20006a
:10aedc002002070022c0b300603d2d00a10b200012
:10aeec001c0207005102070022c0b30060bb200007
:10aefc00a10b2000170207004c02070050cf800066
:10af0c000000e80050cf880051cf800040cf800077
:10af1c00808f5000e6ff390000000000c9003700a8
:10af2c0006730200000000000080fb0060cf880068
:10af3c0006730200000000000080fb0070cf880048
:10af4c0080a3210010407800e24f500007003a0027
:10af5c0060cf80006500b9008000780070cf800061
:10af6c000080400040cf88001c00370080a32100e7
:10af7c0010407800e14f500008003a0060cf80008c
:10af8c00000040008000780070cf800000804000fe
:10af9c000000400040cf88001000370080a3210043
:10afac0010407800e34f500008003a0060cf80005a
:10afbc00000040008000780070cf800000804000ce
:10afcc000000400040cf8800040037000040eb0038
:10afdc002c730200000000009a0037000000eb0008
:10afec0050cf88000900370081cf800050cf8000ff
:10affc00008440000673020000000000004c780042
:10b00c0050cf80000000e80050cf880051cf800066
:10b01c0040cf8000808f5000f3ff390070cf80004c
:10b02c000000e0000300320010c0b3002c730200db
:10b03c00000000000000eb0050cf880072003700c9
:10b04c0081cf800050cf80000080400010407800fd
:10b05c00e14f500042003a0080a3210010407800dc
:10b06c00e34f500014003a0081cf800050cf800095
:10b07c0063004000008040001041780081cf8000c8
:10b08c0050cf80000080e8000080400090407800a5
:10b09c0083cf800050cf80000000e800008041008a
:10b0ac0010407800e000070050cf800064004000a2
:10b0bc0050cf88005400370080a321001040780046
:10b0cc00e14f500014003a0081cf800050cf800037
:10b0dc0063004000008040001041780081cf800068
:10b0ec0050cf80000080e800008040009040780045
:10b0fc0083cf800050cf80000000e800008041002a
:10b10c00104078001101070050cf8000640040000f
:10b11c0050cf88003c00370080a3210010407800fd
:10b12c00e24f500038003a0081cf800050cf8000b1
:10b13c0064004000008040009040780082cf800086
:10b14c0050cf80000000e8000000410052010700d1
:10b15c0050cf80006500400050cf88002a00370097
:10b16c0081cf800050cf80000080400010407800dc
:10b17c00e24f500024003a0080a3210010407800d8
:10b18c00e34f50000a003a0081cf800050cf80007e
:10b19c000000e800008040001040780085000700a7
:10b1ac0050cf80000080e80050cf88001600370098
:10b1bc0080a3210010407800e14f50000a003a00b3
:10b1cc0081cf800050cf80000000e800008040005c
:10b1dc0010407800ba00070050cf80000080e800d3
:10b1ec0050cf88000800370080a321001040780061
:10b1fc00e24f500004003a008c01070050cf800051
:10b20c000000e80050cf880051cf800040cf800074
:10b21c00808f50008aff390070cf80000000e00062
:10b22c0003003a0010c0b3002c73020000000000b1
:10b23c00040037000040eb002c73020000000000fb
:10b24c000000000057003700309e210010407800ad
:10b25c005a9102000000000010c0b3002c730200d1
:10b26c00000000004f003700309e21001040780095
:10b27c00e3406000309e210001487800309e2100a0
:10b28c0090407800609b210001487800609b210071
:10b29c0090407800209e2100104078008e7d0200a6
:10b2ac000000000010c0b30040800200000000004d
:10b2bc0010c0b3002c7302000000000039003700ee
:10b2cc00819c2100114078000040a100804878004a
:10b2dc00309e2100104078000080fb006800600068
:10b2ec000000e00004003a00819c2100114078002d
:10b2fc000040a00080487800209e210021c0b300af
:10b30c0001487800309e2100104078000080fb003e
:10b31c00640060000000e00003003200209e210069
:10b32c0031c0b30001487800819c210011407800a5
:10b33c000030a10080487800309e21001040780039
:10b34c000080fb00620060000000e000040032009e
:10b35c00819c2100114078000030a00080487800ca
:10b36c00609b210090407800209e210010407800c6
:10b37c008e7d02000000000010c0b300408002006f
:10b38c000000000010c0b3002c730200000000008d
:10b39c00040037000040eb002c730200000000009a
:10b3ac000000000067fc37004f0478000080fa00b2
:10b3bc00000006000400fa00204798000040eb0053
:10b3cc00004f7800090037002e409000614060006b
:10b3dc00c87f0200000000002e4090000080fb009f
:10b3ec000000d100204798001e4fe8001e40780056
:10b3fc00e54f5000f4ff3600527f020000000000c1
:10b40c00004078002c73020000000000527f020004
:10b41c0000000000004078002c73020000000000c7
:10b42c000080fa00000006000600fa002047980091
:10b43c003147980042479800ae40900000c8b300d6
:10b44c0000c06000104798000040eb00004f7800ef
:10b45c00090037002e40900061406000c87f020058
:10b46c00000000002e4090000080fb000000d10086
:10b47c00204798001e4fe8001e407800e54f500012
:10b48c00f4ff36001e4090000004e00009003a0072
:10b49c003e4090000080fb00fc7e0200000000009b
:10b4ac004e4090000080fb00fc7e0200000000007b
:10b4bc0001003700000000000080fa0000000600c8
:10b4cc000400fa00204798000040eb00004f780081
:10b4dc00120037002e4090000080fb0061006000dd
:10b4ec00004078000004e0000400320010c0b300fb
:10b4fc00c87f020000000000030037000040eb0092
:10b50c00c87f0200000000002e4090000080fb006d
:10b51c000000d100204798001e4fe8001e40780024
:10b52c00e34f5000ebff3600527f0200000000009a
:10b53c00527f020000000000004078002c730200d3
:10b54c00000000000080fa00000006000600fa006f
:10b55c002047980031479800424798002e409000b1
:10b56c000080fb004600de00104798000040eb0016
:10b57c00004f7800230037001e407800e34f500046
:10b58c000e003a001e4090000004e0000b00320058
:10b59c0010c0b3002c800200000000001e40900080
:10b5ac000080fb008a8b0200000000000040eb00d2
:10b5bc002c80020000000000110037002e4090008b
:10b5cc000080fb0061006000004078000004e00097
:10b5dc000400320010c0b300c87f0200000000005d
:10b5ec00030037000040eb00c87f020000000000a1
:10b5fc002e4090000080fb000000d10020479800f6
:10b60c001e4fe8001e407800e34f5000daff360072
:10b61c003e4090000080fb00fc7e02000000000019
:10b62c004e4090000080fb00fc7e020000000000f9
:10b63c000080fa00000006000000fa000040eb0059
:10b64c00c87f0200000000000040eb00c87f020031
:10b65c00000000000040eb00c87f0200000000006a
:10b66c000040eb00c87f0200000000000000eb006f
:10b67c00fc7e0200000000000000eb00fc7e0200db
:10b68c00000000000000eb00fc7e02000000000047
:10b69c000080fa00000006000400fa00000f780099
:10b6ac00214798000040eb00c87f0200000000001a
:10b6bc000040eb00c87f0200000000000040eb00df
:10b6cc00c87f0200000000000040eb00c87f0200b1
:10b6dc00000000001e007800104078000080fb0085
:10b6ec00fc7e0200000000001e00e8001040780004
:10b6fc000080fb00fc7e0200000000001e80e800c1
:10b70c00104078000080fb00fc7e0200000000006e
:10b71c002e4090006f4060002047980001003700d9
:10b72c00c5ff07002e4090000080fb000000ea00df
:10b73c004f00de0000407800ae4090008140e900f0
:10b74c00214798000004e000f5ff3a000080fa0061
:10b75c00000006000800fa00100798002107980066
:10b76c00624798000040eb00c87f02000000000018
:10b77c000040eb00c87f0200000000000040eb001e
:10b78c00c87f0200000000000040eb00c87f0200f0
:10b79c00000000001e009000ea8b02000000000078
:10b7ac00fc7e0200000000001e009000ae00900025
:10b7bc004809dd004800de0000007100c808de000a
:10b7cc0000007800ea8b020000000000fc7e020002
:10b7dc00000000001e009000ae0090004008de004b
:10b7ec0000007800ea8b020000000000fc7e0200e2
:10b7fc00000000006e4090006f40600060479800b1
:10b80c000040eb00004f7800020037008aff070071
:10b81c001e4fe8006e4090009e40780080cf500094
:10b82c00faff39000080fa00000006000200fa005e
:10b83c0010c0b300c87f0200000000000040eb0005
:10b84c00c87f0200000000000040eb00c87f02002f
:10b85c00000000000040eb00c87f02000000000068
:10b86c000000eb00fc7e020000000000527f020092
:10b87c0000000000004f7800527f02000000000022
:10b88c00004078002c730200000000001e4078007d
:10b89c002c7302000000000067ff070066ff070022
:10b8ac000080fa00000006000200fa00000f780089
:10b8bc001e007800e30f500004003e0010a1a80009
:10b8cc001081a800e0032000120037001e00780051
:10b8dc00fe0f500004003e0010a1a8001081a9002a
:10b8ec00a00f20000b003700400f20009e007800b6
:10b8fc00808f500004003e0010a1a9001081a80008
:10b90c00007d20000300370010a1a9001081a900c0
:10b91c0000e823000080fa00000006000600fa0090
:10b92c001021ef001e21ef009c21ef0090cc800035
:10b93c000000e00007003a005136800000fe2f00a6
:10b94c0000806000503688000000eb0080cc88003e
:10b95c002400370090cc8000d3ff0700000f780044
:10b96c0090cc80009e007800000178001100090046
:10b97c008280d8000000e900100798009e0090001b
:10b98c0061088800a0cc8000800078001e00900028
:10b99c000088b90080007800400620000001780083
:10b9ac00110009008280d8002007980051368000d1
:10b9bc0000fe2f00008060006001b300503688004c
:10b9cc00ae009000d10c88002e019000c20c8800b3
:10b9dc0060002000e00c880011e1a800200020008d
:10b9ec0080cc88000080fa00000006000e00fa00ef
:10b9fc00881f78001021ef001e21ef009c21ef0022
:10ba0c0080cc8000e20f500012003a0051368000ca
:10ba1c0000fe2f000080600050368800c10020001e
:10ba2c00e02b2000be8c0200000000000000eb00a8
:10ba3c0080cc880010c480008000e800f007200053
:10ba4c000080600001802100614078000004e0006b
:10ba5c00920032000000eb001007980010c4800028
:10ba6c008000e800f00720000080600010c488000f
:10ba7c007423020000000000721f0200000000008e
:10ba8c00000f78007423020000000000721f0200f7
:10ba9c0000000000cf80de00100502000000000056
:10baac0020079800310798001e0078000000e00085
:10babc0007003200f0f920009e007800808f5000c3
:10bacc0003003e001e0090000000e80010079800e4
:10badc0018c0b3006011b8002e009000be0090009a
:10baec0094040200000000000000e00001003c0093
:10bafc000044eb000804e0000f00320018c0b30053
:10bb0c0002002000832c24002e009000be00900028
:10bb1c0090040200000000000000e000010035006d
:10bb2c000044eb000804e000030032001e0090000b
:10bb3c000000e800100798001e009000e20f500073
:10bb4c0012003200408821008040eb000148780050
:10bb5c0011012000a02c2000be8c0200000000006f
:10bb6c0011012000b02d2000328c020000000000da
:10bb7c008001eb0002fa20001100200020032000bd
:10bb8c00fe25020000000000000f78001e00780067
:10bb9c0045ff070040079800ce0090001e0078007b
:10bbac0000017800110009008280d8000000e90033
:10bbbc00500798001e009000e20f50000f0032005a
:10bbcc0001012000902f2000328c020000000000a8
:10bbdc008001eb00320620008000eb0020032000e7
:10bbec00fe25020000000000cf80de0010050200e0
:10bbfc000000000020079800310798000200200088
:10bc0c00832c24002e009000be0090000c04020037
:10bc1c000000000020079800310798005e0090009b
:10bc2c008000eb0074050200000000002e01900063
:10bc3c00be0190001e06020000000000da040200a3
:10bc4c0000000000600798005136800000fe2f00b5
:10bc5c00008060006001b30050368800ee00900058
:10bc6c00d10c88006e019000c20c8800600020008e
:10bc7c00e00c8800de0090006108880011e1a8004b
:10bc8c00a100200090302000be8c020000000000bb
:10bc9c002000200080cc880001003700000000004c
:10bcac004f0478000080fa00000006001000fa0033
:10bcbc0080cc8000e20f500005003a00f10120001a
:10bccc0030312000be8c020000000000e40137007f
:10bcdc00f100200020332000328c02000000000014
:10bcec001e21ef001021ef00c942a8003134800062
:10bcfc0000fe2f0000806000a000b30030348800ec
:10bd0c00a003200080088800fd0107006011b80026
:10bd1c00009fbe000297be00f0ff23000100200030
:10bd2c006011b8003e02be002e03be000020e100f0
:10bd3c0001a8e10002b0e10003b8e1000f003600f9
:10bd4c003e00be002e01be00c819dd004812de0008
:10bd5c00830172004811dd00480ade000201720006
:10bd6c00c808dd004802de00810072004800dd00da
:10bd7c00009fbe000297be000a003700b1002000f1
:10bd8c00a0132100328c020000000000a000200053
:10bd9c0080088800da0107006011b800009fbe001f
:10bdac000297be00f0f92000010020006011b800dd
:10bdbc003e02be002e03be000020e10001a8e100ff
:10bdcc0002b0e10003b8e100070036001e00be001f
:10bddc00066f020000000000e0ae2800166e0200a4
:10bdec0000000000990137003e00be002e01be008d
:10bdfc00e00f5000e08f5800e00f5900e08f590021
:10be0c008f013200b1002000a0132100328c0200ff
:10be1c00000000001e007800e70107006011b80068
:10be2c004007980051079800620798007307980024
:10be3c004e029000de0290006e039000fe03900014
:10be4c0000a82100610020006011b8000020e10072
:10be5c0001a8e10002b0e10003b8e1005d0036008a
:10be6c004e009000de0090006e019000fe019000ec
:10be7c0016050200000000000001be00703b24000b
:10be8c00a13b25000c0402000000000098040200f5
:10be9c0000000000009fbe000297be003e00be00e6
:10beac002e01be00046a2800150020006033b80083
:10bebc00de070200000000000000be00066f02005a
:10becc0000000000e0c2b3002c7302000000000070
:10bedc003e00be002e01be00046a280015002000a2
:10beec006033b800ec07020000000000009fbe00a9
:10befc000297be00f0702200010020006011b80013
:10bf0c003e02be002e03be000020e10001a8e100ad
:10bf1c0002b0e10003b8e10003003e0000c3b3002f
:10bf2c002c73020000000000703e20000100200075
:10bf3c006011b8003e02be002e03be000020e100de
:10bf4c0001a8e10002b0e10003b8e10003003e00eb
:10bf5c0000c3b3002c730200000000003006200068
:10bf6c00010020006011b8003e02be002e03be008e
:10bf7c000020e10001a8e10002b0e10003b8e100fb
:10bf8c0003003e0000c3b3002c730200000000004d
:10bf9c003e02be002e03be009000200001002000d7
:10bfac006011b8000020e10001a8e10002b0e1003e
:10bfbc0003b8e10003003e0000c3b3002c73020081
:10bfcc00000000001e00be007c6e0200000000009d
:10bfdc00170137004e029000de0290006e039000b5
:10bfec00fe039000b0e12e00110020006011b8009b
:10bffc000020e10001a8e10002b0e10003b8e1007b
:10c00c00500036004e009000de0090006e01900053
:10c01c00fe01900016050200000000000001be00a9
:10c02c00902f2000512125000c040200000000007c
:10c03c009804020000000000009fbe000297be00a2
:10c04c003e00be002e01be0004712200050020003f
:10c05c006033b800de070200000000000000be00e4
:10c06c00066f020000000000e0c2b3002c73020057
:10c07c00000000003e00be002e01be000471220034
:10c08c00050020006033b800ec070200000000003f
:10c09c00009fbe000297be00703e200001002000f1
:10c0ac006011b8003e02be002e03be000020e1006d
:10c0bc0001a8e10002b0e10003b8e10003003e007a
:10c0cc0000c3b3002c7302000000000030062000f7
:10c0dc00010020006011b8003e02be002e03be001d
:10c0ec000020e10001a8e10002b0e10003b8e1008a
:10c0fc0003003e0000c3b3002c73020000000000dc
:10c10c003e02be002e03be00900020000100200065
:10c11c006011b8000020e10001a8e10002b0e100cc
:10c12c0003b8e10003003e0000c3b3002c7302000f
:10c13c00000000001e0078001c70020000000000cf
:10c14c00bb0037004e029000de0290006e039000a0
:10c15c00fe03900000c42900010020006011b8000b
:10c16c000020e10001a8e10002b0e10003b8e10009
:10c17c00430036004e009000de0090006e019000ef
:10c18c00fe01900016050200000000000001be0038
:10c19c0080b22600e10625000c040200000000001d
:10c1ac009804020000000000009fbe000297be0031
:10c1bc003e00be002e01be00843e20000500200083
:10c1cc006033b800de070200000000000000be0073
:10c1dc00066f020000000000e0c2b3002c730200e6
:10c1ec00000000003e00be002e01be00843e200078
:10c1fc00050020006033b800ec07020000000000ce
:10c20c00009fbe000297be003006200001002000f7
:10c21c006011b8003e02be002e03be000020e100fb
:10c22c0001a8e10002b0e10003b8e10003003e0008
:10c23c0000c3b3002c730200000000003e02be00dd
:10c24c002e03be0090002000010020006011b800f9
:10c25c000020e10001a8e10002b0e10003b8e10018
:10c26c0003003e0000c3b3002c730200000000006a
:10c27c001e0078001c700200000000006c003700eb
:10c28c004e029000de0290006e039000fe039000c0
:10c29c0090162300010020006011b8000020e1007e
:10c2ac0001a8e10002b0e10003b8e100370036005c
:10c2bc004e009000de0090006e019000fe01900098
:10c2cc0016050200000000000001be0000c22b0099
:10c2dc00e1eb24000c0402000000000098040200b2
:10c2ec0000000000009fbe000297be003e00be0092
:10c2fc002e01be0044062000050020006033b8006b
:10c30c00de070200000000000000be00066f020005
:10c31c0000000000e0c2b3002c730200000000001b
:10c32c003e00be002e01be00440620000500200089
:10c33c006033b800ec07020000000000009fbe0054
:10c34c000297be003e02be002e03be0090002000ed
:10c35c00010020006011b8000020e10001a8e100fc
:10c36c0002b0e10003b8e10003003e0000c3b300db
:10c37c002c730200000000001e00780000407800c2
:10c38c008470020000000000290037004e0090006d
:10c39c00de0090006e019000fe0190001605020078
:10c3ac00000000000001be000068290081d12400bb
:10c3bc000c040200000000009804020000000000c1
:10c3cc00009fbe000297be003e00be002e01be00c4
:10c3dc00a4002000050020006033b800de07020036
:10c3ec00000000000000be00066f0200000000000c
:10c3fc00e0c2b3002c730200000000003e00be003f
:10c40c002e01be00a4002000050020006033b800ff
:10c41c00ec07020000000000009fbe000297be0067
:10c42c001e007800004078008470020000000000bc
:10c43c00e0ae2800166e020000000000030037007a
:10c44c0020af2800166e020000000000303480007f
:10c45c00f001b300303488001e21ef001021ef00f2
:10c46c000080fa00000006000400fa001e21ef0014
:10c47c001021ef00c942a8003134800000fe2f00cb
:10c48c0000806000a000b30030348800a0032000be
:10c49c00800888001a000700008fbe00f00f2000f3
:10c4ac00010020001e01be00800f5100818f590039
:10c4bc00070036001e01be004818dd00c810de0063
:10c4cc00810070004810dd00008fbe0004003700b2
:10c4dc00a00020008008880009000700008fbe0023
:10c4ec0030348000f001b300303488001e21ef009e
:10c4fc001021ef001e00be000080fa0000000600b4
:10c50c000000fa000080eb00700888000080eb004f
:10c51c00600888000821ef000621ef001621ef00cb
:10c52c001421ef0080002000f0088800400f20004c
:10c53c00e008880000402200d00888008780a9000d
:10c54c001fe1a80011e1a8000000000031048000e8
:10c55c0000002100008060000000e000fbff3200c2
:10c56c0011e1a9001fe1a9003008800080cd8800ee
:10c57c00400880008000eb0090cd8800a1cd8800a1
:10c58c0090cd8000a1cd8000c001dd000200200014
:10c59c0080cd80008000eb000200400083804800ca
:10c5ac0090cd8800a1cd880090cd8000a1cd8000d9
:10c5bc000080fa00000006000200fa00000f78006c
:10c5cc0084a0a9008420a90071348000f00f2e00f3
:10c5dc008080600000a02000010070007034880092
:10c5ec007134800000fe2f0000806000a000b300ba
:10c5fc00703488000821ef000621ef008000200035
:10c60c008008880011e1a80030002000300a880062
:10c61c0030082000100a880004003700000a80004f
:10c62c008000eb00b0cc8800c1cc8800100a8000e0
:10c63c00680060000000e000f8ff3a0004003700da
:10c64c00200a80008000eb00d0cc8800e1cc880070
:10c65c00300a8000680060000000e000f8ff3a003b
:10c66c0000000000100a8000680060000000e0007c
:10c67c00fcff3200000a80008000eb00d0cc880068
:10c68c00e1cc8800200a80008000eb00f0cc880010
:10c69c0001cd88006000b80010cd880021cd880045
:10c6ac000000eb0030cd88003200370000000000a5
:10c6bc00100a8000680060000000e000fcff3200ff
:10c6cc00000a80008000eb00b0cc8800c1cc880050
:10c6dc00200a80008000eb0040cd880051cd8800fe
:10c6ec0042cd800053cd8000f0cc800001cd800085
:10c6fc000000510081805900c001dd0002002000c3
:10c70c00b4cc8000c5cc8000d0cc8000e1cc8000c3
:10c71c000000520081805a000200400083804800d3
:10c72c0060cd880071cd880012cd800023cd8000b3
:10c73c0060cd800071cd80000200400083804800f5
:10c74c0010cd880021cd880040cd800051cd8000d7
:10c75c00f0cc880001cd8800b0cc8000c1cc80002a
:10c76c00d0cc8800e1cc880030cd80000000e800ff
:10c77c0030cd880030cd80009e0f5000cbff3900ab
:10c78c004221ef004221ef0011e1a90014cd8000fd
:10c79c0025cd80001e0078008000eb000001be005b
:10c7ac000400be0086060200000000000080fa00b3
:10c7bc00000006000000fa00809c21001040780068
:10c7cc00634060000004e00002003a00c942a80087
:10c7dc0001003700c8c2a800e1002000103420007e
:10c7ec00328c0200000000000080fa0000000600fd
:10c7fc000000fa00809c210010407800634060002b
:10c80c000004e00003003a00c942a900cb42a80092
:10c81c0002003700c8c2a900cac2a80081002000cb
:10c82c00f0342000be8c0200000000000080fa00f2
:10c83c00000006000000fa00809c210010407800e7
:10c84c00634060000004e00003003a00c942a90004
:10c85c00cb42a90002003700c8c2a900cac2a90075
:10c86c007100200070352000be8c0200000000001a
:10c87c000080fa00000006000200fa00809c2100f3
:10c88c0010407800634060000004e00008003a00ab
:10c89c00c942a800000000000000000050168000f3
:10c8ac004a00de0061406000004f7800070037004e
:10c8bc00c8c2a80000000000000000005016800054
:10c8cc004600de0061406000004f78001e80fb00d7
:10c8dc000080fa00000006000a00fa00881f7800a9
:10c8ec000040eb00004f78001021ef001e21ef00fc
:10c8fc009c21ef0080cc8000e20f500013003a0026
:10c90c0010c480008000e800f00720000080600068
:10c91c0001802100614078000004e0000b003a0027
:10c92c005136800000fe2f000080600050368800d9
:10c93c00c1002000e02b2000be8c02000000000093
:10c94c000000eb0080cc88008000370010c4800011
:10c95c008000e800f00720000080600010c4880010
:10c96c007423020000000000721f0200000000008f
:10c97c00cf80de00100502000000000010079800b8
:10c98c002107980040882100104078000004e00046
:10c99c000c003a0018c0b3000200200043332400fe
:10c9ac001e009000ae0090009404020000000000f5
:10c9bc000000e00001003c000044eb000804e00033
:10c9cc0016003200408821008040eb0001487800be
:10c9dc0031012000301e2100be8c0200000000003e
:10c9ec008001eb00420b20008000eb00a005200032
:10c9fc00fe25020000000000cf80de0010050200c2
:10ca0c0000000000100798002107980010c0b30028
:10ca1c00004f7800010037000000000010a1a800b2
:10ca2c001081a800204e20003007980002002c0036
:10ca3c00a35524001e009000ae0090000c040200d0
:10ca4c000000000010079800210798003e0090009d
:10ca5c008000eb0074050200000000001e01900035
:10ca6c00ae0190001e060200000000000200200033
:10ca7c00832724005203020000000000da040200a5
:10ca8c0000000000400798005136800000fe2f0087
:10ca9c00008060006001b30050368800ce0090002a
:10caac00d10c8800ce009000c10c880060002000e2
:10cabc00e00c8800be0090006108880011e1a8001d
:10cacc00c1002000601f2100be8c0200000000008d
:10cadc002000200080cc88001e407800e14f5000e0
:10caec001a003a0013002000420b20008000eb00db
:10cafc000080eb00fe25020000000000cf80de006d
:10cb0c001005020000000000100798002107980093
:10cb1c0018c0b3006011b8001e009000ae00900069
:10cb2c0090040200000000000000e000010035004d
:10cb3c000044eb000804e000b7ff320070b128009d
:10cb4c00166e020000000000000000004f04780088
:10cb5c000080fa00000006000200fa000040eb0022
:10cb6c00004f780000a32100104078006240600064
:10cb7c000004e0001600320000a3210010407800f1
:10cb8c00614060000004e00003003a000040eb004c
:10cb9c00c87f02000000000000c2b3002c7302002a
:10cbac00000000003100200030412000328c0200d7
:10cbbc000000000000c2b3002c7302000000000053
:10cbcc0001a32100114078000010a10080487800da
:10cbdc0000a3210010407800614060000004e000d8
:10cbec0003003a00527f020000000000004f780062
:10cbfc0001a32100114078000010a00080487800ab
:10cc0c001e80fb000080fa00000006000200fa0003
:10cc1c00000f780000a321001040780062406000f3
:10cc2c000004e0001600320000c2b3002c730200b6
:10cc3c00000000003100200030412000328c020046
:10cc4c000000000000c2b3002c73020000000000c2
:10cc5c0000a3210010407800614060000004e00057
:10cc6c0003003a000040eb00c87f02000000000007
:10cc7c0001a32100114078000010a1008048780029
:10cc8c0000a3210010407800614060000004e00027
:10cc9c0007003a001e007800fc7e02000000000035
:10ccac00a27f0200000000000080fb00000f780053
:10ccbc0000c2b3002c730200000000001e007800bc
:10cccc000000e00006003a00310020003041200056
:10ccdc00328c0200000000000030200005003700fc
:10ccec004100200060412000328c02000000000056
:10ccfc00001020000080fa00000006000000fa007e
:10cd0c0000a3210010407800624060000004e000a5
:10cd1c00130032004100200060412000328c0200e0
:10cd2c000000000040b72800166e02000000000052
:10cd3c0000a3210010407800614060000004e00076
:10cd4c0003003a0010c0b300c87f020000000000ce
:10cd5c0001a32100114078000010a1008048780048
:10cd6c0000a3210010407800614060000004e00046
:10cd7c000f003a00147e0200000000000000e000ea
:10cd8c000b00320091002000c0202000328c0200e9
:10cd9c00000000005101200050212000328c0200c4
:10cdac000000000040b72800166e020000000000d2
:10cdbc00d1002000a0412000be8c02000000000029
:10cdcc000080fa00000006000000fa0000a3210019
:10cddc0010407800624060000004e0001300320054
:10cdec004100200060412000328c02000000000055
:10cdfc0040b72800166e02000000000000a32100be
:10ce0c0010407800614060000004e00003003a002c
:10ce1c0010c0b300c87f02000000000001a3210075
:10ce2c00114078000010a1008048780000a3210078
:10ce3c0010407800614060000004e00002003a00fd
:10ce4c00607e020000000000c10020007042200043
:10ce5c00be8c0200000000000080fa0000000600fa
:10ce6c000000fa0001012000404f2000328c02002b
:10ce7c00000000000040eb00847002000000000085
:10ce8c0000c2b3002c73020000000000609b210064
:10ce9c0010407800847002000000000000c2b30053
:10ceac002c7302000000000050b72800166e020020
:10cebc00000000000080fa00000006000400fa00e8
:10cecc000000eb001007980001a32100114078002e
:10cedc000000a100804878007423020000000000cc
:10ceec00721f020000000000000f78001e00780086
:10cefc000000e000090034001e007800e40f500030
:10cf0c0006003c001e007800004078008040e900dc
:10cf1c00609b210001487800020037000000eb0004
:10cf2c00000f78001e0078000000e00032003a008c
:10cf3c00408821008040eb000148780001a32100cb
:10cf4c00114078000000a1008048780000a3210067
:10cf5c0010407800614060000004e0000f003a00cf
:10cf6c00b103200080452000be8c020000000000b0
:10cf7c008001eb0042002000110020001000200076
:10cf8c00fe25020000000000004078008040e9000f
:10cf9c00609b21000148780024003700d1cf80002d
:10cfac0030002300808f500004003e00510320000d
:10cfbc0030492000328c020000000000c102200029
:10cfcc00804c2000328c0200000000008001eb003d
:10cfdc00320020001100200010002000fe2502006d
:10cfec0000000000004078008040e900609b2100b8
:10cffc00014878000d003700d1cf800030002300ad
:10d00c00808f500004003e00510320003049200066
:10d01c00328c02000000000091ff070001a32100e8
:10d02c00114078000010a10080487800819c2100fc
:10d03c00114078000040a000804878000080fa0081
:10d04c00000006000000fa0000a321001040780048
:10d05c00614060000004e0000a003a00c922a80008
:10d06c00c902a800cb02a900cb22a900609b210019
:10d07c00104078008040780020c0b3008e7d020004
:10d08c00000000000080fa00000006000000fa001a
:10d09c0001a32100114078000010a1008048780005
:10d0ac0000a3210010407800614060000004e00003
:10d0bc000100320007e2a9000080fa00000006001f
:10d0cc000400fa00100798001e009000e10f5000b9
:10d0dc000a003200e10f500003003900e20f50004b
:10d0ec006d0032007d0037005103200040502000bd
:10d0fc00328c0200000000007c0037008040eb0006
:10d10c00003020005e80020000000000e1022000e0
:10d11c0090532000be8c02000000000051168000cd
:10d12c0000102000008060000000e00005003200cc
:10d13c005116800000202000008060000000e000fc
:10d14c000c003a0091002000c0202000328c02001c
:10d15c00000000005101200050212000328c020000
:10d16c000000000040b72800166e0200000000000e
:10d17c005e0037000000eb00000f78003e00370027
:10d18c0000a3210010407800614060000004e00022
:10d19c0009003a00147e0200000000001e00780016
:10d1ac00fc7e020000000000a27f020000000000d4
:10d1bc000080fb00100798001e0090000000e000ab
:10d1cc0025003a001e007800e28a020000000000f0
:10d1dc0080c2b3002c730200000000001e00780017
:10d1ec000080d100e28a0200000000009e0078005e
:10d1fc00618060000000e00004003a0070b7280075
:10d20c00f26d0200000000000d00370000a32100a9
:10d21c0010407800614060000004e00005003a0016
:10d22c00527f02000000000010c0b300c87f020053
:10d23c0000000000a0b72800f26d02000000000002
:10d24c0050b72800f26d02000000000000c2b300cd
:10d25c002c7302000000000000a321001040780095
:10d26c00614060000004e00002003a00607e0200b1
:10d27c00000000001e0fe800f00f20009e00780058
:10d28c00808f5000beff340040b72800166e02009d
:10d29c00000000001500370000a3210010407800aa
:10d2ac00614060000004e0000100320007e2a900c8
:10d2bc007100200070562000be8c0200000000009f
:10d2cc00f1002000b0182100be8c0200000000000c
:10d2dc0010c0b3000e00070004003700410220000c
:10d2ec00e01d2000be8c0200000000000080fa004f
:10d2fc00000006000000fa00b1002000600b2100c5
:10d30c00be8c0200000000000080fa000000060045
:10d31c000a00fa00004f98000040eb0020479800ec
:10d32c000040eb00304798000040eb00404798006d
:10d33c004272020000000000c922a800c902a80025
:10d34c00cb02a900cb22a90062a0a80062c0a80051
:10d35c008660a900501680004900de006140600024
:10d36c0050479800de409000014f78005016800026
:10d37c004800de006140600050479800de4090009d
:10d38c001147980030048000680060000000e00045
:10d39c0011003a00567202000000000036720200c2
:10d3ac00000000000004e0000900320006730200d7
:10d3bc00000000004047980062a0a90062c0a900cc
:10d3cc000e4890000004e00066003a006800370048
:10d3dc0000000000ebff37008660a90050168000ab
:10d3ec004900de00614060005047980050168000f4
:10d3fc004800de0061406000604798002e409000bd
:10d40c000004e000310032001e4090000004e000f7
:10d41c002e003a006e4090000004e0002b00320019
:10d42c003e409000e74f50000d003e004e409000f3
:10d43c0000404000404798005e4090000004e0002f
:10d44c00030032004e4090000004a00040479800ba
:10d45c003e4090000040e800304798003c00370008
:10d46c000e4890000004e000050032004e40900091
:10d47c000080fb0014710200000000000600370061
:10d48c00c0c5b300d0720200000000004e409000f6
:10d49c00d0720200000000005e4090000004e0002a
:10d4ac0004003200d0c2b300d072020000000000b1
:10d4bc0003003700b0c2b300d072020000000000bd
:10d4cc000040eb0030479800210037001e409000d0
:10d4dc000004e0001e0032006e4090000004e000ea
:10d4ec001b0032001e4078000004e0000b003200ec
:10d4fc005e4090000004e00008003a0010c0b30049
:10d50c00204798000040eb0030479800b0c5b300ae
:10d51c00d0720200000000000d0037001e407800a1
:10d52c000004e0000a003a005e4090000004e000b5
:10d53c00070032000040eb00204798000040eb0051
:10d54c0030479800d0c5b300d07202000000000034
:10d55c00de409000014f7800ee409000114798009b
:10d56c0088ff370040b72800166e0200000000004c
:10d57c000080fa00000006000000fa00d0b7280076
:10d58c00f26d0200000000000080fa0000000600ae
:10d59c000600fa00881f7800c922a800c902a8005a
:10d5ac00cb02a900cb22a900c8c2a900819c2100f2
:10d5bc00114078000040a00080487800819c210038
:10d5cc00114078000030a1008048780080c0eb004a
:10d5dc0020c0b3008e7d020000000000e6ff0700b3
:10d5ec00067302000000000011a32100804878009f
:10d5fc0010a32100104078000080fb004400de00e6
:10d60c008040780020a321000148780020a321004d
:10d61c00104078000080fb00e10f50000c0132003c
:10d62c00e10f500003003c000000e0000600320057
:10d63c0044013700e40f50003a013200e60f50006d
:10d64c00290132003f01370010a32100104078005f
:10d65c000080fb00cf80de00f200200003002000e1
:10d66c00820f5000838f5800f4003e0000600100d0
:10d67c00390137000e0037000f0037001400370057
:10d68c0019003700ed0037001d003700230037006c
:10d69c0029003700a0003700e8003700e70037000a
:10d6ac00e6003700e5003700e4003700dd00370006
:10d6bc00b1ff0700e5003700147e020000000000f7
:10d6cc0010c0b3002c73020000000000df00370014
:10d6dc00607e02000000000010c0b3002c7302003a
:10d6ec0000000000d9003700527f0200000000004b
:10d6fc00004078002c73020000000000d3003700bb
:10d70c000040eb00c87f02000000000010c0b30016
:10d71c002c73020000000000cc00370010c0b300d6
:10d72c00c87f02000000000010c0b3002c73020080
:10d73c0000000000c5003700067302000000000066
:10d74c000080fb00200798002e0090004800dd00b0
:10d75c002007980006730200000000000080fb0008
:10d76c00ae009000010070002007980006730200c4
:10d77c00000000000080fb00100798001e009000c5
:10d78c004800dd001007980006730200000000003e
:10d79c000080fb009e0090000100700010079800b4
:10d7ac00ae00900000002100808f500006003e006b
:10d7bc009e00900000002100808f50000600360073
:10d7cc0001003700000000000040eb002c73020049
:10d7dc00000000009d0037000000eb00000f7800f7
:10d7ec000600370080cf80001e0440000673020044
:10d7fc0000000000004c78001e0fe8002e00900086
:10d80c009e007800808f5000f6ff3900147e0200d5
:10d81c00000000000000eb00000f78000b00370048
:10d82c0080cf80001e004000104078000080fb007c
:10d83c00fc7e020000000000a27f0200000000003d
:10d84c00e14f5000dfff32001e0fe8002e00900069
:10d85c009e007800808f5000f1ff39001e00900070
:10d86c000000e900200798000000eb00000f780092
:10d87c001200370080cf80001e044000527f02004f
:10d88c000000000000407800004c78002e00900052
:10d89c009e007800808f5000040031000040eb00a7
:10d8ac00c87f0200000000000300370010c0b30066
:10d8bc00c87f0200000000001e0fe8001e00900050
:10d8cc009e007800808f5000eaff3900607e0200d5
:10d8dc000000000010c0b3002c7302000000000018
:10d8ec000000eb00000f78000600370080cf8000ae
:10d8fc001e004000104078002c7302000000000055
:10d90c001e0fe8001e0090009e007800808f5000d3
:10d91c00f6ff39004d00370010c0b3002c73020025
:10d92c000000000000000000101180006100600089
:10d93c000000e000fcff32003011800080407800d5
:10d94c0010a3210001487800100020001007980057
:10d95c0010a32100104078000080fb00e20f500063
:10d96c0015003200e20f500005003c000000e00002
:10d97c000b003200e10f50000c0032002100370088
:10d98c00f00f50001300320001022000810f5000f4
:10d99c0016003200e30f50000a0032001900370065
:10d9ac00206402000000000019003700fe63020032
:10d9bc000000000016003700e063020000000000c9
:10d9cc0013003700426402000000000010079800aa
:10d9dc000f003700819c2100114078000000a1004d
:10d9ec000010a1008048780009003700819c2100bc
:10d9fc00114078000000a0000010a10080487800c1
:10da0c00030037000000eb00200798000000000026
:10da1c001e009000004078002c73020000000000f3
:10da2c000a0037000040eb0039fe070010c0b300bd
:10da3c002c73020000000000040037000040eb00d3
:10da4c002c730200000000000000000041003700b1
:10da5c0010a3210010407800ef40600010a32100bb
:10da6c000148780010a32100104078008040e800a5
:10da7c0010a321000148780010c0b3002c730200e1
:10da8c000000000030a321008040eb00014878002a
:10da9c000e00370006730200000000000080fb003f
:10daac00fc7e020000000000a27f020000000000cb
:10dabc002c7302000000000030a3210010407800fd
:10dacc008040e80030a321000148780030a32100f9
:10dadc009040780010a321001040780080cf5000b7
:10daec00ecff39001b00370010a321001040780018
:10dafc00e340600010a321000148780010a321002e
:10db0c00104078008040780020c0b3008e7d020069
:10db1c000000000010c0b3002c73020000000000d5
:10db2c000c00370010a32100104078005a9102001d
:10db3c000000000010c0b3002c73020000000000b5
:10db4c00040037000040eb002c73020000000000c2
:10db5c0000000000a2fe37004f0478000080fa009d
:10db6c00000006000200fa00000f78001e0078008a
:10db7c000000e0000300320010c3b300b302070042
:10db8c000200370000c3b300b00207000080fa00a7
:10db9c00000006000600fa00100798002107980004
:10dbac000000eb00000f7800050037001e0090000d
:10dbbc001e00400010407800a40207001e0fe80071
:10dbcc002e0090009e007800808f5000f7ff3900e7
:10dbdc000080fa00000006000400fa00100798000c
:10dbec00020037001e407800980207001e009000cb
:10dbfc00104f78001e80fb000000ea004f00de0092
:10dc0c00004078009e0090008100e8001107980009
:10dc1c000004e000f3ff3a000080fa000000060068
:10dc2c000400fa0010079800020037001e4078002c
:10dc3c00860207001e009000104f78001e80fb002b
:10dc4c000000ea004f00de00004078009e009000cb
:10dc5c008100e800110798000004e000f3ff3a008f
:10dc6c00d0c0b30079020700a0c0b3007702070050
:10dc7c000080fa00000006000400fa00204798001b
:10dc8c0000c8b30010479800e0b42800d2ff07008a
:10dc9c000040eb00004f78000f003700ae409000c2
:10dcac001e40900000c060000004e0000300320041
:10dcbc0010c3b300650207000200370000c3b300b5
:10dccc00620207001e4090000080fb000000d100a3
:10dcdc00104798001e4fe8001e407800e74f500098
:10dcec00eeff36000080fa00000006000e00fa007d
:10dcfc0050079800610798000040eb0050479800cf
:10dd0c0000102e00515f2000008fbe000040eb0081
:10dd1c0040479800310037001e01be005e009000a5
:10dd2c00ee0090008606020000000000300798000c
:10dd3c00410798005e4090000004e00005003a00a6
:10dd4c003e009000ce009000e00f5000e08f580095
:10dd5c00190032003e009000004078000043b000f3
:10dd6c003a020700ce0090001e0078000088b9002f
:10dd7c00000178009e0090003e0090000088b900e1
:10dd8c0000007800000141003e0090001e00b80029
:10dd9c0001014100820078005e019000ee019000cc
:10ddac0000005100818059005007980061079800cd
:10ddbc0010c0b300504798001e00be00a200200007
:10ddcc00030020008606020000000000008fbe0049
:10dddc004e4090000040e800404798004e409000b4
:10ddec00e74f5000ccff36005e00900000407800fa
:10ddfc000043b000150207000080fa000000060086
:10de0c000c00fa0040079800510798000000eb0046
:10de1c00000f78000000eb00100798006000b800bd
:10de2c0020079800310798004e019000de01900009
:10de3c00f0232400f1002000800f5100818f590045
:10de4c00210036004e009000de00900002242400d9
:10de5c00f300200086060200000000002007980056
:10de6c00310798002e00900070000700c0c2b3006c
:10de7c00f60107004e009000de0090000224240002
:10de8c00f3002000a60602000000000040079800e6
:10de9c00510798004e019000de019000703e20006a
:10deac0001002000800f5100818f590002003e00bc
:10debc0010b5280048ff070010002000000f780064
:10decc0010002000100798004e019000de01900019
:10dedc00703e200001002000800f5100818f5900fe
:10deec00320036004e009000de009000823e200092
:10defc0003002000860602000000000020079800a6
:10df0c00310798002e019000be01900030062000d1
:10df1c0001002000800f5100818f59000300360052
:10df2c002e00900041000700140037001e007800fe
:10df3c000000e0000f0032002e019000be019000a6
:10df4c009000200001002000800f5100818f5900ab
:10df5c000300360000c3b300bc0107000200370009
:10df6c0060b528001cff07002e0090002f00070052
:10df7c00020037002e0090002c000700c0c2b30036
:10df8c00b20107004e009000de009000823e20009f
:10df9c0003002000a60602000000000040079800c5
:10dfac005107980010002000100798004e019000b7
:10dfbc00de0190003006200001002000800f51008f
:10dfcc00818f5900030036004e00900017000700a7
:10dfdc00140037001e0090000000e0000f0032001b
:10dfec004e019000de019000900020000100200006
:10dffc00800f5100818f59000300360000c3b3001d
:10e00c00920107000200370060b52800f2fe0700fd
:10e01c004e00900005000700020037004e009000f3
:10e02c00020007000080fa00000006000800fa0059
:10e03c00300798000040eb00304798000071220038
:10e04c00000f78000040eb002047980022003700ba
:10e05c00be0090001e00780000017800110009003d
:10e06c008280d800200798003e4090000004e00019
:10e07c0003003a002e0090000000e0000d0032007a
:10e08c002e009000004078000043b0006f010700a4
:10e09c00ae0090001e0078000088b90000007800e7
:10e0ac00be009000008050003007980010c0b300f4
:10e0bc00304798009e007800a000200000017800f6
:10e0cc00110009008280d800000f78002e409000cb
:10e0dc000040e800204798002e409000e34f50008d
:10e0ec00dbff36003e009000004078000043b0009b
:10e0fc00560107000080fa00000006000600fa0036
:10e10c00404798000040eb002047980040c6b30001
:10e11c00004f78000040eb001047980023003700b8
:10e12c004e4090008080fb001e80fb0000017800b8
:10e13c00110009008280d800304798002e409000d2
:10e14c000004e00003003a003e4090000004e000b0
:10e15c000d0032003e4090000043b0003b01070030
:10e16c003e4090009e80fb000088b90000007800c3
:10e17c0000407800ce40900000c05000404798000e
:10e18c0010c0b300204798009e80fb00a000200028
:10e19c0000017800110009008280d800004f78003f
:10e1ac001e4090000040e800104798001e40900070
:10e1bc00e14f5000daff36004e4090000043b000b3
:10e1cc00220107000080fa00000006000400fa009b
:10e1dc001007980021002000c0b328006dfe070036
:10e1ec001e0090004400de006f0f6000e0b32800ba
:10e1fc001e00400010407800140107001e00900023
:10e20c006f0f6000e0b328001e0040001040780043
:10e21c000e0107000080fa00000006000400fa005e
:10e22c001007980000c3b300da00070080c7b300e2
:10e23c00d80007001e0090004400de006f0f600045
:10e24c00e0b328001e00400010407800d100070009
:10e25c001e0090006f0f6000e0b328001e0040000d
:10e26c0010407800cb0007000080fa000000060088
:10e27c000400fa001007980021002000c0b3280009
:10e28c0044fe07001e0090004c00de00000f7800da
:10e29c00e0b328001e00400010407800eb0007009f
:10e2ac001e0090004800de006f0f6000e0b32800f5
:10e2bc001e00400010407800e40007001e00900093
:10e2cc004400de006f0f6000e0b328001e00400029
:10e2dc0010407800dd0007001e0090006f0f6000fa
:10e2ec00e0b328001e00400010407800d700070063
:10e2fc000080fa00000006000600fa0020079800d3
:10e30c002e0090007d00b90080007800d002200023
:10e31c0000017800110009008280d800000f7800fd
:10e32c009e007800400620000001780011000900d2
:10e33c008280d8000040780070ff0700e0c2b30074
:10e34c00c20007009e007800400620000001780003
:10e35c00110009008280d8008000fd002047980041
:10e36c002e409000e94f500002003e0000c3b30065
:10e37c00b60007009e0078004006200000017800df
:10e38c00110009008280d8008000fd000040780058
:10e39c005aff07000080fa00000006000800fa008f
:10e3ac00200798003107980032c0bf000080fb00a6
:10e3bc00000f78002e0090000040780032e0b7008b
:10e3cc003e0090001080ba00c800dd003e009000b6
:10e3dc001000ba0001007000100798001e007800b1
:10e3ec000040780032e0b7001e0090000080fa0078
:10e3fc00000006000000fa00209f21001040780069
:10e40c00e94f500008003200209f21001040780096
:10e41c000080fb0080004000009d21000080400037
:10e42c0010007800401188002022ef002062a80024
:10e43c002222ef0021e2a8002342a8008560a90057
:10e44c000080fa00000006000000fa0010118000a5
:10e45c004800de00614060000080fa000000060009
:10e46c000000fa001011800000407800614060004c
:10e47c000080fa00000006000000fa000000eb002b
:10e48c0050d188001000200040d18800e0cf8000df
:10e49c000090a100e0cf88000080fa000000060088
:10e4ac000200fa00111180000020200000806000a2
:10e4bc000000e00016003a0050d18000000fe80088
:10e4cc00000021009e007800808f500002003a006e
:10e4dc000000eb00000f780040d180009e00780017
:10e4ec00808f5000090032009e00780051d18800c6
:10e4fc0081cf800050d18000008040001040780017
:10e50c000080fb0020118800010037000000000093
:10e51c000080fa00000006000200fa00010037003b
:10e52c000000000050d18000000fe8000000210026
:10e53c009e007800808f500002003a000000eb0033
:10e54c00000f780040d180009e007800808f500032
:10e55c000e003200111180000020200000806000ad
:10e56c000000e000eeff3a009e00780051d18800d8
:10e57c0081cf800050d18000008040001040780096
:10e58c000080fb0020118800e6ff37000080fa00b5
:10e59c00000006000200fa00004f780041d1800014
:10e5ac0050d18000808f500005003a00c222a90093
:10e5bc00e0cf80000090a000e0cf88000e00370074
:10e5cc0081cf800040d18000008040009e407800c8
:10e5dc000148780040d180000000e80040d188005c
:10e5ec0041d1800000002100808f500002003a00d1
:10e5fc000000eb0040d188000080fa00000006000b
:10e60c000000fa00000000001011800061006000a2
:10e61c000000e000fcff3200301180000040780068
:10e62c000080fa00000006000000fa000000000064
:10e63c001111800000102000008060000000e0003c
:10e64c00fbff32000080fa00000006000200fa0016
:10e65c00004f7800e1cf80000010200000806000a7
:10e66c000000e00009003a000000000011118000d9
:10e67c0000202000008060000000e000fbff3a005a
:10e68c001e00fb0020118800010037000000000074
:10e69c000080fa00000006000200fa00004f78002b
:10e6ac001e80fb00401188000080fa00000006006c
:10e6bc000000fa00101180000000d10061406000e1
:10e6cc000080fa00000006000000fa001111800022
:10e6dc00d0ff2f0000806000101188000080fa002d
:10e6ec00000006000000fa00a104800000002100d8
:10e6fc00008060000000e00013003a0041d0800070
:10e70c0030d08000808f50001100320000000000db
:10e71c001111800000202000008060000000e0004b
:10e72c00fbff3a008580a9009580a80021d08000cd
:10e73c0030d0800000804000104078000080fb004a
:10e74c002011880003003700000000000100370092
:10e75c00000000000080fa0000000600809fbe0050
:10e76c000000fa00f1cf800010d080000080400043
:10e77c0031118000814078000148780010d0800071
:10e78c000000e80010d0880011d0800000d080007c
:10e79c00808f500001003a009560a9008560a900a7
:10e7ac000080fa004f00be0000400600809fbe00b3
:10e7bc000000fa0030d080000000e80030d0880063
:10e7cc0031d0800040d08000808f500002003a0091
:10e7dc009580a9000600370021d0800030d0800041
:10e7ec0000804000104078000080fb002011880061
:10e7fc008580a9000080fa004f00be000040060092
:10e80c000000fa00a0b82800f26d02000000000021
:10e81c000080fa00000006000600fa00c222a800e0
:10e82c0021010700f6ff07001a010700e1a22100f1
:10e83c0080487800e0a22100104078000004e0003d
:10e84c000e013500e0a22100104078000004e00029
:10e85c0002003a00eaff0700f3ff3700e0a22100b4
:10e86c0010407800e14f500006003a000e010700fe
:10e87c004e420200000000000b010700e0ff070001
:10e88c00e9ff3700e0a2210010407800e24f500071
:10e89c0006003a0004010700ce6a020000000000e6
:10e8ac0001010700d6ff0700dfff3700e0a22100bf
:10e8bc0010407800e34f500006003a00fa000700c1
:10e8cc00c44e020000000000f7000700ccff070058
:10e8dc00d5ff3700e0a2210010407800e44f500033
:10e8ec0004003a00f0000700ef000700c4ff070027
:10e8fc00cdff3700e0a2210010407800e54f50001a
:10e90c0006003a00e80007006c520200000000000c
:10e91c00e5000700baff0700c3ff3700e0a22100a3
:10e92c0010407800e64f500006003a00de00070069
:10e93c003681020000000000db000700b0ff07007a
:10e94c00b9ff3700e0a2210010407800e74f5000db
:10e95c0004003a00d4000700d3000700a8ff07000a
:10e96c00b1ff3700e0a2210010407800ef4f5000bb
:10e97c0008003a0010c0b3002c7302000000000025
:10e98c00c222a9001a730200000000000000fe0061
:10e99c00a5ff3700e0a2210010407800f04f500096
:10e9ac0003003a000040eb00040207009eff370012
:10e9bc00e0a2210010407800f14f500003003a0013
:10e9cc0010c0b300fd01070097ff3700e0a2210043
:10e9dc0010407800f24f500031003a001021ef0047
:10e9ec001e21ef009c21ef005136800000fe2f000d
:10e9fc00008060006001b30050368800a50007005d
:10ea0c000080fb00000f78009e00780062806000a0
:10ea1c000000e0000100320010a1a8001e007800e8
:10ea2c0061006000004078000004e000010032004a
:10ea3c001081a800970007000080fb004800dd0053
:10ea4c00000f7800930007000080fb001e0f700081
:10ea5c001e017800d20c88009e007800c10c880042
:10ea6c0060002000e00c88008a0007000080fb009a
:10ea7c004800dd00000f7800860007000080fb00d6
:10ea8c001e0f70001e0178006208880011e1a800ba
:10ea9c0010c0b3002c7302000000000062ff3700ae
:10eaac00e0a2210010407800f34f50000a003a0019
:10eabc001021ef009c21ef005136800000fe2f004a
:10eacc00008060005036880010c0b3002c73020028
:10eadc000000000054ff3700e0a221001040780035
:10eaec00f44f500010003a0021e3a800c0002000b1
:10eafc00568a020000000000000f780021e3a900f4
:10eb0c001e0078004800de00004078002c730200e4
:10eb1c00000000001e007800004078002c730200fa
:10eb2c000000000040ff3700e0a2210010407800f8
:10eb3c00f54f50001c003a0021e3a80001003700fb
:10eb4c0000000000c0002000568a020000000000f7
:10eb5c00000f78001a730200000000001e007800fd
:10eb6c004800de00004078002c730200000000001a
:10eb7c001e007800004078002c730200000000009a
:10eb8c003672020000000000e14f5000ecff3a002a
:10eb9c0006730200000000000080fb00000f7800ec
:10ebac0021e3a90020ff3700e0a2210010407800eb
:10ebbc00f64f50001e003a003a62020000000000be
:10ebcc0010079800210798001e009000ae009000de
:10ebdc004808de00004078002c73020000000000a2
:10ebec001e009000ae0090004008de00004078004f
:10ebfc002c730200000000001e009000ae0090007c
:10ec0c004809dd004800de0000007100c808de0085
:10ec1c00004078002c730200000000001e009000e1
:10ec2c00004078002c73020000000000fefe37004c
:10ec3c00e0a22100104078000080fb004500de00bf
:10ec4c00004078000080fb00620060000000e000e3
:10ec5c0006003200e0a221001040780019000700e5
:10ec6c002c73020000000000effe37000040eb00a8
:10ec7c002c73020000000000ebfe3700e0a2210024
:10ec8c0010407800a30007002c7302000000000065
:10ec9c00e5fe37000000fa000673020000000000d9
:10ecac000080fa00000006000000fa0000c0eb0033
:10ecbc00040007000040eb00960007000080fa00fb
:10eccc00000006000400fa00204798000040eb000a
:10ecdc00004f78002e4090000080fb007000600018
:10ecec000000e0000200320010c0b300004f7800ba
:10ecfc009e40780061c060000080fb0061006000f5
:10ed0c004a00dd0042168000f1bf2f008100610037
:10ed1c0001007000401688000040eb00004f7800a6
:10ed2c002e4090000080fb00680060000000e000b6
:10ed3c000200320010c0b300004f78009e407800f3
:10ed4c0061c060000080fb00610060004900dd00d4
:10ed5c0042168000f1df2f0081006100010070007d
:10ed6c00401688000040eb00004f78002e409000c9
:10ed7c000080fb00640060000000e0000200320034
:10ed8c0010c0b300004f78009e40780061c0600056
:10ed9c000080fb00610060004800dd00421680002e
:10edac00f1ef2f0081006100010070004016880017
:10edbc000040eb00004f78002e4090000080fb00dc
:10edcc00620060000000e0000200320010c0b300de
:10eddc00004f78009e40780061c060000080fb000e
:10edec00610060004700dd0042168000f1f72f0043
:10edfc008100610001007000401688000040eb00ab
:10ee0c00004f78002e4090000080fb0061006000f5
:10ee1c00004078000004e0000200320010c0b30093
:10ee2c00004f78009e40780061c060000080fb00bd
:10ee3c00610060004600dd0042168000f1fb2f00ef
:10ee4c008100610001007000401688005000200015
:10ee5c00b28b020000000000ae40900000ceb30068
:10ee6c0000c0600020479800511680000040200030
:10ee7c00008060000000e000030032002e40900093
:10ee8c000044a0002047980051168000002020006c
:10ee9c00008060000000e000030032002e40900073
:10eeac000034a0002047980051168000001020006c
:10eebc00008060000000e000030032002e40900053
:10eecc000024a00020479800511680000008200064
:10eedc00008060000000e000030032002e40900033
:10eeec000014a00020479800511680000004200058
:10eefc00008060000000e000030032002e40900013
:10ef0c000004a000204798002e4090000080fa00da
:10ef1c00000006000400fa00204798002e409000e4
:10ef2c008080fb0000042000008060000000e000f6
:10ef3c0003003200c002a900c202a8000200370080
:10ef4c00c002a900c202a9002e4090008080fb00e4
:10ef5c0000022000008060000000e000030032008e
:10ef6c00c962a800cb62a90002003700cb62a900dd
:10ef7c00c962a9000040eb00004f78002e409000c1
:10ef8c000080fb00700060000000e0000200320016
:10ef9c0010c0b300004f78009e40780061c0600044
:10efac000080fb00610060004a00dd00521680000a
:10efbc00f1bf2f0081006100010070005016880025
:10efcc000040eb00004f78002e4090000080fb00ca
:10efdc00680060000000e0000200320010c0b300c6
:10efec00004f78009e40780061c060000080fb00fc
:10effc00610060004900dd0052168000f1df2f0037
:10f00c008100610001007000501688000040eb0088
:10f01c00004f78002e4090000080fb0064006000e0
:10f02c000000e0000200320010c0b300004f780076
:10f03c009e40780061c060000080fb0061006000b1
:10f04c004800dd0052168000f1ef2f0081006100b6
:10f05c0001007000501688000040eb00004f780053
:10f06c002e4090000080fb00620060000000e00079
:10f07c000200320010c0b300004f78009e407800b0
:10f08c0061c060000080fb00610060004700dd0093
:10f09c0052168000f1f72f00810061000100700012
:10f0ac00501688000040eb00004f78002e40900076
:10f0bc000080fb0061006000004078000004e0006c
:10f0cc000200320010c0b300004f78009e40780060
:10f0dc0061c060000080fb00610060004600dd0044
:10f0ec0052168000f1fb2f008100610001007000be
:10f0fc005016880050002000b28b02000000000067
:10f10c00ae40900000ceb30000c0600020479800d5
:10f11c005116800000402000008060000000e000dc
:10f12c00030032002e4090000044a00020479800bd
:10f13c005116800000202000008060000000e000dc
:10f14c00030032002e4090000034a00020479800ad
:10f15c005116800000102000008060000000e000cc
:10f16c00030032002e4090000024a000204798009d
:10f17c005116800000082000008060000000e000b4
:10f18c00030032002e4090000014a000204798008d
:10f19c005116800000042000008060000000e00098
:10f1ac00030032002e4090000004a000204798007d
:10f1bc002e4090000080fa00000006000400fa00c7
:10f1cc0020479800ae4090000040eb0048840200bd
:10f1dc0000000000004f78001e4078000004e000a2
:10f1ec0001003200c222a8001e4078002c730200dd
:10f1fc000000000001003700000000003672020021
:10f20c00000000000004e000100032000673020051
:10f21c0000000000104798001e409000e14f400095
:10f22c00050032001e4090001e4040002c7302006e
:10f23c00000000000500370010c0b3002c73020062
:10f24c00000000000080fa00000006001e4078005c
:10f25c000004e000e8ff3a0060d180000000e0000c
:10f26c000f003a000080eb0060d18800101680007f
:10f27c000000d100614060000004a2006140600009
:10f28c000080fb006100600000004000121680004e
:10f29c00d1ff2f0081006100010070001016880062
:10f2ac0060d180000000e90060d18800d3ff3700f6
:10f2bc000000fa00df000700c1a121001140780016
:10f2cc000020a00080487800c1a1210011407800e6
:10f2dc000030a10080487800c1a1210011407800c5
:10f2ec000040a10080487800067302000000000076
:10f2fc00d1a1210080487800d0a1210010407800d5
:10f30c000080fb00e10f500003003200e20f5000c0
:10f31c0004003200460037008d000700450007004e
:10f32c00430037008a000700730107004100070003
:10f33c0020c0b3009200070000c0eb00960107004c
:10f34c0000c0eb00940107003a00070030c0b30086
:10f35c008b0007000000eb00f0d08800070037009e
:10f36c00f0d080000000e800f0d08800f1d08000e0
:10f37c00900f2000808f5000040036004e010700d3
:10f38c000004e000f6ff320001003700000000002e
:10f39c00280007006e0007002600070030c0b300ed
:10f3ac0077000700f0d0800080407800200020001b
:10f3bc000008dd002c7302000000000000a22100f8
:10f3cc008040eb000148780011003700fc0007007a
:10f3dc002c73020000000000f90007002c730200df
:10f3ec0000000000f60007002c7302000000000073
:10f3fc00f30007002c7302000000000000a22100a3
:10f40c00104078008040e80000a2210001487800fc
:10f41c0000a22100104078008080fb00f0d080001a
:10f42c00808f5000e9ff3900020007000000000047
:10f43c00adff37000000fa00c0a1210010007800d9
:10f44c00634060000080fb00e10f50003d00320083
:10f45c00e10f500003003c000000e0000600320009
:10f46c0039003700e20f50000c003200e30f50005f
:10f47c0027003200340037009d01070010c0b30094
:10f48c0045010700c1a12100114078000000a00037
:10f49c000010a100804878002b003700c0a121008b
:10f4ac0010407800684060000004e0000c0032005e
:10f4bc00c0a1210010407800704060000004e00002
:10f4cc00020032000c010700010037002a0107007e
:10f4dc00c1a12100114078000030a10080487800c3
:10f4ec006301070020c0b3002b0107008001070057
:10f4fc0010c0b30028010700c1a121001140780001
:10f50c000000a0000010a100804878000e00370019
:10f51c005701070020c0b3001f010700740107004a
:10f52c0010c0b3001c010700c1a1210011407800dc
:10f53c000000a0000010a10080487800000000002e
:10f54c0001003700000000000080fa0000000600f7
:10f55c000000fa0046010700a0c0b3000e0107002e
:10f56c0063010700c1a12100114078000000a10037
:10f57c000010a100804878000080fa00000006000e
:10f58c000200fa00004f78001e80fb00e10f5000d3
:10f59c0025003200e10f500003003c000000e000a9
:10f5ac000600320021003700e20f5000110032003b
:10f5bc00e30f5000030032001c003700e4ff07008b
:10f5cc001a0037002a01070010c0b300f200070030
:10f5dc004701070020c0b300ef000700c1a12100c4
:10f5ec00114078000000a0000010a00080487800b6
:10f5fc000e0037001e01070020c0b300e600070014
:10f60c003b01070020c0b300e3000700c1a12100ab
:10f61c00114078000000a1000010a0008048780084
:10f62c000000000001003700000000000080fa001c
:10f63c00000006000000fa00c8e2a800c902a900f8
:10f64c00c922a900c8c2a900cae2a900cb02a9001c
:10f65c00cb22a900cac2a9000080fa000000060053
:10f66c000600fa00404798000040eb001047980055
:10f67c00f7000700c0a1210010407800684060002e
:10f68c000004e00009003200c0a121001000780045
:10f69c004400de006140600076000700c1a121003b
:10f6ac00114078000030a1008048780010c0b300f1
:10f6bc00204798000040eb00004f78003a003700dc
:10f6cc00ce4090002e40900000c060000004e0008e
:10f6dc0002003a00a800070001003700860007006e
:10f6ec00bb000700501680004700de006140600040
:10f6fc00304798004e4090000080fb000000d10085
:10f70c00404798001e4090000080fb000000d10094
:10f71c00104798003e409000e14f500004003a0022
:10f72c009e40900000c8b30000c0400010479800f5
:10f73c00c7000700c0a121001040780063406000a2
:10f74c00e24f500017003a001e407800e64f500080
:10f75c0014003a00c1a12100114078000030a00033
:10f76c0080487800ce4090002e40900000c0600091
:10f77c000004e00005003a00c1a12100114078000e
:10f78c000040a1008048780004003700c1a121008e
:10f79c00114078000040a000804878001e40900086
:10f7ac00050037001e4fe8001e407800e74f500060
:10f7bc00c3ff36001e4090000080fa0000000600d7
:10f7cc000400fa000040eb0010479800a00007006e
:10f7dc00c0a1210010407800684060000004e000e7
:10f7ec0009003200c0a12100100078004400de00a6
:10f7fc00614060001f000700c1a12100114078008a
:10f80c000030a100804878000040eb00004f7800e9
:10f81c00120037006e000700501680004700de0013
:10f82c0061406000204798001e4090000080fb0063
:10f83c000000d100104798002e4090000004e0001a
:10f84c00040032009e40900000c8b30000c040008d
:10f85c00104798007e0007001e4fe8001e407800fd
:10f86c00e74f5000ebff36001e4090000080fa007e
:10f87c00000006000400fa00204798002e4090007b
:10f88c000004e00002003a003b00070001003700d2
:10f89c00190007004e000700501680004700de00dc
:10f8ac0061406000004f7800690007001e4078003e
:10f8bc000080fa00000006000200fa004400070075
:10f8cc00501680004700de0061406000004f780059
:10f8dc005f0007001e4078000080fa000000060060
:10f8ec000000fa00501680004700de006140600006
:10f8fc000080fa00000006000000fa00c0a1210000
:10f90c00100078004200de006140600000c0ea0098
:10f91c00614060000080fb00610060004900dd0078
:10f92c0042168000f1df2f008100610001007000a1
:10f93c0040168800c0a12100100078004200de00b3
:10f94c00614060000080fb00610060004900dd0048
:10f95c0052168000f1df2f00810061000100700061
:10f96c005016880040012000b28b020000000000fd
:10f97c000080fa00000006000000fa00cb22a9006b
:10f98c00c922a90040012000b28b02000000000037
:10f99c000080fa00000006000400fa0020479800de
:10f9ac000040eb00004f7800030037000800070010
:10f9bc00270007001e4fe8002e4090009e40780064
:10f9cc0080cf5000f9ff39000080fa0000000600db
:10f9dc000000fa00c0a12100100078004200de00f7
:10f9ec006140600000c0ea00614060000080fb00e4
:10f9fc00610060004800dd0042168000f1ef2f002e
:10fa0c00810061000100700040168800c0a1210037
:10fa1c00100078004200de00614060000080fb00b6
:10fa2c00610060004800dd0052168000f1ef2f00ed
:10fa3c008100610001007000501688004006200013
:10fa4c00b28b0200000000000080fa0000000600eb
:10fa5c000000fa00cb02a900c902a9004006200050
:10fa6c00b28b0200000000000080fa0000000600cb
:10fa7c000000fa00c0a12100100078004200de0056
:10fa8c006140600000c0ea00614060000080fb0043
:10fa9c00610060004600dd0042168000f1fb2f0083
:10faac00810061000100700040168800c0a1210097
:10fabc00100078004200de00614060000080fb0016
:10facc00610060004600dd0052168000f1fb2f0043
:10fadc008100610001007000501688004001200078
:10faec00b28b0200000000000080fa00000006004b
:10fafc000000fa00cac2a900c8c2a9004001200037
:10fb0c00b28b0200000000000080fa00000006002a
:10fb1c000200fa00004f780011479800a0a02100c5
:10fb2c001e4878001e407800e34f500005003a0054
:10fb3c000020200060d088000008200070d08800d1
:10fb4c00040037000020200060d088000020200036
:10fb5c0070d088001e4090000080fb00e10f500028
:10fb6c000e003200e20f5000160032000000e000e0
:10fb7c001e003a0000a1210041c1b30001487800e9
:10fb8c0010a1210041c6b3000148780020a121003a
:10fb9c0021c3b300014878001e00370000a12100ea
:10fbac0021c0b3000148780010a12100a1c0b3000e
:10fbbc000148780020a1210051c0b3000148780011
:10fbcc001400370000a1210011c0b30001487800d7
:10fbdc0010a1210051c0b3000148780020a12100e0
:10fbec0021c0b300014878000a00370000a12100b1
:10fbfc008040eb000148780010a121008040eb0010
:10fc0c000148780020a121008040eb0001487800d9
:10fc1c00000000000080fa00000006000200fa005c
:10fc2c000000eb00000f780010a1210010407800bc
:10fc3c0080407800003020001d0107005116800024
:10fc4c0000102000008060000000e0000500320081
:10fc5c005116800000202000008060000000e000b1
:10fc6c0002003a0010002000000f780010a12100c3
:10fc7c00104078008040780000202000250107000b
:10fc8c0010a1210010407800804078000010200066
:10fc9c002001070010a1210010407800804078005e
:10fcac0000202000020107001e0078000080fa00ee
:10fcbc00000006000000fa0010a12100104078009e
:10fccc0080407800003020001201070010a12100b4
:10fcdc00104078008040780000102000f4000700ed
:10fcec0010a12100104078008040780000202000f6
:10fcfc00ef0007000000eb000080fa000000060097
:10fd0c000c00fa00500798000000eb002007980048
:10fd1c00709b2100104078000080fb000000e9007f
:10fd2c00110020000008dd0030079800de00900074
:10fd3c00110798000000eb00000f7800230037003b
:10fd4c0000a12100904078001e0190003e00900020
:10fd5c00000061000141780001202000fe00070036
:10fd6c0010a1210010407800804078000010200085
:10fd7c00cf00070000082000220107000080fb00d4
:10fd8c004007980010a121001040780080407800b6
:10fd9c0000102000df0007001e0090000000400053
:10fdac00100798002e0090000000400020079800db
:10fdbc004e0090000000e000030032002e00900086
:10fdcc000000e800200798001e0fe800709b21003f
:10fddc00104078000080fb009e0f5000d8ff3e00c2
:10fdec002e0090000080fa00000006000800fa00c7
:10fdfc0030079800709b2100104078000080fb00b9
:10fe0c000000e900110020000008dd002007980028
:10fe1c00be009000110798000000eb00000f780066
:10fe2c001600370000a12100904078001e019000c0
:10fe3c002e0090000000610001417800012020009c
:10fe4c00c500070010a12100104078008040780008
:10fe5c00001020009600070010a12100104078002f
:10fe6c008040780000102000aa0007001e009000bf
:10fe7c0000004000100798001e0fe800709b210046
:10fe8c00104078000080fb009e0f5000e5ff3e0004
:10fe9c000080fa00000006000600fa000000eb00eb
:10feac001007980000202000d60007000000eb008f
:10febc00000f78001800370010a1210010407800c6
:10fecc0080407800001020007900070000202000fe
:10fedc00cc0007000080fb002007980010a1210037
:10feec001040780080407800001020008900070046
:10fefc001e00900000004000100798002e0090009b
:10ff0c000000e000030032001e0090000000e8003a
:10ff1c00100798001e0fe800709b2100104078001d
:10ff2c000080fb009e0f5000e3ff3e001e0090007f
:10ff3c000080fa00000006000200fa0070d0800079
:10ff4c00b000070010a1210010407800804078001c
:10ff5c00001020005600070070d08000a900070098
:10ff6c00004f780010a121001040780080407800ec
:10ff7c0000102000670007001e4078000080fa0087
:10ff8c00000006000200fa00004f780000a12100da
:10ff9c001041780061d080001e80fb006e000700cd
:10ffac0010a1210010407800804078000010200043
:10ffbc003f00070010a1210010407800804078001d
:10ffcc0000102000530007000080fa00000006001b
:10ffdc000400fa00204798000040eb00004f780026
:10ffec000b00370010a121001040780080407800f1
:10fffc00001020002e00070010a1210010407800f6
:020000040001f9
:10000c008040780000102000420007001e4fe800de
:10001c002e4090009e40780080cf5000f1ff3900b8
:10002c000080fa00000006000200fa00004f780081
:10003c0000a121001041780061d080001e80fb00df
:10004c00450007000080fa00000006000200fa00dc
:10005c00004f780000a12100904078001e80fb002a
:10006c0001417800011020003b0007000080fa00dd
:10007c00000006000200fa00004f780000a12100e9
:10008c00904078001e80fb000141780001042000a4
:10009c00310007000080fa00000006000000fa00a2
:1000ac0070d08000570007000080fa0000000600a6
:1000bc000400fa00000f780021479800809c210072
:1000cc0010407800704060000004e00008003a0026
:1000dc00601680001e007000601688009e80ea008a
:1000ec004016800000806000401688000300370036
:1000fc00401680001e007000401688002e409000b4
:10010c000080fb00b28b0200000000000080fa00af
:10011c00000006000400fa00000f78002147980048
:10012c009e80ea00601680000080600060168800e7
:10013c009e80ea0040168000008060004016880017
:10014c002e4090000080fb00b28b020000000000eb
:10015c000080fa00000006000600fa00000f78008c
:10016c0011079800424798001e0078000000e0003c
:10017c000b003a001e0090008080ea0060168000a0
:10018c0000806000601688001e0090008080ea00ed
:10019c004016800000806000401688001300370075
:1001ac00809c210010407800704060000004e0004a
:1001bc000a003a00611680001e00900001007000d9
:1001cc00601688001e0090008080ea0040168000b7
:1001dc000080600040168800040037004116800043
:1001ec001e00900001007000401688004e409000e8
:1001fc000080fb00b28b0200000000000080fa00bf
:10020c00000006000200fa00000f78004016800083
:10021c001e00700040168800000000000000000066
:10022c0000000000501680001e0060000000e0007e
:10023c000200320010c0b300010037000040eb0098
:10024c000080fa00000006000000fa00c0b9280087
:10025c00f26d0200000000000080fa0000000600b1
:10026c000800fa0081cf80002107980010002000c0
:10027c00e0d18800f4ff07000673020000000000c4
:10028c00604798006e4090000080fb00e30f500028
:10029c0017003200e30f500007003c00e10f500044
:1002ac005c003200e10f500060003c000000e000f8
:1002bc00ef003200e2003700e60f50000a00320077
:1002cc00e60f500003003c00e50f50009e0032008a
:1002dc00db003700e70f50006c003200e80f5000d5
:1002ec005c003200d6003700d7ff0700df00370074
:1002fc002e00900031c0b300014878002e00900011
:10030c000000e80081c0b3000148780021e3a80098
:10031c00c0002000568a020000000000000f780088
:10032c002e0090000080e8009e007800c808de00d7
:10033c0081407800014878002e0090006300400056
:10034c009e0078008140780001487800b0002000c1
:10035c00568a020000000000000f78002e0090006a
:10036c00640040009e007800c808de0081407800e0
:10037c00014878002e009000650040009e00780037
:10038c008140780001487800a0002000568a0200c5
:10039c0000000000000f78002e0090006600400066
:1003ac009e007800c808de00814078000148780083
:1003bc002e009000670040009e007800814078007d
:1003cc000148780090002000568a020000000000ce
:1003dc00000f78002e009000680040009e0078000e
:1003ec00c808de0081407800014878002e0090009b
:1003fc00690040009e007800814078000148780038
:10040c0021e3a900a10020002e009000c4000700e9
:10041c009600370006730200000000006047980049
:10042c006e409000940007009000370006730200a5
:10043c0000000000604798000673020000000000f6
:10044c0070479800fe4090006e409000c600070078
:10045c008600370006730200000000006047980019
:10046c000673020000000000704798006e40900078
:10047c000080fb00c800dd007e4090000080fb0087
:10048c0001007000e0d1880078003700067302008c
:10049c0000000000604798006e4090000080fb0058
:1004ac00000f78006e409000e14f500004003a00bd
:1004bc0030c0b3005273020000000000030037008c
:1004cc0020c2b30052730200000000000673020049
:1004dc000000000060479800067302000000000056
:1004ec0070479800ee409000a0cab30080cf500037
:1004fc0004003a00fe40900050c5b30080cf50007d
:10050c00050032000000eb00000f780020c2b300a1
:10051c0052730200000000002e00900071c0b30066
:10052c00014878002e0090000000e8009e00780042
:10053c008140780001487800210020002e009000b6
:10054c007700070049003700067302000000000026
:10055c006047980006730200000000007047980086
:10056c008560a9006e4090000080fb00c800dd0093
:10057c007e4090000080fb00010070001007980086
:10058c009e00900000002200808f50000200360078
:10059c0000002200100798001e0090006700400029
:1005ac004300de00000f78002e00900051c0b30015
:1005bc00014878002e0090000000e800ee4090000a
:1005cc00014878002e0090000080e800fe4090006a
:1005dc0001487800310020002e00900050000700e8
:1005ec0080cf8000f0cf88001e0078000000400013
:1005fc0000d088000000eb0010d0880081cf800074
:10060c00408320000080400020d088000000eb00d8
:10061c0030d088000000eb0040d088009560a80026
:10062c00e2d1800021d08000f0cf800082017800e0
:10063c001e019000da900200000000000b00370051
:10064c002e0090008040eb00014878002e009000b6
:10065c000000e8008040eb00014878001100200009
:10066c002e0090002e0007000000000002ff370053
:10067c000080fa00000006000200fa00004f78002b
:10068c00cac2a900cb22a900cb02a900cb42a90067
:10069c00ca02a9001e407800e24f500006003a0042
:1006ac00cac2a800cb02a800cb22a800cb42a8004b
:1006bc00ca02a80005003700cac2a900cb02a900d3
:1006cc00cb22a900cb42a900ca02a9001e40780087
:1006dc00e14f5000030032001e407800e24f500002
:1006ec0007003a00c8c2a900c922a900c902a90082
:1006fc00c942a900c802a900c8e2a8000600370038
:10070c00c8c2a800c922a800c902a800c942a800f2
:10071c00c802a800c8e2a8000080fa000000060089
:10072c000600fa0010079800210798000000eb0063
:10073c00000f7800060037001e0090001e004000dd
:10074c00104078002c730200000000001e0fe8001f
:10075c002e0090009e007800808f5000f6ff39002c
:10076c000080fa00000006000200fa00004f78003a
:10077c00114798001e80fb00e40f50002a00320045
:10078c00e40f500005003c00e10f5000080032005f
:10079c00e20f50001200320038003700e80f500012
:1007ac002b003200f00f50001600320033003700df
:1007bc00c022a9001e409000614060000080fb0038
:1007cc00610060000000400012168000d1ff2f0075
:1007dc0081006100010070001016880027003700ae
:1007ec001e4090000004e00003003200c002a9008b
:1007fc00c202a80021003700c002a900c202a90051
:10080c001e0037001e4090000004e0000300320080
:10081c00c962a800cb62a90018003700cb62a900fe
:10082c00c962a900150037001e40900061406000ad
:10083c000080fb006100600052168000e1ff2f0079
:10084c008100610001007000501688000b00370019
:10085c001e409000614060000080fb006100600061
:10086c004a00dd0052168000f1bf2f0081006100ac
:10087c000100700050168800000000000080fa0093
:10088c00000006000200fa00004f780011479800a3
:10089c00a0a321008040eb00014878001e407800a6
:1008ac000004a2000004e00003003200e0cf80004e
:1008bc000080a000e0cf88001e4078000004e0001b
:1008cc000d0032001e4090000004e0000a003200cf
:1008dc00f103200050ae2000be8c0200000000008e
:1008ec0011012000a0192100be8c020000000000a4
:1008fc0006730200000000004100200040b22000fe
:10090c00be8c020000000000cb42a800c942a90026
:10091c003100200080b22000328c02000000000068
:10092c00501680004a00de00614060000080fb0031
:10093c0000f0a7000000ea000000ea004f00de0013
:10094c000040780011c0b3003a010700cb42a90067
:10095c00c942a800c222a800c022a9008100200020
:10096c00b0b22000328c0200000000001016800093
:10097c000000d100614060000080fb0000f0a70087
:10098c000000ea000000ea004f00de0000407800a2
:10099c0011c0b30027010700c222a900c962a80038
:1009ac00cb62a9008100200030b32000328c020001
:1009bc0000000000501680004b00de00614060001b
:1009cc000080fb0000f0a7000000ea000000ea0035
:1009dc004f00de000040780011c0b3001501070085
:1009ec00cb62a900c962a90081002000b0b320002d
:1009fc00328c020000000000501680004b00de001c
:100a0c00614060000080fb0000f0a7000000ea00dd
:100a1c000000ea004f00de00004078008040eb0050
:100a2c0004010700c002a900c202a8002000200097
:100a3c008a8b0200000000004100200030b420002e
:100a4c00328c02000000000010168000004078007c
:100a5c00614060000080fb0000f0a7000000ea008d
:100a6c000000ea004f00de000040780011c0b30027
:100a7c00f0000700e100200070b42000be8c0200e2
:100a8c000000000021e3a8002100200050b5200048
:100a9c00328c02000000000072352000712b200007
:100aac0090002000820007001e4090000004e0002f
:100abc00080032003100200070b52000328c02009a
:100acc000000000072352000712b2000b0002000c7
:100adc007700070041002000a0b52000328c0200f6
:100aec000000000002252000011b2000a0002000b7
:100afc006f0007001e4090000004e0000800320068
:100b0c0031002000e0b52000328c02000000000013
:100b1c0002252000011b2000c000200064000700fb
:100b2c0021e3a9008100200010b62000be8c020039
:100b3c000000000041168000f0c32f000080600010
:100b4c004016880061168000003c200001007000f7
:100b5c0060168800400620008a8b0200000000000e
:100b6c0010c0b30073000700a100200090b6200055
:100b7c00be8c02000000000061168000f0c32f0044
:100b8c0000806000601688001e4090000004e000a9
:100b9c0002003200c962a800cb62a9004006200006
:100bac008a8b0200000000000040eb00610007008f
:100bbc001e4090000004e0000d003200a100200057
:100bcc0030b72000be8c02000000000041168000ef
:100bdc00003c2000010070004016880040062000f8
:100bec008a8b02000000000010c0b3005100070007
:100bfc001e4078000004e000180032001e409000f7
:100c0c000004e00015003200c002a900c202a800d6
:100c1c00201680000010a000201688000102200081
:100c2c00d0b72000be8c020000000000f1002000b4
:100c3c00b0182100be8c02000000000006730200f8
:100c4c000000000021168000d0ff2f000080600003
:100c5c0020168800c002a900c202a900128a020054
:100c6c000000000061002000d0b92000328c02008e
:100c7c0000000000a0a32100104078008470020046
:100c8c00000000008100200030ba2000be8c020061
:100c9c0000000000e0cf80000080a100e0cf8800c1
:100cac00a0a32100104078000080fa00000006008c
:100cbc000800fa00100798002107980032079800e6
:100ccc0080c2b3002c730200000000001e009000d4
:100cdc00568a020000000000000f78001e00780009
:100cec00827102000000000090c2b3002c7302005d
:100cfc00000000002e0090009e007800808f5000b5
:100d0c00060036003e0090009e007800808f500058
:100d1c000200310010002000010037000000eb0041
:100d2c000040780011c0b300420007000080fa00b8
:100d3c00000006000200fa00004f7800410020007d
:100d4c00b0ba2000328c0200000000005016800067
:100d5c004900de00614060000080fb0000f0a7004d
:100d6c000000ea000000ea004f00de0000407800be
:100d7c009e4078002f00070031002000f0ba2000c0
:100d8c00328c020000000000501680004800de008b
:100d9c00614060000080fb0000f0a7000000ea004a
:100dac000000ea004f00de00004078009e40780012
:100dbc00200007004100200020bb2000328c0200e4
:100dcc0000000000501680004700de00614060000b
:100ddc000080fb0000f0a7000000ea000000ea0021
:100dec004f00de00004078009e40780011000700a4
:100dfc002100200060bb2000328c020000000000ab
:100e0c00501680004600de00614060000080fb0050
:100e1c0000f0a7000000ea000000ea004f00de002e
:100e2c00004078009e407800020007000080fa0025
:100e3c00000006000200fa00004f780011479800ed
:100e4c001e4090009e40780080cf500005003a0074
:100e5c003100200080bb2000be8c0200000000008e
:100e6c000900370051002000b0bb2000be8c0200ee
:100e7c0000000000a0a32100104078008040e80092
:100e8c00a0a32100014878000080fa0000000600b1
:100e9c000000fa0041168000007c20000100700068
:100eac00401688001400070020c0b300270007007c
:100ebc000100370000000000367202000000000044
:100ecc000004e00005003200067302000000000080
:100edc001e0007000004e00004003a00fd000700bb
:100eec000004e000f3ff32000100370000000000b6
:100efc000080fa00000006000000fa00c222a900df
:100f0c006820ef006a20ef006020ef006220ef0005
:100f1c001e21ef006005800000c0a10000d0a100e0
:100f2c0000e0a100600588001c21ef000064200097
:100f3c00d00888000000210030d188000000eb00b0
:100f4c0010d188000080fa00000006000e00fa00a4
:100f5c00404f9800e4004700020009008018eb00a5
:100f6c008058eb0020d18000e10f50003e00320091
:100f7c00e10f500003003900e20f50004600320030
:100f8c00d10037004e4890000080fb00e20f50006b
:100f9c0011003200e20f500005003c000000e000a0
:100fac000a003200e10f500010003200240037001c
:100fbc00f10f500021003200f30f50001f003200df
:100fcc00e40f5000180032001d003700caff070064
:100fdc0010c0b300bd00370041002000f0b628005f
:100fec00d06d0200000000001e003700c222a800d5
:100ffc001e21ef001621ef001421ef001e61a80046
:10100c008660a9009660a9006005800000c0a00061
:10101c0000d0a10000e0a1006005880010002000b5
:10102c0010d188000f00370051012000a0b5280016
:10103c00d06d0200000000000a00370009003700e4
:10104c004e4990004247980040c0b300104f9800a2
:10105c000040eb00204f98001000200020d18800a9
:10106c0000000000980037002e4890000040e80077
:10107c00204f98002e4890000080fb000000470095
:10108c00ce49900043409800ae4890001e48900016
:10109c0080cf50008b0039004e4090000080fb0048
:1010ac0011082000810f50003b0032001108200075
:1010bc00810f500004003c0001082000810f5000fb
:1010cc00450032007c00370021082000810f5000c1
:1010dc0074003200010c2000810f500076003a00a1
:1010ec005e4090000080fb00700060000000e0009b
:1010fc0003003200100380000000a00010038800e1
:10110c005e4090000080fb00680060000000e00082
:10111c000400320011038000000220000100700066
:10112c00100388005e4090000080fb0064006000ab
:10113c000000e000040032001103800000042000d5
:10114c0001007000100388005e4090000080fb00de
:10115c00620060000000e000040032001103800017
:10116c000008200001007000100388005e40900011
:10117c000080fb0061006000004078000004e0008b
:10118c004a003200110380000010200001007000a2
:10119c0010038800480037006e4090000080fb0070
:1011ac00c800dd005e4090000080fb000080400025
:1011bc000000e8004200dd0030d1880031d1800011
:1011cc0000002100808f50003a0036000000210002
:1011dc0030d18800380037007e4090000080fb0042
:1011ec008000eb00c001dd00020020006e4090008a
:1011fc000082fb008002eb004828dd00c820de00e6
:10120c00810070004820dd0002014000838148000d
:10121c005e4090000080fb008000eb00020040006c
:10122c008380480061014000e08148004218dd00e5
:10123c00ce10de00810070004210dd009201200013
:10124c00030020008606020000000000008fbe0094
:10125c001e01be000001200001002000800f510083
:10126c00818f59000500360002ff2f00f3ff2f007d
:10127c001e0f41005e97490003003700100020004c
:10128c0001002000008fbe001e00be004008de00e2
:10129c0000007800e00888001e007800d008880064
:1012ac0005003700000000000300370000000000bc
:1012bc0001003700000000000000eb0020d1880086
:1012cc0001003700000000000040eb000080fa0035
:1012dc00000006000200fa0010d18000e10f50005f
:1012ec0030003a0030048000680060000000e0002c
:1012fc0003003a00100380000000e0002b003a00cd
:10130c001fe1a8008780a9000000eb00000f780007
:10131c000e00370080cf80001e0040005116800068
:10132c00c608de008140780001487800000000000b
:10133c003104800000002100008060000000e0000b
:10134c00fbff32008780a9001e0fe80030d180001f
:10135c009e007800808f5000eeff39006220ef0075
:10136c001e21ef0031d18000010f780007003700fb
:10137c0081cf80001e00e900008040001040780002
:10138c002c730200000000001e0fe9001e00780004
:10139c000000e000f6ff3a00d7fe070010c0b300d3
:1013ac0004003700000000000100370000000000be
:1013bc000040eb000080fa00000006000000fa007c
:1013cc00819c2100114078000040a10080487800e9
:1013dc00609b21008040eb0001487800819c21003b
:1013ec00114078000020a10080487800819c2100e9
:1013fc00114078000000a1000010a1008048780086
:10140c00819c2100114078000030a10080487800b8
:10141c000080fa00000006000000fa00c922a800b3
:10142c00c902a800c8e2a800c8c2a800c942a80006
:10143c00c222a900c022a9005136800000fe2f0054
:10144c0000806000503688000000eb00b0cf8800b0
:10145c00daff0700cb62a900c962a900c002a9008b
:10146c00c202a9002d83a9002d43a9002d23a90098
:10147c002d63a900001980000050a0000060a0009e
:10148c000070a000001988003023ef0020f021002c
:10149c00201988002223ef000080fa0000000600cb
:1014ac000200fa00000f78009e00780041198800b5
:1014bc002023a8002003a9000000000000198000d0
:1014cc00610060000000e000fcff320000188000aa
:1014dc000080fa00000006000000fa0021e3a800da
:1014ec00c0002000eeff0700827102000000000027
:1014fc0021e3a9000080fa00000006000200fa00b7
:10150c00e1002000e0352000be8c0200000000004d
:10151c00f1002000b0182100be8c02000000000079
:10152c00f1002000c0362000328c020000000000c8
:10153c000000eb008271020000000000110020008e
:10154c00b0372000328c0200000000000f00370082
:10155c0021e3a800c0002000d1ff0700000f780095
:10156c0021e3a90020b82800f26d02000000000061
:10157c001e007800827102000000000011002000a3
:10158c00b0372000328c02000000000036720200de
:10159c00000000000004e000edff320006730200c2
:1015ac000000000080b82800166e02000000000049
:1015bc000080fa00000006000200fa00000f78001c
:1015cc00709b210010407800ef4f500007003e0048
:1015dc00709b2100104078000080fb006f00100011
:1015ec00f1ff27000088de001e0f6000a0cf8000f6
:1015fc00e10f500014003200e10f500005003900db
:10160c00e20f50001e003200e30f50002d0032009c
:10161c003b003700809c2100104078000042b20053
:10162c000004e000040032001e0078003e7102004d
:10163c0000000000320037001e007800ec70020041
:10164c00000000002e003700809c21001040780024
:10165c000042b2000004e000040032001e007800da
:10166c001c70020000000000250037001e007800ee
:10167c000040780084700200000000002000370059
:10168c00809c2100104078000042b2000004e00071
:10169c00070032001e00780000407800426e020005
:1016ac000000000000c2b3002c7302000000000018
:1016bc001e00780000407800426e0200000000001e
:1016cc000f003700809c2100104078000042b200cf
:1016dc000004e000050032001e0078004800de0027
:1016ec00004078002c730200000000001e007800ff
:1016fc00004078002c730200000000000000000085
:10170c000080fa00000006000400fa0010079800a0
:10171c000000eb00000f780009003700a00f20003c
:10172c000d000700a00f20000b000700a00f2000e9
:10173c0009000700a00f2000070007001e0fe8009b
:10174c001e0090009e007800808f5000f3ff39003f
:10175c000080fa00000006000400fa001007980050
:10176c000000eb00000f78001100370000000000b3
:10177c00000000000000000000000000000000005d
:10178c00000000000000000000000000000000004d
